:04000000ABEF00F072
:100008005682D9CF08F0DACF09F0899289940F0186
:1000180012A918D08EA802D083A20ED0899425EEFA
:1000280004F0010EDBBE07D0DB5003E1020EDE5CFC
:1000380002E3899201D089828EB883B201D0898483
:1000480012997DD012A17BD08EB883B28992901C70
:100058000A6E8E1C0B6E04C50CF005C50DF00DBEA6
:1000680003D0020E0D5C2FE28EA802D083A22BD003
:100078000C4A0D2A0CC004F50DC005F502C50CF09C
:1000880003C50DF0060E0C24D96E050E0D20DA6E90
:100098000AC0DFFF060E0C24D96E070E0D20DA6E9B
:1000A8000BC0DFFF0C4A0D2A0468010E056E0CC058
:1000B80006F00DC007F0045006160550071606C0D6
:1000C80002F507C003F58EB883B2898489848EA0AF
:1000D800FED78EA802D083A202D0899401D0898449
:1000E8000BA81FD00BD0838202D0838405D08394C1
:1000F80018D083A216D08394839213D00A507F0B12
:10010800046E056A05500DE10450040AF2E0100A75
:10011800F0E0340AE8E01F0AEFE07F0AE6E01F0A91
:10012800E6E025EE04F0010EDBBE06D0DB5002E16E
:10013800DE0402E3899201D089820F0112910E0137
:10014800CA9909C0DAFF08C0D9FF5692110089EF91
:1001580052F07DC0D9FF7EC0DAFFDE6ADD6A7CC05E
:100168000EF0CCEC4AF00EC098F00FC099F00001E8
:1001780099BF0B0CD8909835D96E9935DA6E4E0E1A
:10018800D926010EDA22DECFAFF0DDCFB0F0AF51C5
:10019800B01101E10C0C7DC0D9FF7EC0DAFFAFC001
:1001A800DEFFB0C0DDFF7F91AFC0D9FFB0C0DAFF7E
:1001B800DF5012E020EE01F0AF51D926B051DA221B
:1001C800DF50D0EC67F00001A46FA4B105D07F51D7
:1001D800D8A4A4A5000C0A0CAFC0D9FFB0C0DAFFA0
:1001E800DF6A20EE01F0AF51D926B051DA2298C06B
:1001F800DFFF20EE01F0AF51D926B051DA22DF50EF
:100208006DEC47F00001A46FA4B1030C7F5102E02C
:10021800A4B50A0CAFC060F0B0C061F0636B626B4C
:1002280067EC4BF060C0ADF061C0AEF0040EAD19E4
:10023800AE1101E1010CAE5103E1020EAD5D01E327
:100248000D0C20EE2BF0AF51D926B051DA22DECFBB
:10025800A0F0DECFA1F0DECFA2F0DECFA3F03A0E01
:10026800AF250E6E000EB0210F6EE5EC65F0020EA4
:100278000F180E1001E00D0C450E0001AF250E6E93
:10028800000EB0210F6EE5EC65F00EC0A9F00FC0AE
:10029800AAF00001AB6BAC6BA951AA11AB11AC1160
:1002A80010E1530EAF250E6E000EB0210F6ED5EC87
:1002B80059F00EC0A9F00FC0AAF010C0ABF011C0E1
:1002C800ACF0000120EE17F0AF51D926B051DA2278
:1002D800A9C0DEFFAAC0DEFFABC0DEFFACC0DEFFF8
:1002E80020EE3FF0AF51D926B051DA2210EE02F0DD
:1002F800AF51E126B051E222DFCFE7FF20EE02F056
:10030800AF51D926B051DA22DE040AE020EE02F01D
:10031800AF51D926B051DA22020EDE1801E00D0CD9
:10032800A9C00EF0AAC00FF0ABC010F0ACC011F01D
:1003380020EE02F0AF51D926B051DA22DF50126E0A
:10034800136A146A156A33EC5EF00EC0A9F00FC088
:10035800AAF010C0ABF011C0ACF020EE3CF0AF51E9
:10036800D926B051DA22DF50806F816B20EE09F078
:10037800AF51D926B051DA2280C0DEFF81C0DDFF3F
:1003880020EE09F0AF51D926B051DA22DE50DE1046
:10039800D8B40D0C20EE09F0AF51D926B051DA22AD
:1003A800DECF80F0DDCF81F08269836920EE09F02D
:1003B800AF51D926B051DA22DECF84F0DDCF85F0F7
:1003C8008251842783518523805184178151851751
:1003D8008451851101E00D0C400EAF250E6E000E04
:1003E800B0210F6EE5EC65F0000120EE07F0AF518B
:1003F800D926B051DA220EC0DEFF0FC0DDFF20EE95
:1004080007F0AF51D926B051DA22DF50806F0F0EB6
:10041800801701E00D0C420EAF250E6E000EB021C4
:100428000F6EE5EC65F00EC09CF00FC09DF000016A
:100438009E6B9F6B9C519D119E119F1110E14F0E59
:10044800AF250E6E000EB0210F6ED5EC59F00EC020
:100458009CF00FC09DF010C09EF011C09FF03D0EA3
:100468000001AF250E6E000EB0210F6EE5EC65F0B1
:100478000EC09AF00FC09BF000019A519B1101E148
:100488000D0C20EE07F0AF51D926B051DA22DECF9D
:1004980080F0DDCF81F0040E826FD89081338033F5
:1004A800822FFBD79A518025836F9B518121846FBE
:1004B800856BD8B0852B866BA9518325946FAA517B
:1004C8008421956FAB518521966FAC518621976F2A
:1004D80094519C5D95519D5996519E5997519F599C
:1004E80001E20D0C94519C5D0E6E95519D590F6E55
:1004F80096519E59106E97519F59116E20EE09F032
:10050800AF51D926B051DA22DECF80F0DDCF81F0AD
:1005180080C012F081C013F0146A156AF0EC5EF026
:100528000EC0A5F00FC0A6F010C0A7F011C0A8F02B
:100538000001A551A611A711A81101E10D0CAD6B81
:10054800AE6BF60EA55DFF0EA659FF0EA7590F0E4E
:10055800A85903E2AE6B030EAD6FA851A71108E1CD
:10056800F60EA55DFF0EA65903E2AE6B020EAD6F47
:10057800A851A71108E1F60EA55D0F0EA65903E2D2
:10058800AE6B010EAD6FAD51AE1101E10D0C020E57
:10059800A525806F000EA621816F000EA721826F0E
:1005A800000EA821836F20EE13F0AF51D926B05169
:1005B800DA2280C0DEFF81C0DEFF82C0DEFF83C09A
:1005C800DEFF20EE1BF0AF51D926B051DA22A0C0D1
:1005D800DEFFA1C0DEFFA2C0DEFFA3C0DEFF9A518E
:1005E800A025806F9B51A121816F000EA221826FEF
:1005F800000EA321836F20EE1FF0AF51D926B05112
:10060800DA2280C0DEFF81C0DEFF82C0DEFF83C049
:10061800DEFF9451A025806F9551A121816F9651DD
:10062800A221826F9751A321836F20EE27F0AF514B
:10063800D926B051DA2280C0DEFF81C0DEFF82C039
:10064800DEFF83C0DEFF030EAD19AE114DE1590E7A
:10065800AF250E6E000EB0210F6EE5EC65F00E5062
:100668000F1001E00D0C000120EE07F0AF51D92664
:10067800B051DA22DE50DE1001E00D0C5B0EAF2522
:100688000E6E000EB0210F6ED5EC59F0000120EE71
:1006980023F0AF51D926B051DA220EC0DEFF0FC0C9
:1006A800DEFF10C0DEFF11C0DEFF20EE13F0AF51F9
:1006B800D926B051DA22DECF80F0DECF81F0DECF4E
:1006C80082F0DECF83F0020ED890803781378237F0
:1006D8008337E82EF9D780C090F081C091F082C0AE
:1006E80092F083C093F0B8D020EE07F0AF51D9262E
:1006F800B051DA22DE50DE1001E10D0C20EE1FF0C1
:10070800AF51D926B051DA22DECF80F0DECF81F0AA
:10071800DECF82F0DECF83F0A9518025846FAA5105
:100728008121856FAB518221866FAC518321876F00
:1007380020EE23F0AF51D926B051DA2284C0DEFF73
:1007480085C0DEFF86C0DEFF87C0DEFF020EAD1962
:10075800AE116BE020EE13F0AF51D926B051DA227A
:10076800DECF80F0DECF81F0DECF82F0DECF83F007
:10077800010E8015846F856B866B876B20EE13F0F6
:10078800AF51D926B051DA22DECF88F0DECF89F01A
:10079800DECF8AF0DECF8BF0030E8803F3CF8CF028
:1007A800F4CF8DF08E6B8F6B8903F3508D27F45047
:1007B8008E23000E8F238803F3508D27F4508E2349
:1007C800000E8F23030E8A03F3508E27F4508F23D5
:1007D800000E8903F3508E27F4508F23000E8803F0
:1007E800F3508E27F4508F23030E8B03F3508F277B
:1007F800000E8A03F3508F27000E8903F3508F27CA
:10080800000E8803F3508F27D8908F338E338D33A3
:100818008C3384518C25906F85518D21916F865131
:100828008E21926F87518F2116D020EE13F0AF5191
:10083800D926B051DA22DECF80F0DECF81F0DECFCC
:1008480082F0DECF83F0D8908035906F8135916F3C
:100858008235926F8335936FFF0E9025806F010E5E
:100868009121816F000E9221826F000E9321836F78
:100878000A0E05D0D8908333823381338033E82E33
:10088800F9D720EE17F0AF51D926B051DA228051AE
:10089800DE5C8151DE588251DE588351DE5801E218
:1008A8000D0C20EE0FF0AF51D926B051DA22DE68D8
:1008B800DE68DE68DD68DD52DD5210EE0BF0AF5108
:1008C800E126B051E222DECFE6FFDECFE6FFDECF43
:1008D800E6FFDECFE6FF20EE04F0AF51D926B05197
:1008E800DA22800EDF6E030EAD19AE1101E090D052
:1008F8005F0EAF250E6E000EB0210F6EE5EC65F0B1
:100908000E040F1001E084D0AFC03AF0B0C03BF045
:10091800010E0001A0253C6E000EA1213D6E000EC7
:10092800A2213E6E000EA3213F6E18EC5BF0000979
:100938006FE1000120EE04F0AF51D926B051DA2260
:10094800DF6A2D0EAF250E6E020EB0210F6EE5EC9C
:1009580065F0550E0E185CE1AA0E0F1859E12F0E1E
:100968000001AF250E6E000EB0210F6ED5EC59F0C8
:10097800520E0E184DE1520E0F184AE1610E101872
:1009880047E1410E111844E1130E0001AF250E6E28
:10099800020EB0210F6ED5EC59F0720E0E1838E128
:1009A800720E0F1835E1410E101832E1610E111860
:1009B8002FE1170E0001AF250E6E020EB0210F6E4B
:1009C800D5EC59F0000120EE0FF0AF51D926B05107
:1009D800DA220EC0DEFF0FC0DEFF10C0DEFF11C03E
:1009E800DEFF1B0EAF250E6E020EB0210F6ED5EC8A
:1009F80059F0000120EE0BF0AF51D926B051DA22A0
:100A08000EC0DEFF0FC0DEFF10C0DEFF11C0DEFF2C
:100A1800AFC0D9FFB0C0DAFFADC0DFFF01014C4B5A
:100A28004D2B000120EE05F0AF51D926B051DA2246
:100A38004CC1DEFF4DC1DDFF000C77C07AF078C0F5
:100A48007BF00101426B436B96D376C060F07A0E5F
:100A58000001616F79C062F06151D96EDA6ADECF48
:100A6800F6FFDDCFF7FFF86A000EF86E0800F550C4
:100A7800250AD8A45ED36151D96EDA6ADE2A000E3F
:100A8800DD220101446B456B4C6A4D6A4669476932
:100A980000016151D96EDA6ADECFF6FFDDCFF7FFCC
:100AA800F86A000EF86E0800F550640AD8B40FD042
:100AB8006151D96EDA6ADECFF6FFDDCFF7FFF86A4B
:100AC800000EF86E0800F550690AD8A47DD161516E
:100AD800D96EDA6ADE2A000EDD226251D96EDA6A30
:100AE800DF50DF2ADF2AD96EDA6ADECF65F0DDCF84
:100AF80066F0000E66BFFF0E676F686F696F6A6FFA
:100B08006B6F6C6F60C028F065C029F066C02AF072
:100B180067C02BF068C02CF069C02DF06AC02EF0B9
:100B28006BC02FF06CC030F029C041F02AC042F0F1
:100B38002BC043F02CC044F02DC045F02EC046F029
:100B48002FC047F030C048F048AE02D0010E01D0A7
:100B5800000E3F6E406A3F504010D8B410D0481E77
:100B6800471E461E451E441E431E421E416C000E73
:100B7800422243224422452246224722482201019A
:100B880047BF01D04C9247BF05D0475107E1460502
:100B9800D8B004D03C6A010E3B6E04D046C13BF08D
:100BA80047C13CF044C13DF045C13EF03F504010C4
:100BB800D8A402D04CA403D03D06D8A03E064A6A69
:100BC8001F0E496E0201976B6ED04906D8A04A06DF
:100BD800780E4924D96E020E4A20DA6E41C00EF012
:100BE80042C00FF043C010F044C011F045C012F0ED
:100BF80046C013F047C014F048C015F00A0E166E30
:100C0800176A186A196A1A6A1B6A1C6A1D6AD7EC7D
:100C18004EF00EC031F00FC032F010C033F011C0EA
:100C280034F012C035F013C036F014C037F015C0D8
:100C380038F031C020F033C021F030EC66F020509D
:100C4800300FDF6E3B06D8A03C063D06D8A03E0616
:100C580041C00EF042C00FF043C010F044C011F084
:100C680045C012F046C013F047C014F048C015F054
:100C78000A0E166E176A186A196A1A6A1B6A1C6ABB
:100C88001D6A2AEC4AF00EC041F00FC042F010C0B5
:100C980043F011C044F012C045F013C046F014C030
:100CA80047F015C048F04ABE1FD04A5003E1490436
:100CB800D8A01AD041504210431044104510461095
:100CC80047104810D8A481D73CBE05D03C5002E15B
:100CD8003B04D8B07AD73EBE07D03E5003E13D046E
:100CE800D8A002D04CB271D73F504010D8A402D03F
:100CF8004CA415D04906D8A04A063F504010D8A4A5
:100D080003D03A6A2B0E02D03A6A2D0E396E780E4D
:100D18004924D96E020E4A20DA6E39C0DFFF28C096
:100D28001DF0780E49241E6E020E4A201F6E3DC02B
:100D380020F03EC021F04CA008D01EC017F01FC004
:100D480018F01DC019F048EC66F021BE05D020C08F
:100D580025F021C026F002D0256A266A236A246A73
:100D68000AD0000E106E200E0F6E1DC011F0ACECF4
:100D78005DF0234A242A2550235C2450800A226EE1
:100D88002650800A2258D8A0ECD74CB008D01EC0F4
:100D980017F01FC018F01DC019F048EC66F01EC00F
:100DA8000EF01FC00FF0B7EC63F025500E241D6E37
:100DB80026500F201E6E1DC028F01EC029F028C026
:100DC80060F029C061F0CFD16151D96EDA6ADECF07
:100DD800F6FFDDCFF7FFF86A000EF86E0800F55051
:100DE800780AD8B40FD06151D96EDA6ADECFF6FF2F
:100DF800DDCFF7FFF86A000EF86E0800F550580AC4
:100E0800D8A46CD16151D96EDA6ADECFF6FFDDCF96
:100E1800F7FFF86A000EF86E0800F5CF75F061511B
:100E2800D96EDA6ADE2A000EDD226251D96EDA6ADC
:100E3800DF50DF2ADF2AD96EDA6ADECF63F0DDCF32
:100E480064F063C06DF064C06EF06F6B706B716BB3
:100E5800726B736B746B60C027F06DC028F06EC046
:100E680029F06FC02AF070C02BF071C02CF072C04E
:100E78002DF073C02EF074C02FF075C030F0010152
:100E880047BF01D04C9247BF05D0475107E14605FF
:100E9800D8B004D03A6A010E396E04D046C139F090
:100EA80047C13AF044C143F045C144F04CA804D0CE
:100EB800FE0E4326FF0E442228C03BF029C03CF01A
:100EC8002AC03DF02BC03EF02CC03FF02DC040F0B2
:100ED8002EC041F02FC042F0486A1F0E476E020133
:100EE800976B6DD04706D8A048060F0E3B14456E89
:100EF800466A46BE08D0465004E10A0E455CD8A0B2
:100F080002D0570E01D0300E4526000E4622BF0EE5
:100F1800316E32683050336E346A31503326325075
:100F28003422345005E11A0E335C02E2010E01D07E
:100F3800000E356E366A35503610D8B425D09F0E5F
:100F4800316E3268200E4510336E000E4610346E36
:100F58003150332632503422345005E11A0E335CB6
:100F680002E2010E01D0000E376E386A3750381091
:100F7800D8B40AD045C014F046C015F074EC63F03C
:100F880014C045F015C046F0780E4724D96E020EFD
:100F98004820DA6E45C0DFFF3906D8A03A06430676
:100FA800D8A04406040E316ED89042324132403205
:100FB8003F323E323D323C323B32312EF5D748BECD
:100FC80020D0485004E1020E475CD8A01AD03B500C
:100FD8003C103D103E103F10401041104210D8A464
:100FE80081D73ABE05D03A5002E13904D8B07AD751
:100FF80044BE07D0445003E14304D8A002D04CB209
:1010080071D74CA816D04706D8A04806780E4724B2
:10101800D96E020E4820DA6E30C0DFFF4706D8A02E
:101028004806780E4724D96E020E4820DA6E300E34
:10103800DF6E27C01DF0780E47241E6E020E482072
:101048001F6E43C020F044C021F04CA008D01EC041
:1010580017F01FC018F01DC019F048EC66F021BE4B
:1010680005D020C025F021C026F002D0256A266AC6
:10107800236A246A0AD0000E106E200E0F6E1DC05F
:1010880011F0ACEC5DF0234A242A2550235C24504F
:10109800800A226E2650800A2258D8A0ECD74CB07D
:1010A80008D01EC017F01FC018F01DC019F048EC7A
:1010B80066F01EC00EF01FC00FF0B7EC63F02550AD
:1010C8000E241D6E26500F201E6E1DC027F01EC058
:1010D80028F027C060F028C061F045D06151D96E72
:1010E800DA6ADECFF6FFDDCFF7FFF86A000EF86E9A
:1010F8000800F550250AD8A413D06151D96EDA6AD0
:10110800DE2A000EDD22000E106E250E0F6E60C066
:1011180011F0ACEC5DF00001616B010E606F23D043
:101128006151D96EDA6ADE2A000EDD22606B616BCE
:101138001AD06151D96EDA6ADECFF6FFDDCFF7FF3C
:10114800F86A000EF86E0800F5500F6E106A60C05D
:1011580011F0ACEC5DF000016151D96EDA6ADE2A5B
:10116800000EDD22D8D7000160510101422700019D
:101178006151010143237AC0F6FF7BC0F7FF0800E5
:10118800F55001E062D442C176F043C177F0120015
:101198004A6E496AD1D2090E4A1817E1525015E031
:1011A800496A8390496A010E516E53501E0D1B0EF9
:1011B800F324D96E020EF420DA6E200EDF6E030ED1
:1011C80001015F6F4E6A4F6A83904A5008E152509E
:1011D80006E0496A4F6A0A0EAAD0839025D3020E08
:1011E8004A1806E1525004E0496A4F6A140E9FD02B
:1011F8001F0E4A6438D0300E4A6035D0525033E062
:101208004A50E00F536E496A0F0E531805E15EC14C
:1012180051F001015E6B8DD25350220D0A0EF3245A
:10122800D96E030EF420DA6EDE50DE10DE10DE100A
:1012380003E0030E53647DD2536A010E516E53507E
:101248001E0D1B0EF324D96E020EF420DA6E5350D5
:101258001E0D1B0EF324E16E020EF420E26EE75021
:101268001009DF6E66D23F0E4A6428D0480E4A60E5
:1012780025D0525023E053501E0D000EF324D96E92
:10128800020EF420DA6E4A50C00FDF6E53501E0D66
:10129800000EF324D96E020EF420DA6EDF500CE053
:1012A80053501E0D1B0EF324D96E020EF420DA6E75
:1012B800100EDF6E010E516E496A3BD2480E4A1875
:1012C80007E1525005E0496A120E4F6EC00E2FD04A
:1012D800310E4A1806E1525004E00C0E4F6E1D0EF6
:1012E80012D2340E4A1806E1525004E04E6A4F6A90
:1012F800496A73D7350E4A1807E1525005E0496A22
:101308000D0E4F6EAC0E13D0370E4A1807E152502F
:1013180005E083800E0E4F6E750EF5D10D0E4A183E
:1013280008E1525006E0496A020E4F6EBC0E4E6E3E
:1013380054D7100E4A1806E1525004E0030E4F6EBF
:10134800E90EE1D1180E4A1806E1525004E0070EE2
:101358004F6E090ED8D13B0E4A1806E1525004E0F0
:101368000E0E4F6E7E0ECFD13E0E4A1801E05CD2B3
:10137800525001E159D20F0E4F6E3D0EC4D1535059
:101388001E0D010EF324D96E020EF420DA6E4AC047
:10139800DFFF030E4F6EEA0EB6D153501E0D020E3C
:1013A800F324D96E020EF420DA6E4AC0DFFF030E72
:1013B8004F6EEB0EA8D153501E0D030EF324D96EB9
:1013C800020EF420DA6E4AC0DFFF030E4F6EEC0EF9
:1013D8009AD153501E0D040EF324D96E020EF42038
:1013E800DA6E4AC0DFFF030E4F6EED0E8CD15350FC
:1013F8001E0D050EF324D96E020EF420DA6E4AC0D3
:10140800DFFF030E4F6EEE0E7ED153501E0D060EFB
:10141800F324D96E020EF420DA6E4AC0DFFF53506F
:101428001E0D050EF324D96E020EF420DA6EDF507D
:10143800266E26C027F0286A296A2A6A29C02AF057
:1014480028C029F027C028F0276A53501E0D040E23
:10145800F324D96E020EF420DA6EDF502B6E2BC007
:101468002CF02D6A2E6A2F6A2DC02FF02CC02EF07A
:101478002D6A2C6A53501E0D030EF324D96E020EEA
:10148800F420DA6EDF50306E30C031F0326A336AE1
:10149800346A31C034F0336A326A316A2C503124EC
:1014A800356E2D503220366E2E503320376E2F5029
:1014B8003420386E27503524396E285036203A6E3D
:1014C800295037203B6E2A5038203C6E53501E0D51
:1014D800060EF324D96E020EF420DA6EDF5039249A
:1014E8003D6E000E3A203E6E000E3B203F6E000E11
:1014F8003C20406E3DC041F03EC042F03FC043F04A
:1015080040C044F0456A44BE456845C046F045C001
:1015180047F045C048F053501E0D070EF324D96E0E
:10152800020EF420DA6E41C0DEFF42C0DEFF43C087
:10153800DEFF44C0DEFF45C0DEFF46C0DEFF47C019
:10154800DEFF48C0DEFF53501E0D1C0EF324D96E7B
:10155800020EF420DA6EDECF26F0DDCF27F026C0AB
:101568000EF027C00FF0106A116A126A136A146A23
:10157800156A53501E0D070EF324D96E020EF4207F
:10158800DA6EDECF28F0DECF29F0DECF2AF0DECF0C
:101598002BF0DECF2CF0DECF2DF0DECF2EF0DECF1D
:1015A8002FF028C016F029C017F02AC018F02BC059
:1015B80019F02CC01AF02DC01BF02EC01CF02FC043
:1015C8001DF066EC5DF00EC030F00FC031F010C0B9
:1015D80032F011C033F012C034F013C035F014C02B
:1015E80036F015C037F053501E0D070EF324D96E90
:1015F800020EF420DA6E30C0DEFF31C0DEFF32C0EA
:10160800DEFF33C0DEFF34C0DEFF35C0DEFF36C08C
:10161800DEFF37C0DEFF83904E6A4F6A05D1535014
:101628001E0D1A0EF324D96E020EF420DA6E4AC08B
:10163800DFFF070E4F6E0A0E66D053501E0D190EAF
:10164800F324D96E020EF420DA6E4AC0DFFF070ECB
:101658004F6E0B0E58D053501E0D180EF324D96E32
:10166800020EF420DA6E4AC0DFFF070E4F6E0C0E32
:101678004AD053501E0D170EF324D96E020EF420D3
:10168800DA6E4AC0DFFF55D04E6A4F6A516AA5D557
:101698004AC030F10F0E4F6E3E0E35D04AC031F1C0
:1016A8000F0E4F6E3F0E2FD04AC032F10F0E4F6E05
:1016B800400E29D04AC033F10F0E4F6E410E23D091
:1016C8004AC034F10F0E4F6E420E1DD04AC035F19C
:1016D8000F0E4F6E430E17D04AC036F10F0E4F6EE5
:1016E800440E11D04AC037F124D00C0E4F6E1E0E96
:1016F8000AD00C0E4F6E1C0E4E6E0A0E496E6DD53A
:101708000E0E4F6E760E4E6E8FD04E6A4F6A090ED1
:10171800496E838089D04A500CE053501E0D1B0E31
:10172800F324D96E020EF420DA6E080EDF6E010E75
:10173800516E4E6A4F6A51D54EC026F04FC027F001
:10174800275013E0030A15E0040A27E00B0A33E0E8
:10175800010A37E0030A3BE0010A42E01D0A5AE0A9
:101768000E0A5DE03B0A5EE05FD0265001E113D52A
:101778005BD02650E90A01E102D6030A01E10DD641
:10178800010A01E118D6070A01E123D6010A01E19D
:101798002ED6030A01E139D647D02650090A01E1BD
:1017A8003ED7030A01E149D7010A01E154D7070AE4
:1017B80001E15FD739D026501D0A97E0030A99E066
:1017C80033D02650480A01E127D7E40A2DD0265005
:1017D800750A96E0030A99E0080A01E155D724D072
:1017E80026503D0A01E154D7030A01E157D7010AFF
:1017F80001E15AD77F0A01E15DD7010A01E160D70B
:10180800030A01E163D7010A01E166D7070A01E18A
:1018180069D70AD02650C00A01E17DD705D02650E5
:101828002A0A02D026500F0A49501200A0C0B6F06A
:10183800A1C0B7F0A451D96EDA6ADE6ADD6A9EC02B
:101848000FF09FC010F0C60E116E7FEC59F000012A
:10185800B56FB5510AE120EE0FF09E51D9269F5180
:10186800DA22DF50B56FB55102E0B551120020EE13
:101878000EF09E51D9269F51DA22DFA2070C20EEE6
:1018880010F09E51D9269F51DA2210EE10F09E5189
:10189800E1269F51E222E6CFA9F0E6CFAAF0E6CFF3
:1018A800ABF0E6CFACF0A251A925AD6FA351AA21A8
:1018B800AE6F000EAB21AF6F000EAC21B06FDE50E3
:1018C800AD5DDE50AE59DE50AF59DE50B05901E380
:1018D800DFD220EE10F09E51D9269F51DA22DECFBA
:1018E800A5F0DDCFA6F0A51DA26FA61DA36FD0D2CF
:1018F80020EE10F09E51D9269F51DA22FF0EDE14F9
:10190800A56F010EDE14A66F000EDE14A76F000E81
:10191800DE14A86FA551A611A711A81101E0FDD1E9
:1019280020EE10F09E51D9269F51DA22DECFA5F085
:10193800DECFA6F0DECFA7F0DECFA8F00A0E05D0E6
:10194800D890A833A733A633A533E82EF9D7A969C9
:10195800AA6920EE09F0C651D926C751DA22DECF8E
:10196800ABF0DDCFACF0A951AB27AA51AC23A55100
:10197800AB15B86FA651AC15B96FB81101E091D08D
:1019880020EE10F09E51D9269F51DA22DE50DE104B
:10199800DE10DE101EE120EE06F09E51D9269F5182
:1019A800DA22DECFC0F0DECFC1F0DECFC2F0DECF6C
:1019B800C3F0C051C111C211C31127E19EC081F00B
:1019C8009FC082F0836B846B856B866B3BEC28F041
:1019D80014D09EC081F09FC082F020EE14F09E517A
:1019E800D9269F51DA22DECF83F0DECF84F0DECF16
:1019F80085F0DECF86F03BEC28F081C0C0F082C0D5
:101A0800C1F083C0C2F084C0C3F0C051C111C2117B
:101A1800C31101E141D2C005C111C211C31109E1CD
:101A280020EE0FF09E51D9269F51DA22020EDF6E6A
:101A3800020CC0290FE1C1290DE1C2290BE1C3291C
:101A480009E120EE0FF09E51D9269F51DA22010EAE
:101A5800DF6E010C20EE14F09E51D9269F51DA2238
:101A6800C0C0DEFFC1C0DEFFC2C0DEFFC3C0DEFFF4
:101A780020EE06F09E51D9269F51DA22DE50DE1064
:101A8800DE10DE100EE120EE06F09E51D9269F51A1
:101A9800DA22C0C0DEFFC1C0DEFFC2C0DEFFC3C0A5
:101AA800DEFF20EE18F09E51D9269F51DA2210EE63
:101AB8002BF0C651E126C751E222DE50E61812E1AA
:101AC800DE50E6180FE1DE50E6180CE1DE50E618AD
:101AD80009E1C6C027F0C7C028F02BEC48F0000980
:101AE80001E053D1C6C00EF0C7C00FF0000120EED0
:101AF80014F09E51D9269F51DA22DECF10F0DECFA6
:101B080011F0DECF12F0DECF13F0F2EC4FF00EC082
:101B1800BCF00FC0BDF010C0BEF011C0BFF0000196
:101B2800BC51BD11BE11BF1101E17AD7B851BC2714
:101B3800B951BD23000EBE23BF23A2C0A5F0A3C088
:101B4800A6F0090EA76FD890A633A533A72FFBD709
:101B5800A5C0BAF0A6C0BBF0BA51BB1101E1A2D032
:101B6800BA51B825A56FBB51B921A66F20EE09F06F
:101B7800C651D926C751DA22A551DE5CA651DE58D6
:101B880010E220EE09F0C651D926C751DA22DECF7D
:101B9800A5F0DDCFA6F0B851A55DBA6FB951A65929
:101BA800BB6FB6C01DF0B7C01EF0BCC01FF0BDC0F3
:101BB80020F0BEC021F0BFC022F0BAC023F0BBC0E5
:101BC80024F020EE01F0C651D926C751DA22DF50A1
:101BD80060EC56F0000901E0D8D00001BA51A56FB9
:101BE800BB51A66FA76BA86B20EE2BF0C651D92668
:101BF800C751DA22DECFA9F0DECFAAF0DECFABF0F4
:101C0800DECFACF0BC51A95DAD6FBD51AA59AE6F26
:101C1800BE51AB59AF6FBF51AC59B06FA551AD5D57
:101C2800A651AE59A751AF59A851B0592CE22F0E61
:101C3800C6250E6E000EC7210F6E20EE2BF0C65182
:101C4800D926C751DA22DECFA5F0DDCFA6F0BC51E8
:101C5800A55FBD51A65B090ED890A537A637E82E1B
:101C6800FBD7A551B625106EA651B721116E020EED
:101C7800136E126AD8EC63F020EE03F0C651D92631
:101C8800C751DA22DF6ABAC0A5F0BBC0A6F0090EB8
:101C9800D890A537A637E82EFBD7A5C0C4F0A6C0B4
:101CA800C5F0A7D020EE0AF09E51D9269F51DA221E
:101CB80010EE10F09E51E1269F51E222DE50E65CC4
:101CC800DE50E658DE50E658DE50E65818E3C6C047
:101CD80027F0C7C028F02BEC48F0000901E055D0E8
:101CE800000120EE2BF0C651D926C751DA22BCC01C
:101CF800DEFFBDC0DEFFBEC0DEFFBFC0DEFF20EEE0
:101D080018F09E51D9269F51DA22BCC0DEFFBDC013
:101D1800DEFFBEC0DEFFBFC0DEFFA569010EA66FF5
:101D280020EE10F09E51D9269F51DA22DECFA7F07F
:101D3800DDCFA8F0A551A717A651A817A7510008ED
:101D4800C46FA851D8A0E82A0208C56FC451A25D83
:101D5800C551A35904E2A2C0C4F0A3C0C5F0C6C0CF
:101D68003AF0C7C03BF020EE18F09E51D9269F519B
:101D7800DA22DECF3CF0DECF3DF0DECF3EF0DECF24
:101D88003FF018EC5BF0000902E000015AD60001B0
:101D9800A569010EA66F20EE10F09E51D9269F511D
:101DA800DA22DECFA7F0DDCFA8F0A551A717A651FC
:101DB800A817C6C0A9F0C7C0AAF0A751A927A8515B
:101DC800AA232F0EA9250E6E000EAA210F6EB6C0EB
:101DD80010F0B7C011F0C4C012F0C5C013F0D8ECB1
:101DE80063F020EE03F0C651D926C751DA22010E5E
:101DF800DF6EC451A25FC551A35BA451D96EDA6AE4
:101E0800C451DE26C551DD22C451B627C551B723BA
:101E180020EE10F09E51D9269F51DA22C451DE26B9
:101E2800C551DE22000EDE22DE2220EE10F09E5189
:101E3800D9269F51DA2210EE0AF09E51E1269F51D1
:101E4800E222DE50E65CDE50E658DE50E658DE5010
:101E5800E65820EE0AF0D8A020EE10F09E51D926C0
:101E68009F51DA22DECFB1F0DECFB2F0DECFB3F091
:101E7800DECFB4F020EE0AF09E51D9269F51DA2227
:101E8800B1C0DEFFB2C0DEFFB3C0DEFFB4C0DEFF0C
:101E9800A251A31101E02CD520EE0EF09E51D926B7
:101EA8009F51DA22000EDB8C000C0F6A0E6A8BEC55
:101EB80067F00101FA6F636B0F010D6B156B1D6BFA
:101EC800226B070E8C6E010E0101FB6F696B0F0E02
:101ED8000F01596F116B196B216B266B2E6B0E6BF3
:101EE800166B1E6B236B2B6B886889688A688A8ED1
:101EF800889088928382020E026EB7EC66F088940E
:101F08008384889C839C889E838E8B688968460E10
:101F180000019C6FF90E9D6FA40E9E6FFF0E9F6FC0
:101F2800A30EA06FFE0EA16F290EA26FFF0EA36F66
:101F3800ADEC67F08A988588FFEC65F0520E0001D9
:101F48009C6FFB0E9D6FFAC19EF09F6BADEC67F026
:101F58000101FA2901E1FA6B0F0EFA1765EC4FF04F
:101F68000101FA6F6A0E00019C6FFB0E9D6FFAC1AA
:101F78009EF09F6BADEC67F00400520E0101B16F4B
:101F88002B0EB06F000EE82EFED7B02FFCD7B12F66
:101F9800FAD700F0D250F00B0109D26ED09E0E0194
:101FA800C691CF0ECF16CF82CF80C2890F01138181
:101FB80013891489F28E0E01BA892BEC5FF0839293
:101FC8008394EDEC55F0EDEC55F0000E0E6E340EEA
:101FD80001EC63F0440E126EFF0E136EB3EC5EF06C
:101FE800A40E126EFF0E136EB3EC5EF0000E0E6EB2
:101FF800390E01EC63F08FA22FD0290E0101B16FC9
:10200800960EB06F7F0EE82EFED7B02FFCD7B12FFB
:10201800FAD7000E0E6E800E01EC63F0160E126EEB
:10202800FE0E136EB3EC5EF017D0580E00019C6FD5
:10203800FE0E9D6F8FCF9EF09F6BADEC67F0290E63
:102048000101B16F960EB06F7F0EE82EFED7B02F4C
:10205800FCD7B12FFAD704008FB2E7D783800400EA
:1020680049EC4EF00101B66FE2EC36F00101B66FB3
:10207800FB050EE167510CE1430E00019C6FFD0E5C
:102088009D6FADEC67F0020E0101676F220E666F5F
:10209800FB510EE167510CE1330E00019C6FFD0E00
:1020A8009D6FADEC67F0010E0101676F040E666F5E
:1020B800625102E0FDEC44F0CFC193FF04EC32F032
:1020C8006FEC58F0000E0E6E800E01EC63F0CCEC55
:1020D80066F0000E0E6E800E01EC63F00101FA51FD
:1020E8000F0D350EF324126E0D0EF420136EB3ECA3
:1020F8005EF0010169BF86EC49F00101B56BBA6B6E
:10210800000EB86F010EB76FB8BF05D0B85166E1C1
:10211800040EB75D63E20F0EB703F3CFB0F1F4CF4F
:10212800B1F1B803F350B127250EB0250E6E0E0E8F
:10213800B1210F6EB7EC63F00F5003E1030E0E5C94
:1021480049E3A00E00019C6FFD0E9D6F0F0E01016B
:10215800B703F3CFB0F1F4CFB1F1B803F350B1271F
:10216800250EB02500019E6F0E0E0101B121000160
:102178009F6FADEC67F0220E0101B703F3CFB0F10A
:10218800F4CFB1F1B803F350B127000EB025000128
:10219800CE6F030E0101B1210001CF6F0F0E0101B7
:1021A800B703F3CFB2F1F4CFB3F1B803F350B327C9
:1021B800250EB2250001D06F0E0E0101B3210001DA
:1021C800D16F030ED26F4AEC15F00101B66FB6510C
:1021D800B0EC62F00101B74BB82B96D7640502E169
:1021E800070E8C6E020E641901E036D10F01108BB8
:1021F800070E2D6F31D1849284948EA88994CBECEC
:1022080065F02150221001E1FBD0BAC1B4F1B90E3A
:102218000E6E010E0F6EF0EC5DF00101BA6FB9B9E8
:10222800BA9F69511CE0350EBA1907E1740E000116
:102238009C6FF90E9D6FADEC67F0320E00019C6F3C
:10224800FF0E9D6FBAC19EF09F6B0101010EB9A9E7
:10225800000E0001A06FA16BADEC67F004D06A0E10
:10226800E82EFED700D00101B9A931D0600EBA1905
:102278002EE15F0EB4192BE14C0E00019C6FFF0E8E
:102288009D6FADEC67F002500209026ED10E9C6F93
:10229800FE0E9D6F67C19EF09F6B66C1A0F0A16B9B
:1022A800ADEC67F02BEE35F067C1DFFF2BEE36F0B3
:1022B80066C1DFFF8384020E66EC5BF083940292B2
:1022C80001016C6B64EC67F00101BA6BC5D0FB517E
:1022D80047E0B951100B0001ED6F000EEE6F0101E0
:1022E800BA5128EC3CF0EDC0BBF1EEC0BCF1080ED1
:1022F8000101BB19BC1101E100F0070E0101BB1976
:10230800BC1102E150EC61F0BB05BC1102E126EC06
:1023180059F0020E0101BB19BC1102E15FEC3EF05D
:10232800030E0101BB19BC1104E14AEC2CF00101B8
:10233800B56F050EBB19BC1104E166EC40F0010154
:10234800B56F090EBB19BC1102E1CBEC58F00A0EAF
:102358000101BB19BC1101E07FD084EC54F07CD0A2
:10236800B9C121F0226ABA5112EC18F021C0BBF1B0
:1023780022C0BCF1070E0101BB19BC1102E1ECEC53
:1023880060F0020EBB19BC1102E1D8EC5FF0BB058E
:10239800BC1102E1BAEC1FF0030EBB19BC1102E13B
:1023A80042EC57F0040EBB19BC1102E10CEC65F0CD
:1023B800050EBB19BC1102E17CEC50F0060E0101C0
:1023C800BB19BC1102E1DAEC67F0080EBB19BC11AD
:1023D80002E170EC3FF0090EBB19BC1102E178EC88
:1023E80055F00A0E0101BB19BC1102E159EC64F069
:1023F8000C0E0101BB19BC112FE161EC35F02CD09A
:1024080065EC4FF00101636F645126E0FA516319DE
:1024180023E0838E000E0E6EC00E01EC63F0CCEC50
:1024280066F0000E0E6EC00E01EC63F0C60E126E62
:10243800FE0E136EB3EC5EF063C1FAF1000E0001FC
:102448006D6F030E6E6FB5EC64F0E2EC36F00101CF
:10245800625102E0FDEC44F08FB22ED0050E01016E
:10246800B5192AE0C8D6580E00019C6FFE0E9D6F64
:102478008FCF9EF09F6BADEC67F0290E0101B16F15
:10248800960EB06F7F0EE82EFED7B02FFCD7B12F77
:10249800FAD70400000E0E6EC00E01EC63F0CCEC0F
:1024A80066F0000E0E6EC00E01EC63F0540E126E54
:1024B800FF0E136EB3EC5EF08FB2D5D7090E010193
:1024C800B16F1E0EB06FE40EE82EFED7B02FFCD70A
:1024D800B12FFAD700F0839483920001B16BB26BED
:1024E800760EB36FF90EB46FB56B90EC5CF0B7D5A0
:1024F8009EC00FF09FC010F0BC0E116E7FEC59F01B
:102508000001BE6FBE5108E120EE0FF09E51D926A2
:102518009F51DA22DF50BE6FBE5102E0BE51120059
:1025280020EE0AF09E51D9269F51DA22A051DE5C96
:10253800A151DE58A251DE58A351DE5816E220EE12
:102548000EF09E51D9269F51DA22DFB20ED020EE2E
:102558000AF09E51D9269F51DA22DECFA0F0DECFB5
:10256800A1F0DECFA2F0DECFA3F020EE10F09E5156
:10257800D9269F51DA22DECFB4F0DECFB5F0DECF18
:10258800B6F0DECFB7F0B86BB96BBA6BBB6B20EEA9
:1025980010F09E51D9269F51DA22B8C0DEFFB9C08B
:1025A800DEFFBAC0DEFFBBC0DEFFA051A111A21141
:1025B800A31101E100D220EE09F0BC51D926BD518A
:1025C800DA22DECFA4F0DDCFA5F0A451A66FA55185
:1025D800A76FA86BA96B090ED890A637A737A8379D
:1025E800A937E82EF9D7A6C0BFF0A7C0C0F0A8C089
:1025F800C1F0A9C0C2F0B451B511B611B71101E1CB
:1026080096D0FF0EA0250E6EFF0EA1210F6EFF0EB5
:10261800A221106EFF0EA321116EBFC012F0C0C020
:1026280013F0C1C014F0C2C015F0F0EC5EF00EC09B
:10263800A4F00FC0A5F010C0A6F011C0A7F0FF0EBF
:102648000001B4250E6EFF0EB5210F6EFF0EB621E8
:10265800106EFF0EB721116EBFC012F0C0C013F08C
:10266800C1C014F0C2C015F0F0EC5EF00E500001CD
:10267800A45D0F50A5591050A6591150A75957E3FA
:10268800FF0EBF25A46FFF0EC021A56FFF0EC1214D
:10269800A66FFF0EC221A76FA41DA86FA51DA96F65
:1026A800A61DAA6FA71DAB6FFF0EB425AC6FFF0E5A
:1026B800B521AD6FFF0EB621AE6FFF0EB721AF6F1C
:1026C800A851AC15B06FA951AD15B16FAA51AE158F
:1026D800B26FAB51AF15B36F20EE10F09E51D926F3
:1026E8009F51DA22B0C0DEFFB1C0DEFFB2C0DEFF0C
:1026F800B3C0DEFF20EE10F09E51D9269F51DA229A
:10270800DE50A05FDE50A15BDE50A25BDD50A35B14
:1027180020EE14F09E51D9269F51DA22DECFC3F065
:10272800DECFC4F0DECFC5F0DECFC6F060D020EE3D
:1027380006F09E51D9269F51DA22DECFC3F0DECFB4
:10274800C4F0DECFC5F0DECFC6F0C351C411C51149
:10275800C6113FE19EC081F09FC082F0836B846BFD
:10276800856B866B3BEC28F081C0C3F082C0C4F057
:1027780083C0C5F084C0C6F0C305C411C511C61115
:1027880009E120EE0FF09E51D9269F51DA22020E60
:10279800DF6E020CC3290FE1C4290DE1C5290BE145
:1027A800C62909E120EE0FF09E51D9269F51DA2261
:1027B800010EDF6E010C20EE06F09E51D9269F51C6
:1027C800DA22C3C0DEFFC4C0DEFFC5C0DEFFC6C05C
:1027D800DEFF20EE14F09E51D9269F51DA22C3C0A5
:1027E800DEFFC4C0DEFFC5C0DEFFC6C0DEFFC351CA
:1027F800C411C511C61101E085D0DDD0BF51A05F5D
:10280800C051A15BC151A25BC251A35B20EE10F085
:102818009E51D9269F51DA22BF51DE26C051DE22B1
:10282800C151DE22C251DE2220EE0EF09E51D92681
:102838009F51DA22DFA220D09EC081F09FC082F093
:10284800C3C083F0C4C084F0C5C085F0C6C086F09C
:102858003BEC28F081C0C3F082C0C4F083C0C5F04F
:1028680084C0C6F0C351C411C511C6111BE1A06BC9
:10287800A16BA26BA36B50D09EC045F09FC046F0E1
:10288800C3C047F0C4C048F0C5C049F0C6C04AF04C
:1028980045EC30F045C0C3F046C0C4F047C0C5F0B1
:1028A80048C0C6F00001C32907E1C42905E1C529CC
:1028B80003E1C62901E176D7C651C511C41104E167
:1028C800020EC35D01E25DD720EE13F0BC51D9269C
:1028D800BD51DA22DE50C35DDE50C459DE50C55901
:1028E800DE50C65901E34DD720EE14F09E51D9268B
:1028F8009F51DA22C3C0DEFFC4C0DEFFC5C0DEFFC1
:10290800C6C0DEFFA051BF5DA151C059A251C15937
:10291800A351C25901E272D720EE10F09E51D92678
:102928009F51DA22A051DE26A151DE22A251DE22D9
:10293800A351DE22A051A46F010EA115A56FA66BAD
:10294800A76BA411A611A71136E0BCC00EF0BDC03C
:102958000FF0C3C010F0C4C011F0C5C012F0C6C05B
:1029680013F0F2EC4FF00EC0B8F00FC0B9F010C081
:10297800BAF011C0BBF00001B851B911BA11BB11BE
:1029880001E1FFD6A0C0A4F0A1C0A5F0A2C0A6F0A6
:10299800A3C0A7F00A0E05D0D890A733A633A53355
:1029A800A433E82EF9D7A451B827A551B923A651C5
:1029B800BA23A751BB2320EE10F09E51D9269F5170
:1029C800DA2210EE0AF09E51E1269F51E222DE50F3
:1029D800E65CDE50E658DE50E658DE50E6581CE26B
:1029E80020EE10F09E51D9269F51DA2210EE0AF0FF
:1029F8009E51E1269F51E222DECFE6FFDECFE6FFC1
:102A0800DECFE6FFDECFE6FF20EE0EF09E51D926A0
:102A18009F51DA22000EDB8C20EE10F09E51D92651
:102A28009F51DA22FF0EDE14A46F010EDE14A56F8B
:102A3800000EDE14A66F000EDE14A76FA451A511B8
:102A4800A611A71101E16AD520EE18F09E51D926EA
:102A58009F51DA22B851DE180AE1B951DE1807E1B0
:102A6800BA51DE1804E1BB51DE1801E157D520EE5A
:102A780018F09E51D9269F51DA22B8C0DEFFB9C09E
:102A8800DEFFBAC0DEFFBBC0DEFF48D5CE51CF1196
:102A980001E1090C3F0ED217D00E7C6F810E7D6FBD
:102AA800010E7E6FD2C07FF0ADEC00F00101836FA4
:102AB800835101E0A8D281C184F182C185F1840EDD
:102AC8000001C06F010EC16FD0C0C2F0D1C0C3F009
:102AD800D7EC45F00101836F835104E1ABAF02D01D
:102AE800060E836FD2C0D3F01C0E0001D31701E18C
:102AF800D1D0010183510FE0040E831909E1840E3E
:102B08000001C46F010EC56F11EC58F00101836F0D
:102B18000001D2870DD088C1D3F0110E0001D31760
:102B280002E0070E03D0D2A503D0080E0101836F7F
:102B38000101835101E0BDD00001D2A7BAD081C103
:102B480015F082C116F09EC117F09FC118F065EC10
:102B58005FF015C071F116C072F117C073F118C09B
:102B680074F10E0E01019E250E6E000E9F210F6E50
:102B7800106A116A210E126E500E136EB6EC60F0D8
:102B8800010120EE0BF09E51D9269F51DA22200E2A
:102B9800DF6E81C112F082C113F09EC114F09FC193
:102BA80015F0166A176A186A196A39EC64F01C0E6F
:102BB80001019E250E6E000E9F210F6E106A116A8C
:102BC800126A136AB6EC60F0010120EE03F081513D
:102BD800D9268251DA22010EDF6E715172117311FA
:102BE800741167E020EE2BF08151D9268251DA2248
:102BF800DECF75F1DECF76F1DECF77F1DECF78F17B
:102C0800840E0001816F010E826F71C183F072C161
:102C180084F073C185F074C186F0876B886B896B0B
:102C28008A6BA4EC46F00101836F835142E181C1B4
:102C38003AF082C13BF075C13CF076C13DF077C1F6
:102C48003EF078C13FF018EC5BF00101836FFF0E96
:102C580071250001D36FFF0E010172210001D46FAD
:102C6800FF0E010173210001D56FFF0E01017421D0
:102C78000001D66F010120EE0BF08151D926825157
:102C8800DA22D3C0DEFFD4C0DEFFD5C0DEFFD6C057
:102C9800DEFF0FD0010183510CE188A902D0040E98
:102CA80007D00001D2A305D0010188A102D0070EE8
:102CB800836F0101835123E10001D2B7D28D010155
:102CC80020EE2BF08151D9268251DA22000110EE34
:102CD8001CF0CE51E126CF51E222DECFE6FFDECF57
:102CE800E6FFDECFE6FFDECFE6FF20EE20F0CE5196
:102CF800D926CF51DA229EC1DEFF9FC1DDFF010137
:102D0800835101E080D181C115F082C116F09EC1C6
:102D180017F09FC118F065EC5FF0000120EE06F097
:102D2800CE51D926CF51DA2215C0DEFF16C0DEFFFC
:102D380017C0DEFF18C0DEFF1C0E01019E250E6EB7
:102D4800000E9F210F6ED5EC59F0000120EE0AF01D
:102D5800CE51D926CF51DA220EC0DEFF0FC0DEFFDA
:102D680010C0DEFF11C0DEFFCEC0D9FFCFC0DAFF32
:102D780081C1DEFF82C1DDFF010120EE05F0815136
:102D8800D9268251DA22000110EE02F0CE51E12656
:102D9800CF51E222DECFE6FFDDCFE5FF20EE0EF0D9
:102DA800CE51D926CF51DA22D2C0DFFF20EE0FF064
:102DB800CE51D926CF51DA22DF6A20EE18F0CE5153
:102DC800D926CF51DA22DE6ADE6ADE6ADD6A20EEB3
:102DD80010F0CE51D926CF51DA22DE6ADE6ADE6AD9
:102DE800DD6AD2AB10D120EE0AF0CE51D926CF51F0
:102DF800DA22DE50DE10DE10DE1001E104D120EE12
:102E08000AF0CE51D926CF51DA2210EE10F0CE5169
:102E1800E126CF51E222DECFE6FFDECFE6FFDECFAE
:102E2800E6FFDECFE6FF010120EE09F08151D92649
:102E38008251DA22DECFD3F0DDCFD4F00001D351B6
:102E4800D56FD451D66FD76BD86B090ED890D537BC
:102E5800D637D737D837E82EF9D7D5C06DF1D6C0D1
:102E68006EF1D7C06FF1D8C070F120EE06F0CE51E8
:102E7800D926CF51DA22DECF7DF1DECF7EF1DECF4B
:102E88007FF1DECF80F120EE0AF0CE51D926CF5166
:102E9800DA22DECF79F1DECF7AF1DECF7BF1DECF39
:102EA8007CF132D0CEC045F0CFC046F07DC147F0AE
:102EB8007EC148F07FC149F080C14AF045EC30F04E
:102EC80045C07DF146C07EF147C07FF148C080F122
:102ED800010180517F117E1105E1020E7D5D02E244
:102EE800020E836F7D2908E17E2906E17F2904E12E
:102EF800802902E1010E836F6D51795F6E517A5B13
:102F08006F517B5B70517C5B0101835109E1795101
:102F18006D5D7A516E597B516F597C517059C2E37E
:102F2800000120EE14F0CE51D926CF51DA227DC10E
:102F3800DEFF7EC1DEFF7FC1DEFF80C1DEFF010153
:102F4800835161E179510001D36F010E01017A15B6
:102F58000001D46FD56BD66BD311D511D61153E0C0
:102F680081C10EF082C10FF07DC110F07EC111F059
:102F78007FC112F080C113F0F2EC4FF00EC075F172
:102F88000FC076F110C077F111C078F101017551C9
:102F980076117711781103E1020E836F34D079C16D
:102FA800D3F07AC1D4F07BC1D5F07CC1D6F00A0E3B
:102FB80006D00001D890D633D533D433D333E82E96
:102FC800F8D7010175510001D325D76F010176515A
:102FD8000001D421D86F010177510001D521D96FA3
:102FE800010178510001D621DA6F20EE18F0CE5198
:102FF800D926CF51DA22D7C0DEFFD8C0DEFFD9C02C
:10300800DEFFDAC0DEFF0101835106E0CEC0D9FF42
:10301800CFC0DAFFDE6ADD6A83511200276E2150C5
:10302800100B256E225002E06FEC58F0266A2550EE
:1030380001E120D2279E040E271802E1505003E137
:10304800140E271807E10101486B496B226A070E25
:10305800216E070C3F0E271807E1506A0101486BE3
:10306800496B216A226A12005F0E271807E10101E5
:103078005C6B486B496B216A226A12003F0E276419
:103088000BD05F0E276008D0400E271805E001011D
:103098005C6B216A226A1200400E27180AE1010EB1
:1030A80001015C6F506A0101486B496B216A226A11
:1030B8001200200E271801E0DDD1010E506EF3D763
:1030C800600E27180CE101015C5109E05A51080E05
:1030D800D8B4030E266E0101486B496B33D2600EDB
:1030E800271809E1505007E001015A5102E0090E82
:1030F800F1D7050EEFD7680E271809E1505007E001
:103108001A0E0101496F900E5FD183801BD2680EA1
:10311800271805E101015C5102E0020EDBD76A0EB7
:10312800271807E1505005E01A0E0101496FF40E07
:103138004BD16C0E271807E1505005E01A0E01011B
:10314800496F2C0E41D1700E271808E101015C511E
:1031580005E0040E266E486B496BD7D7700E27180A
:1031680001E0F0D1505001E1EDD11B0E0101496F92
:10317800620E2AD1838027500CE121AA05D0266A45
:103188000101486B496B83901A0E0101496FAF0E1C
:10319800486F020E271805E11A0E0101496F920EB9
:1031A800486F050E271805E11A0E0101496FAE0E8A
:1031B800486F070E271805E11A0E0101496FB80E6E
:1031C800486F080E271805E11A0E0101496FCC0E49
:1031D800486F030E271802E027280CE18380680E49
:1031E800236EE40EE82EFED7232EFCD700D0266AE5
:1031F800839071D7140E271805E11A0E0101496F43
:103208009E0E486F160E271801E09CD11A0E010178
:10321800496FA40ECAD0050E271805E11A0E010140
:10322800496FF50E486F080E271801E08BD11A0E6A
:103238000101496FCC0E486F010E5A6F83D127C028
:1032480053F01A0E0101496F950EAFD02750246E26
:10325800236A53500C0D000EF324D96E010EF4208E
:10326800DA6E23C0DEFF24C0DDFF1A0E0101496FAC
:10327800960E9BD02750236E246A53500C0D000ED7
:10328800F324D96E010EF420DA6E23C0DEFF24C0C9
:10329800DDFF1A0E0101496F970E87D053500C0DB0
:1032A800020EF324D96E010EF420DA6E27C0DFFF78
:1032B8001A0E0101496F980E78D053500C0D030E69
:1032C800F324D96E010EF420DA6E27C0DFFF010166
:1032D800486B496B010E37D01A0E0101496FB90EC0
:1032E80073D01A0E0101496FBA0E5FD01A0E010190
:1032F800496FBB0E486F240E00019C6FFE0E9D6F38
:10330800ADEC67F001015B6B486B496B55D001016F
:10331800486B496B240E00019C6FFE0E9D6FADEC4F
:1033280067F04AD0DC0E00019C6FFE0E9D6FADEC7D
:1033380067F00101486B496B010E586F3DD00101E0
:10334800486B496B060E266EFDD027C053F001016D
:10335800486B496B266A30D001015A6B1A0E496FC7
:10336800F70E486F29D01A0E0101496FF70E1DD0CC
:103378008390270E0101496F0F0E17D0180E2718DA
:1033880001E0E0D01A0E0101496F2D0E0ED01A0E81
:103398000101496F2E0E09D01A0E0101496F2F0E37
:1033A80004D01A0E0101496F300E486FCBD00101CD
:1033B800486B496B0A0E266E8390C4D0040E266EA5
:1033C800270E0101496F0F0E486F9FD683800101B8
:1033D80004D08390010E01015A6F486B496B266A2D
:1033E800B1D08390010E01015A6F486B496B266A70
:1033F80053500C0D000EF324D96E010EF420DA6E32
:10340800DE6ADD6A53500C0D020EF324D96E010EEC
:10341800F420DA6E2744E846030BDF6E53500C0D98
:10342800030EF324D96E010EF420DA6E27503F0BF9
:10343800DF6E8D0E00019C6FFC0E9D6F27C09EF005
:103448009F6B53500C0D020EF324D96E010EF4201D
:10345800DA6EDF50A06FA16B53500C0D030EF324EE
:10346800D96E010EF420DA6EDF50A26FA36BADECBB
:1034780067F068D048C123F049C124F0245007E020
:103488001A0A09E0010A54E03C0A5AE05BD02350CA
:1034980001E116D657D023502C0A01E16FD7010A53
:1034A80001E175D7030A01E177D7010A01E179D76C
:1034B8001F0A01E17CD7A00A01E15CD6020A01E1FA
:1034C800BED6070A01E1C2D6030A01E1D3D6010A32
:1034D80001E1E4D60F0A01E1F0D6060A01E122D79C
:1034E8003A0A01E12CD70A0A01E173D7010A01E17E
:1034F80078D7170A01E1F0D6010A01E1F2D6030AEA
:1035080001E1F4D6010A01E102D7790A01E105D601
:103518000E0A01E11AD7380A01E17DD6010A01E154
:103528001BD7030A01E11FD7010A01E121D70AD0FD
:103538002350580A01E142D73A0A01E147D702D09D
:1035480023500F0A26C021F0226A1200B30EF66E2D
:10355800F80EF76E0900F5CFE5F00A00F5CFE6F0B2
:103568000001E96BEC6B0101F06B030ECF6105D034
:103578009650CF19F00BCF1905D0CFC193FF9650B5
:10358800F00B0A09966ECD6ACE6A0FD1ED6B350E37
:10359800176E0B0E186EE50E196EFCEC5BF017C07B
:1035A800EAF018C0EBF0EAC0D9FFEBC0DAFF3B0E37
:1035B800DE1801E0F5D0F9D0ED5113E1EAC012F0C0
:1035C800EBC013F010EC60F00001EC6F800EEC65BE
:1035D80003D0EC51800FE96F030EE965D5D0E96B94
:1035E800D3D0ED0511E10101FA510001EC1903E016
:1035F8007F0EEC1909E1EAC012F0EBC013F010ECF1
:1036080060F00101676FC0D0020EED1911E10101F0
:10361800FA510001EC1903E07F0EEC1909E1EAC048
:1036280012F0EBC013F010EC60F00101666FACD043
:10363800020EED652CD0080EED6129D00101FA517A
:103648000001EC190CE07F0EEC1909E0810EEC1971
:1036580006E0820EEC1903E0830EEC1918E1E9513B
:10366800050DD10EF324E76F010EF420E86FEAC0D0
:1036780012F0EBC013F010EC60F00001C26FED51D6
:10368800E725C36F000EE821C46FFD0E5DD0070E5D
:10369800ED652CD01B0EED6129D00101FA51000116
:1036A800EC190CE07F0EEC1909E0810EEC1906E02C
:1036B800820EEC1903E0830EEC1918E1E951130DA1
:1036C800AA0EF324E76F030EF420E86FEAC012F0A5
:1036D800EBC013F010EC60F00001C26FED51E7256C
:1036E800C36F000EE821C46FF80E2ED01A0EED65D8
:1036F80033D0280EED6130D00101FA510001EC19E8
:103708000CE07F0EEC1909E0810EEC1906E0820E40
:10371800EC1903E0830EEC191FE1E9510D0D980E29
:10372800F324E76F020EF420E86FEAC012F0EBC052
:1037380013F010EC60F00001C26FED51E725C36F84
:10374800000EE821C46FE50EC325D96EFF0EC42113
:10375800DA6EC2C0DFFF18D0280EED1915E101019D
:10376800FA510001EC1903E07F0EEC190DE1F00E9F
:103778000E6E010E0F6EEAC010F0EBC011F0136A66
:10378800080E126EDFEC61F00001ED2B176A186A63
:10379800E50E196EFCEC5BF017C0EAF018C0EBF010
:1037A8000001EA51EB1101E007D7350E00019F6FC8
:1037B8000B0EA06FA26B910EA16F000EA36F030EEC
:1037C800A46F46EC5CF09F51A01101E0DFD6ED6BD1
:1037D800ED510D0DA20EF324D96E020EF420DA6E0F
:1037E800DF50C26FC2C0C3F0C46BC56BC66BC5C027
:1037F800C6F0C4C0C5F0C3C0C4F0C36BED510D0D15
:10380800A10EF324D96E020EF420DA6EDF50C76FD2
:10381800C7C0C8F0C96BCA6BCB6BC9C0CBF0C8C0F6
:10382800CAF0C96BC86BED510D0DA00EF324D96E0B
:10383800020EF420DA6EDF50CC6FCCC0CDF0CE6B28
:10384800CF6BD06BCDC0D0F0CF6BCE6BCD6BC851EA
:10385800CD25D16FC951CE21D26FCA51CF21D36F97
:10386800CB51D021D46FC351D125D56FC451D221AA
:10387800D66FC551D321D76FC651D421D86FED511A
:103888000D0DA30EF324D96E020EF420DA6EDF506C
:10389800D525D96F000ED621DA6F000ED721DB6F40
:1038A800000ED821DC6FD9C0DDF0DAC0DEF0DBC055
:1038B800DFF0DCC0E0F0E16BE0BFE169E1C0E2F01D
:1038C800E1C0E3F0E1C0E4F0ED511E0D0F0EF3246A
:1038D800D96E020EF420DA6EDDC0DEFFDEC0DEFF38
:1038E800DFC0DEFFE0C0DEFFE1C0DEFFE2C0DEFFDA
:1038F800E3C0DEFFE4C0DEFFED51130DAE0EF3248E
:10390800D96E030EF420DA6EDF50C36FC26BED512F
:10391800130DAF0EF324D96E030EF420DA6EDF50C8
:10392800C46FC56BC251C427C351C523ED511E0DC9
:103938001C0EF324D96E020EF420DA6EC4C0DEFF2A
:10394800C5C0DDFFED511E0D1C0EF324D96E020E0D
:10395800F420DA6EDECFC2F0DDCFC3F0C2C00EF0C5
:10396800C3C00FF0106A116A126A136A146A156AE2
:10397800ED511E0D0F0EF324D96E020EF420DA6EEF
:10398800DECFC4F0DECFC5F0DECFC6F0DECFC7F0A5
:10399800DECFC8F0DECFC9F0DECFCAF0DECFCBF085
:1039A800C4C016F0C5C017F0C6C018F0C7C019F0DB
:1039B800C8C01AF0C9C01BF0CAC01CF0CBC01DF0AB
:1039C80066EC5DF00EC0CCF00FC0CDF010C0CEF0AC
:1039D80011C0CFF012C0D0F013C0D1F014C0D2F093
:1039E80015C0D3F00001ED511E0D0F0EF324D96E52
:1039F800020EF420DA6ECCC0DEFFCDC0DEFFCEC0F2
:103A0800DEFFCFC0DEFFD0C0DEFFD1C0DEFFD2C0F8
:103A1800DEFFD3C0DEFF6A0E9C6FFA0E9D6FEDC00D
:103A28009EF09F6BED511E0D1C0EF324D96E020EF5
:103A3800F420DA6EDECFA0F0DDCFA1F0ADEC67F0B8
:103A4800ED2B030EED65C4D6D60E9C6FFA0E9D6F56
:103A5800F00E9E6F010E9F6FADEF67F076C091F08C
:103A680077C092F07AC0D9FF7BC0DAFFDE6ADD6AE0
:103A780074C00FF075C010F09D0E116E7FEC59F0F8
:103A880000018C6F8C510AE120EE0FF07451D92699
:103A98007551DA22DF508C6F8C5102E08C51120084
:103AA80020EE0EF07451D9267551DA22DFA0070CEA
:103AB80020EE10F07451D9267551DA22DECF7CF051
:103AC800DECF7DF0DECF7EF0DECF7FF020EE0AF095
:103AD8007451D9267551DA22DECF80F0DECF81F01D
:103AE800DECF82F0DECF83F07C51805D886F7D5120
:103AF8008159896F7E5182598A6F7F5183598B6FA3
:103B080078517C6F79517D6F7E6B7F6B7C51885DBE
:103B18007D5189597E518A597F518B5901E321D2B0
:103B280088C078F089C079F01CD220EE10F074516A
:103B3800D9267551DA22FF0EDE147C6F010EDE14D1
:103B48007D6F000EDE147E6F000EDE147F6F7C51D9
:103B58007D117E117F1101E083D120EE10F07451A8
:103B6800D9267551DA22DECF7CF0DECF7DF0DECFAC
:103B78007EF0DECF7FF00A0E05D0D8907F337E33FB
:103B88007D337C33E82EF9D78069816920EE09F00E
:103B98009D51D9269E51DA22DECF82F0DDCF83F007
:103BA80080518227815183237C518215936F7D51E7
:103BB8008315946F931166E120EE10F07451D926A5
:103BC8007551DA22DE50DE10DE10DE100FE120EE35
:103BD80006F07451D9267551DA22DECF8DF0DECF8A
:103BE8008EF0DECF8FF0DECF90F01CD074C045F0A1
:103BF80075C046F020EE14F07451D9267551DA22BA
:103C0800DECF47F0DECF48F0DECF49F0DECF4AF016
:103C180045EC30F045C08DF046C08EF047C08FF0BF
:103C280048C090F0000190518F118E110CE1020EE6
:103C38008D5D09E220EE0FF07451D9267551DA2214
:103C4800020EDF6E020C8D290FE18E290DE18F29FE
:103C58000BE1902909E120EE0FF07451D926755136
:103C6800DA22010EDF6E010C20EE14F07451D92611
:103C78007551DA228DC0DEFF8EC0DEFF8FC0DEFFF9
:103C880090C0DEFF9DC00EF09EC00FF020EE14F035
:103C98007451D9267551DA22DECF10F0DECF11F03B
:103CA800DECF12F0DECF13F0F2EC4FF00EC095F03D
:103CB8000FC096F010C097F011C098F00001955110
:103CC80096119711981101E1B5D793519527945101
:103CD8009623000E9723982378C07CF079C07DF056
:103CE800090E7E6FD8907D337C337E2FFBD77CC046
:103CF80099F07DC09AF099519A1101E1A3D0995198
:103D080093257C6F9A5194217D6F20EE09F09D5187
:103D1800D9269E51DA227C51DE5C7D51DE5810E2B4
:103D280020EE09F09D51D9269E51DA22DECF7CF093
:103D3800DDCF7DF093517C5D996F94517D599A6FD9
:103D480091C01DF092C01EF095C01FF096C020F0E3
:103D580097C021F098C022F099C023F09AC024F0AF
:103D680020EE01F09D51D9269E51DA22DF5029EC30
:103D78005AF0000901E0ACD0000120EE03F09D519B
:103D8800D9269E51DA22DF504EE099517C6F9A5124
:103D98007D6F7E6B7F6B20EE2BF09D51D9269E5157
:103DA800DA22DECF80F0DECF81F0DECF82F0DECF08
:103DB80083F09551805D846F96518159856F975135
:103DC8008259866F98518359876F7C51845D7D51E4
:103DD80085597E5186597F51875925E220EE2BF06F
:103DE8009D51D9269E51DA22DECF7CF0DDCF7DF0C1
:103DF80095517C5F96517D5B090ED8907C377D3755
:103E0800E82EFBD77C5191250E6E7D5192210F6EC5
:103E18002F0E9D25106E000E9E21116E020E136E40
:103E2800126AD8EC63F099C07CF09AC07DF0090E54
:103E3800D8907C377D37E82EFBD77CC09BF07DC0BF
:103E48009CF072D020EE18F07451D9267551DA2200
:103E580095C0DEFF96C0DEFF97C0DEFF98C0DEFF8C
:103E68007C69010E7D6F20EE10F07451D9267551D2
:103E7800DA22DECF7EF0DDCF7FF07C517E177D51D8
:103E88007F177E5100089B6F7F51D8A0E82A02084F
:103E98009C6F9B51785D9C51795904E278C09BF0E6
:103EA80079C09CF09DC03AF09EC03BF020EE18F01F
:103EB8007451D9267551DA22DECF3CF0DECF3DF0C1
:103EC800DECF3EF0DECF3FF018EC5BF0000902E0F9
:103ED8000001C1D691C00EF092C00FF000017C69BC
:103EE800010E7D6F20EE10F07451D9267551DA223B
:103EF800DECF7EF0DDCF7FF07C517E177D517F17BE
:103F08009DC080F09EC081F07E5180277F51812323
:103F18002F0E8025106E000E8121116E9BC012F0AD
:103F28009CC013F0D8EC63F09B51785F9C51795B8F
:103F38007AC0D9FF7BC0DAFF9B51DE269C51DD2277
:103F48009B5191279C51922320EE10F07451D92651
:103F58007551DA229B51DE269C51DE22000EDE22AC
:103F6800DE227851791101E0E0D5000C53500C0D98
:103F7800000EF324D96E010EF420DA6E0001C9692F
:103F8800CA6953500C0D080EF324E16E010EF4209B
:103F9800E26EE6CFCBF0E5CFCCF0C951CB27CA51C2
:103FA800CC23DE50CB5DCC51800ACD6FDE50800A29
:103FB800CD594AE353500C0D020EF324D96E010E6D
:103FC800F420DA6EDF50C76FC86BC969CA695350ED
:103FD8000C0D0A0EF324D96E010EF420DA6EDF50B0
:103FE800CB6FCC6BC951CB27CA51CC23C751CB5D02
:103FF800CC51800ACD6FC851800ACD5925E3535062
:104008000C0D030EF324D96E010EF420DA6EDF5086
:10401800C76FC86BC969CA6953500C0D0B0EF324DE
:10402800D96E010EF420DA6EDF50CB6FCC6BC9511C
:10403800CB27CA51CC23C751CB5DCC51800ACD6F59
:10404800C851800ACD5961E21F0E0101596F010E56
:104058005B6F83909D0E00019C6FF90E9D6F53500E
:104068000C0D000EF324D96E010EF420DA6EDECFAB
:104078009EF0DDCF9FF053500C0D080EF324D96E3F
:10408800010EF420DA6EDECFC7F0DDCFC8F0FF0EE8
:10409800C725A06FFF0EC821A16F53500C0D020E4B
:1040A800F324D96E010EF420DA6EDF50A26FA36BF1
:1040B80053500C0D0A0EF324D96E010EF420DA6E5B
:1040C800DF50C96FFF0EC925A46FA56BFF0EA5238E
:1040D80053500C0D030EF324D96E010EF420DA6E42
:1040E800DF50A66FA76B53500C0D0B0EF324D96E3F
:1040F800010EF420DA6EDF50CA6FFF0ECA25A86FD2
:10410800A96BFF0EA923ADEC67F053500C0D030EFD
:10411800F324D96E010EF420DA6EDF50C76FC7C0E2
:10412800C8F0C96BCA6BCB6BCAC0CBF0C9C0CAF0A8
:10413800C8C0C9F0C86B53500C0D0B0EF324D96ED0
:10414800010EF420DA6EDF50CC6FCCC0CDF0CE6B10
:10415800CF6BD06B53500C0D020EF324D96E010EA9
:10416800F420DA6EDF50D16FD1C0D2F0D36BD46BAC
:10417800D56BD4C0D5F0D3C0D4F0D2C0D3F0D26BB5
:10418800D251CD03F3CFD6F0F4CFD7F0D86BD96B9B
:10419800CE03F350D727F450D823000ED923D35198
:1041A800CD03F350D727F450D823000ED923D2518A
:1041B800CF03F350D827F450D923D351CE03F3506B
:1041C800D827F450D923D451CD03F350D827F4502D
:1041D800D923D051D203F350D927D351CF03F35069
:1041E800D927D451CE03F350D927D551CD03F35055
:1041F800D92753500C0D0A0EF324D96E010EF42062
:10420800DA6EDF50DA6FDAC0DBF0DC6BDD6BDE6BA9
:1042180053500C0D0B0EF324D96E010EF420DA6EF8
:10422800DF50DF6FDFC0E0F0E16BE26BE36B535010
:104238000C0D000EF324D96E010EF420DA6EDECFD9
:10424800E4F0DDCFE5F0E4C0E6F0E5C0E7F0000E0D
:10425800E7BFFF0EE86FE96FE651E003F3CFEAF03E
:10426800F4CFEBF0EC6BED6BE103F350EB27F4507C
:10427800EC23000EED23E751E003F350EB27F45055
:10428800EC23000EED23E651E203F350EC27F45043
:10429800ED23E751E103F350EC27F450ED23E85107
:1042A800E003F350EC27F450ED23E351E603F35019
:1042B800ED27E751E203F350ED27E851E103F3500E
:1042C800ED27E951E003F350ED27ECC0EDF0EBC02A
:1042D800ECF0EAC0EBF0EA6BEA51DB03F3CFEEF067
:1042E800F4CFEFF0F06BF16BDC03F350EF27F450F1
:1042F800F023000EF123EB51DB03F350EF27F450CA
:10430800F023000EF123EA51DD03F350F027F450B7
:10431800F123EB51DC03F350F027F450F123EC5177
:10432800DB03F350F027F450F123DE51EA03F35096
:10433800F127EB51DD03F350F127EC51DC03F35087
:10434800F127ED51DB03F350F127D651EE25F26F3B
:10435800D751EF21F36FD851F021F46FD951F121E2
:10436800F56FC851F225F76FC951F321F86FCA519B
:10437800F421F96FCB51F521FA6F5350220D000E3D
:10438800F3249E6F030EF4209F6FF7C0A0F0F8C0CF
:10439800A1F0F9C0A2F0FAC0A3F07CEC12F0F66F1D
:1043A800F65111E0220E9C6FFB0E9D6FF7C09EF038
:1043B800F8C09FF0F9C0A0F0FAC0A1F0F6C0A2F0D2
:1043C800A36BADEC67F053500C0D040EF324D96EBB
:1043D800010EF420DA6EF7C0DEFFF8C0DEFFF9C088
:1043E800DEFFFAC0DEFF01015B6B83901200020E54
:1043F800806F65516411631104E1020E625D01E290
:1044080011D220EE13F06051D9266151DA22DE5024
:10441800625DDE506359DE506459DE50655901E231
:10442800EED100D262C07EF063C07FF0D8907F31B9
:104438006B6F7E316A6F6A517E276B517F2360C034
:104448003AF061C03BF020EE1FF06051D92661516F
:10445800DA22DECF6AF0DECF6BF0DECF6CF0DECF93
:104468006DF07EC06EF07FC06FF0090E706FD8904F
:104478006F336E33702FFBD76E516A253C6E6F51C8
:104488006B213D6E000E6C213E6E000E6D213F6E5D
:1044980018EC5BF00001806F805101E0C3D16A69BC
:1044A800010E6B6F7EC06CF07FC06DF06A516C17A7
:1044B8006B516D1760C06EF061C06FF06C516E2764
:1044C8006D516F232F0E6E257C6F000E6F217D6F4F
:1044D8007E4B7F2B62B104D066C078F0796B1AD01E
:1044E80066516A6F6B6B6A3B6B3BF00E6B176A51D8
:1044F8000F0B6B13F00E6A177CC0D9FF7DC0DAFF73
:10450800DF500F0B6C6F6D6B6A516C11786F6B51CC
:104518006D11796F7CC0D9FF7DC0DAFF78C0DFFFED
:1045280020EE03F06051D9266151DA22010EDF6EC8
:1045380060C03AF061C03BF020EE1FF06051D92610
:104548006151DA22DECF6AF0DECF6BF0DECF6CF09D
:10455800DECF6DF07EC06EF07FC06FF0090E706F19
:10456800D8906F336E33702FFBD76E516A253C6E2F
:104578006F516B213D6E000E6C213E6E000E6D2159
:104588003F6E18EC5BF00001806F805101E04AD16A
:104598006A69010E6B6F7EC06CF07FC06DF06A5166
:1045A8006C176B516D1760C06EF061C06FF06C5185
:1045B8006E276D516F232F0E6E257C6F000E6F21B5
:1045C8007D6F62B10CD067C06AF00F0E6A177CC0AD
:1045D800D9FF7DC0DAFFDF50F00B6A1112D066C038
:1045E8006AF067C06BF068C06CF069C06DF0050ECA
:1045F80005D0D8906D336C336B336A33E82EF9D716
:104608006A517A6F7B6B7CC0D9FF7DC0DAFF7AC0B4
:10461800DFFF4FD060C03AF061C03BF020EE1FF0E2
:104628006051D9266151DA22DECF6AF0DECF6BF015
:10463800DECF6CF0DECF6DF063516E6F64516F6F3B
:104648006551706F716B6A516E253C6E6B516F21AD
:104658003D6E6C5170213E6E6D5171213F6E18ECAC
:104668005BF00001806F805101E0DCD06A69010EC7
:104678006B6F62C06CF063C06DF0D8906C376D37AB
:104688006A516C176B516D1760C06EF061C06FF0A6
:104698006C516E276D516F232F0E6E250E6E000E16
:1046A8006F210F6E66C010F067C011F0F5EC66F070
:1046B800A4D020EE03F06051D9266151DA22010E10
:1046C800DF6EB0D060C03AF061C03BF020EE1FF062
:1046D8006051D9266151DA22DECF6AF0DECF6BF065
:1046E800DECF6CF0DECF6DF062C06EF063C06FF0AD
:1046F80064C070F065C071F0080E05D0D8907133B1
:1047080070336F336E33E82EF9D76A516E253C6EDD
:104718006B516F213D6E6C5170213E6E6D51712150
:104728003F6E18EC5BF00001806F80517BE16A6995
:10473800010E6B6F62C06CF063C06DF0D8906C377F
:104748006D37D8906C376D376A516C176B516D1790
:1047580060C06EF061C06FF06C516E276D516F23B1
:104768002F0E6E250E6E000E6F210F6ED5EC59F0D0
:104778000001706B716B726BF00E1114736F6651E0
:10478800746F6751756F6851766F0F0E6915776F83
:1047980070517411666F71517511676F725176118E
:1047A800686F73517711696F6A69010E6B6F62C028
:1047B8006CF063C06DF0D8906C376D37D8906C375B
:1047C8006D376A516C176B516D1760C06EF061C020
:1047D8006FF06C516E276D516F232F0E6E250E6E84
:1047E800000E6F210F6E66C010F067C011F068C030
:1047F80012F069C013F0B6EC60F000015AD760C03F
:10480800D9FF61C0DAFFDF506A6F6B6B6B510AE149
:104818006A51010A01E106D6030A01E1FBD6010A41
:1048280001E150D7805112002D6E1EC044F01FC008
:1048380045F02D5001E0040C010E426E55B0030CFA
:10484800E9D17FEC67F0000901E1FDD1426AFBD1B3
:10485800176A186A196A1A6A090E44EC65F00009A1
:1048680001E0F1D12E0E0E6E0F6A116A100E106E55
:10487800B0EC61F0000901E1E6D12E44E846030BF3
:10488800E8064DE135C020F03F0E201620C021F08B
:10489800226A236A246A22C024F021C023F0226AF3
:1048A800216A3650266E256A3750276E286A2550A9
:1048B80027262650282227502124296E28502220D6
:1048C8002A6E000E23202B6E000E24202C6E292821
:1048D8003E6E000E2A203F6E000E2B20406E000E0A
:1048E8002C20416E3EC020F03FC021F040C022F095
:1048F80041C023F00A0ED8902036213622362336BE
:10490800E82EF9D71EC0D9FF1FC0DAFF20C0DEFF8E
:1049180021C0DEFF22C0DEFF23C0DEFF97D7206A5A
:1049280038AE01D0202A010E201633C021F00F0E18
:1049380021163750030B020DF35021242024020FB7
:10494800436E3450030B206E216A0A0ED89020362D
:104958002136E82EFBD73550226E236AD8902236AE
:104968002336D890223623363644E846030B246E85
:10497800256A2250242623502522205024262150FF
:104988002522242A000E252224C03EF025C03FF00F
:10499800406A416A43C020F0F70E20263EC021F04D
:1049A8003FC022F040C023F041C024F0202A05D0A7
:1049B800D8902136223623362436202EF9D734D003
:1049C80054A43FD0176A186A196A1A6A8D0E44EC03
:1049D80065F0000901E037D1C9EC67F02E0E0E6EC4
:1049E8000F6A116A100E106EB0EC61F0000901E157
:1049F8002AD1300E436E03D0C9EC67F0430643500A
:104A0800FBE138C020F0203A0F0E2016100E216E60
:104A1800226A236A246A202A05D0D89021362236B1
:104A280023362436202EF9D71EC0D9FF1FC0DAFF3F
:104A380021C0DEFF22C0DEFF23C0DEFF24C0DEFF70
:104A480005D7176A186A196A1A6A090E44EC65F0DC
:104A5800000901E0F8D02E0E0E6E0F6A116A100ED2
:104A6800106EB0EC61F0000901E1EDD054A232D033
:104A78003BC020F0060E216ED8902032212EFCD7A4
:104A8800FF0E202638503F0B226E236AD89022361C
:104A980023363944010B2226000E2322222A232200
:104AA800202A03D0D89022362336202EFBD7225036
:104AB800246E2350256E266A276A1EC0D9FF1FC0A0
:104AC800DAFF24C0DEFF25C0DEFF26C0DEFF27C0D8
:104AD800DEFFBCD63950030B206E216AD8902036F1
:104AE8002136D89020362136D890203621363938CC
:104AF800E842070B2026000E2122202A21223840D6
:104B0800E8423F0B1F0B226E236A222A000E232243
:104B180020502202F3CF24F0F4CF25F02302F350E3
:104B2800252621502202F35025262450266E255092
:104B3800276E286A296A1EC0D9FF1FC0DAFF26C05F
:104B4800DEFF27C0DEFF28C0DEFF29C0DEFF7ED6DD
:104B580044C0D9FF45C0DAFF54C0DFFF77D6176AD3
:104B6800186A196A1A6A090E44EC65F000096BE1C3
:104B780044C00EF045C00FF0116A100E106EB0EC74
:104B880061F0000901E062D65ED0176A186A196AF6
:104B98001A6A0A0E44EC65F0000955E144C00EF0AB
:104BA80045C00FF0116A100E106EB0EC61F0E9D735
:104BB800176A186A196A1A6A3A0E44EC65F000090D
:104BC80042E1040E436E0AD0C9EC67F044C0D9FF35
:104BD80045C0DAFFDF6E444A452A4306435001E1E7
:104BE80035D6F2D7176A186A196A1A6A8D0E44EC14
:104BF80065F0000928E1C9EC67F044C00EF045C033
:104C08000FF0116A400E106EB0EC61F0BAD7040EC6
:104C1800426E19D01D50206E216A2150F8E12050B3
:104C280001E10FD6010A01E113D6020A01E1C8D653
:104C3800090A8EE0010A93E0070AA7E0010AB8E032
:104C4800030AD0E0E4D7D6EC67F0425012001BC04C
:104C5800F6FF1CC0F7FF0800F5CF9BF01B4A1C2A83
:104C680000019B5101E11200250E9B1904E09B51A4
:104C7800A2EC67F0ECD7946B956B966B976B1BC0A7
:104C8800F6FF1CC0F7FF0800F5CF9BF01B4A1C2A53
:104C9800300E9B190DE1976B010E966F1BC0F6FF46
:104CA8001CC0F7FF0800F5CF9BF01B4A1C2A06D052
:104CB8002D0E9B1903E1976B020EEFD72A0E9B1955
:104CC80043E11D50D96EDA6A020EDF26DF5CD96E29
:104CD800DA6ADECF8CF0DECF8DF08DAF0BD08C5141
:104CE80000088C6F8D51D8A0E82A00088D6F976B4B
:104CF800020E966F8CC094F08DC095F01BC0F6FF25
:104D08001CC0F7FF0800F5CF9BF01B4A1C2A22D0D5
:104D18000A0E9403F3CF1EF0F4CF1FF09503F3505F
:104D28001F269B511E26000E1F22D00E1E24946F94
:104D3800FF0E1F20956F1BC0F6FF1CC0F7FF080071
:104D4800F5CF9BF01B4A1C2A2F0E9B6503D0390E0A
:104D58009B65DED76C0E9B1903E04C0E9B190AE18C
:104D680096851BC0F6FF1CC0F7FF0800F5CF9BF027
:104D78001B4A1C2A9B5101E112009BC09AF0600E4D
:104D88009A6575D0200E9A5F72D01D50D96EDA6A76
:104D9800020EDF26DF5CD96EDA6ADECF84F0DECF62
:104DA80085F0926B936B03D00001924B932B925139
:104DB80084251E6E935185211F6E1EC0F6FF1FC0ED
:104DC800F7FF000EF86E0E0EF76403D00800F550DA
:104DD80005D0F6CFE9FFF7CFEAFFEF50000904E06E
:104DE800E3D7200EA2EC67F0000196B30BD09251E6
:104DF8001E6E93511F6E924B932B94511E5C9551CE
:104E08001F58EFE384C00FF085C010F034EC62F057
:104E180003D0200EA2EC67F0000192511E6E935150
:104E28001F6E924B932B94511E5C95511F5801E3B2
:104E38000ED7EFD71D50D96EDA6ADF50DF2ADF2A86
:104E4800D96EDA6ADF50A2EC67F001D7876B020EE1
:104E580008D0876B080E05D0876B0A0E02D0876BC7
:104E6800100E866F1AD09B51A2EC67F0F0D69A51BB
:104E78001E6E1F6A1F50F7E11E50420AE7E0010A42
:104E8800D9E0070AE9E00B0AE4E01C0A01E17DD752
:104E9800060AE2E00D0AE3E0E6D796A511D01D5018
:104EA800D96EDA6A040EDF26DF5CD96EDA6ADECFE5
:104EB8008EF0DECF8FF0DECF90F0DECF91F027D0EE
:104EC800440E9A1913E01D50D96EDA6ADF50DF2AB2
:104ED800DF2AD96EDA6ADECF1EF0DDCF1FF01EC0E2
:104EE8008EF01FC08FF0906B916B11D01D50D96E52
:104EF800DA6ADF50DF2ADF2AD96EDA6ADECF8EF06F
:104F0800DDCF8FF0000E8FBFFF0E906F916F440EB4
:104F18009A190CE191AF0AD08E6D8F1FD8B08F2BE4
:104F2800901FD8B0902B000E91579689986B996B6B
:104F38008EC088F08FC089F090C08AF091C08BF045
:104F480088C00EF089C00FF08AC010F08BC011F035
:104F580086C012F087C013F0146A156A1FEC61F05E
:104F68000E5000019A6F88C00EF089C00FF08AC0F9
:104F780010F08BC011F086C012F087C013F0146ACD
:104F8800156AF0EC5EF00EC088F00FC089F010C012
:104F98008AF011C08BF0090E00019A650BD0780ECB
:104FA8009B1903E0816B070E02D0816B270E806F7F
:104FB80080519A279851600FD96EDA6A9A51300F4A
:104FC800DF6E984B992B885189118A118B1105E056
:104FD800995103E1200E985DB3E396A908D0985142
:104FE800600FD96EDA6A2D0EDF6E984B992B98C038
:104FF80092F099C093F096B103D0836B200E02D043
:10500800836B300E826F82C09AF003D09A51A2EC63
:1050180067F0000196B30BD092511E6E93511F6E2C
:10502800924B932B94511E5C95511F58EFE39807B0
:10503800D8A099079851600FD96EDA6ADF50A2ECB0
:1050480067F000019851991104E0F1D7200EA2EC05
:1050580067F0000192511E6E93511F6E924B932B75
:1050680094511E5C95511F5801E3F1D5EFD781C0CB
:10507800D9FF82C0DAFFDECF98F0DDCF99F08351F7
:1050880084118511861128E120EE0BF09851D9265C
:105098009951DA22DECF90F0DECF91F0DECF92F098
:1050A800DECF93F090519111921193110FE020EE01
:1050B80013F09851D9269951DA22DE50905DDE50CE
:1050C8009159DE509259DE50935952E3010E906F78
:1050D800916B926B936B4CD081C045F082C046F0C7
:1050E80083C047F084C048F085C049F086C04AF0C4
:1050F80045EC30F045C09AF046C09BF047C09CF0A4
:1051080048C09DF000019D519C119B1109E1020EC0
:105118009A5D06E2010E816F826B836B846B000CD3
:105128009A290FE19B290DE19C290BE19D2909E1B1
:105138009AC081F09BC082F09CC083F09DC084F02F
:10514800120020EE13F09851D9269951DA22DE5038
:105158009A5DDE509B59DE509C59DE509D59E8E31C
:1051680083C090F084C091F085C092F086C093F01F
:1051780020EE0FF09851D9269951DA22DE50DE1030
:10518800DE10DE1005E1816B826B836B846B12008D
:10519800946B956B966B976B8351901909E18451C9
:1051A800911906E1855192197DE186519319D8A488
:1051B80079D09029946F000E9121956F000E92215D
:1051C800966F000E9321976F20EE13F09851D92611
:1051D8009951DA22DE50945DDE509559DE50965989
:1051E800DE50975905E3020E946F956B966B976B9B
:1051F80081C045F082C046F094C047F095C048F0A1
:1052080096C049F097C04AF045EC30F045C09AF096
:1052180046C09BF047C09CF048C09DF000019A052D
:105228009B119C119D1184E09A2907E19B2905E1B6
:105238009C2903E19D2901E17BD79A519B119C117F
:105248009D1130E020EE0BF09851D9269951DA22C1
:10525800DECF9AF0DECF9BF0DECF9CF0DECF9DF064
:105268009D519C119B1103E1020E9A5D17E320EEFC
:1052780013F09851D9269951DA22DE509A5DDE5002
:105288009B59DE509C59DE509D5908E29AC090F017
:105298009BC091F09CC092F09DC093F0946B956B6D
:1052A800966B976B945195119611971162E190C086
:1052B80094F091C095F092C096F093C097F0942B1B
:1052C800000E95239623972320EE13F09851D926A4
:1052D8009951DA22DE50945DDE509559DE50965988
:1052E800DE5097590DE3020E946F956B966B976B92
:1052F80093519211911104E1020E905D01E243D79E
:1053080081C045F082C046F094C047F095C048F08F
:1053180096C049F097C04AF045EC30F045C09AF085
:1053280046C09BF047C09CF048C09DF000019A51D0
:105338009B119C119D111DE09A059B119C119D11BB
:1053480001E1F6D69A2907E19B2905E19C2903E1A9
:105358009D2901E1EDD690519419B1E1915195192A
:10536800AEE192519619ABE19351971901E10BD730
:10537800A6D798C060F099C061F094C062F095C05B
:1053880063F096C064F097C065F0666967696869FC
:105398006969FBEC21F08F6F8F511CE183518411F7
:1053A8008511861117E098C060F099C061F083C03C
:1053B80062F084C063F085C064F086C065F094C074
:1053C80066F095C067F096C068F097C069F0FBEC8E
:1053D80021F08F6F8F5143E120EE0BF09851D926C1
:1053E8009951DA2294C0DEFF95C0DEFF96C0DEFF39
:1053F80097C0DEFF20EE0FF09851D9269951DA2296
:1054080010EE13F09851E1269951E222FE0EE6249F
:105418008B6FFF0EE6208C6FFF0EE6208D6FFF0E60
:10542800E6208E6FDE508B5DDE508C59DE508D5934
:10543800DE508E590BE320EE0FF09851D926995182
:10544800DA22DE06000EDE5ADE5ADE5A20EE04F0BC
:105458009851D9269951DA22000EDB800DD08F059C
:1054680007E0010E946F000E956B966B976B04D056
:10547800946995699669976994C081F095C082F09E
:1054880096C083F097C084F01200000E0001746F7C
:10549800030E756F350E766F0B0E776F020E796FF0
:1054A800786BF30E7A6F7B6B32EC1DF00101686F3D
:1054B800630E00019C6FFD0E9D6FF3C09EF0F4C05B
:1054C8009FF0ADEC67F0F56BF66BF16BF26BF76B79
:1054D800F86BF751D30FD96EDA6ADF6AF751E20F2A
:1054E800D96EDA6A000EDF6EF74BF82BF8BFF1D7EA
:1054F800F85103E10F0EF75DECE3F96BFA6B43D15A
:10550800350EF925D96E0B0EFA21DA6E0D0EDE185E
:1055180001E0FED08C0E0E6EFF0E0F6ED30E106ED5
:10552800B1EC5BF00E500F1007E1E20E156E08ECBF
:1055380052F015500101FB6F860E0E6EFF0E0F6EB6
:10554800D30E106EB1EC5BF00E500F1007E1E20EB7
:10555800156E08EC52F015500101696F6B0E0E6E56
:10556800FF0E0F6ED30E106EB1EC5BF00E500F10E5
:1055780007E1E20E156E08EC52F015500101646F58
:10558800D40E0E6EFF0E0F6ED30E106EB1EC5BF0E4
:105598000E500F1007E1E20E156E08EC52F0155090
:1055A8000101626FDC0E0E6EFF0E0F6ED30E106ED1
:1055B800B1EC5BF00E500F1007E1E20E156E08EC2F
:1055C80052F015500101CF6FD80E0E6EFF0E0F6E00
:1055D800D30E106EB1EC5BF00E500F1008E1E20E26
:1055E800156E08EC52F015C052F116C053F10001C7
:1055F800FB6BFC6BC40E7C6F7D6B720E7E6FFF0EB7
:105608007F6FFBC080F0FCC081F0D2EC64F0C40E68
:105618000E6E0F6AD30E106EB1EC5BF00E500F10C9
:1056280018E10F0E0001FB03F3CFC2F0F4CFC3F073
:10563800FC03F350C327350EC2250E6E0D0EC32191
:105648000F6EE20E106E116A136A0F0E126EDFEC07
:1056580061F00001FB4BFC2BFCBFCCD7FC5103E1F4
:10566800100EFB5DC7E3FC6B010EFB6FC40E7C6F75
:105678007D6B790E7E6FFF0E7F6FFBC080F0FCC0E4
:1056880081F0D2EC64F0C40E0E6E0F6AD30E106E69
:10569800B1EC5BF00E500F1018E10F0E0001FB0388
:1056A800F3CFC2F0F4CFC3F0FC03F350C327250EA9
:1056B800C2250E6E0E0EC3210F6EE20E106E116A19
:1056C800136A0F0E126EDFEC61F00001FB4BFC2B2E
:1056D800FCBFCCD7FC5103E1040EFB5DC7E3F76BBD
:1056E800F86BF751D30FD96EDA6ADF6AF751E20F18
:1056F800D96EDA6A000EDF6EF74BF82BF8BFF1D7D8
:10570800F85103E10F0EF75DECE3F16BF26B15D086
:10571800350EF925D96E0B0EFA21DA6E0A0EDE184F
:1057280030E0350EF925D96E0B0EFA21DA6E200E0F
:10573800DE1806E1F26B010EF16FF56BF66B21D006
:10574800F151F21109E0350EF925D96E0B0EFA2147
:10575800DA6EF551E20F08D0350EF925D96E0B0E29
:10576800FA21DA6EF551D30FE16EE26ADFCFE7FF77
:10577800F6BF05D0F65105E10F0EF55D02E2F54BD7
:10578800F62BF94BFA2BF351F95DF451FA5901E272
:10579800B7D6530E9C6FFD0E9D6F64C19EF09F6B34
:1057A800ADEC67F0CD0E9C6FFD0E9D6FFBC19EF0BA
:1057B8009F6BADEC67F0AF0E9C6FFD0E9D6F69C1DE
:1057C8009EF09F6BADEC67F0BE0E9C6FFD0E9D6F5B
:1057D800CFC19EF09F6BADEC67F0320E9C6FFC0E54
:1057E8009D6F52C19EF053C19FF0ADEC67F0FB6B0B
:1057F800FC6BC00E9C6FFC0E9D6FFBC09EF0FCC046
:105808009FF00F0EFB03F3CFC2F0F4CFC3F0FC03FD
:10581800F350C327350EC225A06F0D0EC321A16F0B
:10582800ADEC67F0FB4BFC2BFCBFE3D7FC5103E16D
:10583800100EFB5DDEE3FA6B010EF96FD10E9C6F63
:10584800FC0E9D6FF9C09EF0FAC09FF00F0EF90391
:10585800F3CFC2F0F4CFC3F0FA03F350C327250EF9
:10586800C225A06F0E0EC321A16FADEC67F0F94BF6
:10587800FA2BFABFE3D7FA5103E1040EF95DDEE330
:10588800740E9C6FF90E9D6FADEF67F0838E838069
:1058980056EC41F0FC6FFC5118E053501E0D1B0EE6
:1058A800F324D96E020EF420DA6E53501E0D1B0E2F
:1058B800F324E16E020EF420E26EE7500409DF6E75
:1058C8005FEC66F00001FC511200010162514EE0EC
:1058D800385139113A113B1149E0535047E15350BF
:1058E8001E0D070EF324D96E020EF420DA6E38C1AD
:1058F80076F139C177F13AC178F1756B000E7525EB
:10590800796F010E76217A6F000E77217B6F000E7A
:1059180078217C6F7D6B7E6B7F6B806BDE50791995
:1059280025E1DE507A1922E1DE507B191FE1DE50B5
:105938007C191CE1DE507D1919E1DE507E1916E153
:10594800DE507F1913E1DE50801910E1350E2B6E01
:105958000B0E2C6E6251FFEC54F00292000E66ECB6
:105968005BF00292516A83905150120053501E0D01
:10597800170EF324D96E020EF420DA6EDECF6DF125
:10598800DECF6EF1DECF6FF1DECF70F16EC16DF15B
:105998006FC16EF170C16FF1706B6DC1F2F06EC1C5
:1059A800F3F06FC1F4F070C1F5F053501E0D170EEF
:1059B800F324D96E020EF420DA6EDECF6DF1DDCF5E
:1059C8006EF16D510001F66FF76B0292F86BF96B8F
:1059D800FA6BFB6BF251F311F411F51104E1F26962
:1059E800F36BF46BF56BF06BF16BCBD08EB80AD020
:1059F800FA0E00019C6FFE0E9D6FADEC67F0BAD0F9
:105A08008394BAD0F0C06DF1F1C06EF1000E6EBF94
:105A1800FF0E6F6F706FFF0E0001F2250101716FAD
:105A2800FF0E0001F3210101726FFF0E0001F42146
:105A38000101736FFF0E0001F5210101746F6D51B3
:105A4800711910E16E5172190DE16F5173190AE164
:105A58007051741907E10001F651F71103E1025082
:105A68000209026E5350220D000EF3240001746FD8
:105A7800030EF420756F350E766F0B0E776F010EDF
:105A8800796F786BFD0E7A6F7B6B32EC1DF0FF6FD0
:105A9800FF5101E002D7FD51FE1101E1FED6D00E03
:105AA80001016D6FC90EE82EFED76D2FFCD700D00F
:105AB8008EB808D0FA0E00019C6FFE0E9D6FADECFB
:105AC80067F058D00001FD5166EC5BF00001FD5114
:105AD800F827FE51F923000EFA23FB2353501E0D1D
:105AE800070EF324D96E020EF420DA6E000EDE24BF
:105AF80001016D6F010EDE206E6F000EDE206F6FEC
:105B0800000EDE20706F000EDE20716F000EDE20AA
:105B1800726F000EDE20736F000EDE20746F53501C
:105B28001E0D070EF324D96E020EF420DA6E6DC135
:105B3800DEFF6EC1DEFF6FC1DEFF70C1DEFF71C127
:105B4800DEFF72C1DEFF73C1DEFF74C1DEFF8EB8F7
:105B580008D0FA0E00019C6FFE0E9D6FADEC67F049
:105B680009D08EBC0BD0F00E00019C6FFE0E9D6F0D
:105B7800ADEC67F0516A44D7839086D00001F04BB2
:105B8800F12BF0C06DF1F1C06EF1000E01016EBF96
:105B9800FF0E6F6F706F0001F25101016D5D000122
:105BA800F35101016E590001F45101016F590001CF
:105BB800F5510101705901E219D70001F651F711A9
:105BC80060E05350220D000EF324746F030EF4208E
:105BD800756F350E766F0B0E776FF6C078F0F7C0DD
:105BE80079F0FD0E7A6F7B6B32EC1DF0FF6FFF5181
:105BF80001E053D602500209026EF65166EC5BF0E2
:105C08000001FD51F827FE51F923000EFA23FB236A
:105C180053501E0D070EF324D96E020EF420DA6ECF
:105C2800000EDE2401016D6F010EDE206E6F000E86
:105C3800DE206F6F000EDE20706F000EDE20716FA9
:105C4800000EDE20726F000EDE20736F000EDE2065
:105C5800746F53501E0D070EF324D96E020EF420F4
:105C6800DA6E6DC1DEFF6EC1DEFF6FC1DEFF70C18F
:105C7800DEFF71C1DEFF72C1DEFF73C1DEFF74C1DA
:105C8800DEFF0292516A78D7839E6ED653500C0D70
:105C9800030EF324D96E010EF420DA6EDF2A535076
:105CA8000C0D030EF324D96E010EF420DA6EDF50CA
:105CB8000001C76FC86BC969CA6953500C0D0B0E38
:105CC800F324D96E010EF420DA6EDF50CB6FCC6B63
:105CD800C951CB27CA51CC23C751CB5DCC51800ABF
:105CE800CD6FC851800ACD594BE253500C0D030EAD
:105CF800F324D96E010EF420DA6EDF6A53500C0DCE
:105D0800020EF324D96E010EF420DA6EDF2A535006
:105D18000C0D020EF324D96E010EF420DA6EDF505A
:105D2800C76FC86BC969CA6953500C0D0A0EF324B2
:105D3800D96E010EF420DA6EDF50CB6FCC6BC951EF
:105D4800CB27CA51CC23C751CB5DCC51800ACD6F2C
:105D5800C851800ACD5914E253500C0D020EF32499
:105D6800D96E010EF420DA6EDF6A53500C0D000E66
:105D7800F324D96E010EF420DA6EDE2A000EDD223D
:105D880053500C0D030EF324D96E010EF420DA6E75
:105D9800DF50C76FC7C0C8F0C96BCA6BCB6BCAC02E
:105DA800CBF0C9C0CAF0C8C0C9F0C86B53500C0DBD
:105DB8000B0EF324D96E010EF420DA6EDF50CC6F8F
:105DC800CCC0CDF0CE6BCF6BD06B53500C0D020E08
:105DD800F324D96E010EF420DA6EDF50D16FD1C0F2
:105DE800D2F0D36BD46BD56BD4C0D5F0D3C0D4F07C
:105DF800D2C0D3F0D26BD251CD03F3CFD6F0F4CFCB
:105E0800D7F0D86BD96BCE03F350D727F450D823EB
:105E1800000ED923D351CD03F350D727F450D823FC
:105E2800000ED923D251CF03F350D827F450D923E9
:105E3800D351CE03F350D827F450D923D451CD03EE
:105E4800F350D827F450D923D051D203F350D9278F
:105E5800D351CF03F350D927D451CE03F350D927C8
:105E6800D551CD03F350D92753500C0D0A0EF32406
:105E7800D96E010EF420DA6EDF50DA6FDAC0DBF08B
:105E8800DC6BDD6BDE6B53500C0D0B0EF324D96EFF
:105E9800010EF420DA6EDF50DF6FDFC0E0F0E16B57
:105EA800E26BE36B53500C0D000EF324D96E010E18
:105EB800F420DA6EDECFE4F0DDCFE5F0E4C0E6F002
:105EC800E5C0E7F0000EE7BFFF0EE86FE96FE651A7
:105ED800E003F3CFEAF0F4CFEBF0EC6BED6BE1030A
:105EE800F350EB27F450EC23000EED23E751E003C9
:105EF800F350EB27F450EC23000EED23E651E203B8
:105F0800F350EC27F450ED23E751E103F350EC276D
:105F1800F450ED23E851E003F350EC27F450ED235F
:105F2800E351E603F350ED27E751E203F350ED2781
:105F3800E851E103F350ED27E951E003F350ED2771
:105F4800ECC0EDF0EBC0ECF0EAC0EBF0EA6BEA5124
:105F5800DB03F3CFEEF0F4CFEFF0F06BF16BDC0383
:105F6800F350EF27F450F023000EF123EB51DB033D
:105F7800F350EF27F450F023000EF123EA51DD032C
:105F8800F350F027F450F123EB51DC03F350F027E2
:105F9800F450F123EC51DB03F350F027F450F123D4
:105FA800DE51EA03F350F127EB51DD03F350F127FB
:105FB800EC51DC03F350F127ED51DB03F350F127EB
:105FC800D651EE25F26FD751EF21F36FD851F0215A
:105FD800F46FD951F121F56FC851F225F66FC95107
:105FE800F321F76FCA51F421F86FCB51F521F96FFE
:105FF80053500C0D040EF324D96E010EF420DA6E02
:10600800F6C0DEFFF7C0DEFFF8C0DEFFF9C0DEFF36
:106018005350220D000EF3249E6F030EF4209F6F41
:1060280053500C0D040EF324D96E010EF420DA6ED1
:10603800DECFA0F0DECFA1F0DECFA2F0DECFA3F05E
:106048007CEC12F04B6E4B5019E0220E9C6FFB0E4D
:106058009D6F53500C0D040EF324D96E010EF420DD
:10606800DA6EDECF9EF0DECF9FF0DECFA0F0DECF7F
:10607800A1F04BC0A2F0A36BADEC67F001015B6B24
:10608800120045C0D9FF46C0DAFFDECF72F0DDCF7F
:1060980073F04A504910481003E1020E475C10E3C0
:1060A800000120EE13F07251D9267351DA22DE5026
:1060B800475CDE504858DE504958DE504A5808E3DD
:1060C800010E00016C6F000E6D6B6E6B6F6B8FD1E4
:1060D8006C696D696E696F6976D147C070F048C0A8
:1060E80071F0D8907131616F7031606F60517027B5
:1060F8006151712372C03AF073C03BF020EE1FF07B
:106108007251D9267351DA22DECF60F0DECF61F00A
:10611800DECF62F0DECF63F070C064F071C065F06E
:10612800090E666FD89065336433662FFBD76451C8
:1061380060253C6E655161213D6E000E62213E6E08
:10614800000E63213F6E18EC5BF0000901E04FD1AF
:1061580000016069010E616F70C062F071C063F088
:10616800605162176151631772C064F073C065F0C3
:1061780062516427635165232F0E6425D96E000E82
:106188006521DA6EDF506A6F6B6B704B712B72C0D2
:106198003AF073C03BF020EE1FF07251D9267351CC
:1061A800DA22DECF60F0DECF61F0DECF62F0DECF44
:1061B80063F070C064F071C065F0090E666FD89026
:1061C80065336433662FFBD7645160253C6E655197
:1061D80061213D6E000E62213E6E000E63213F6E0E
:1061E80018EC5BF0000901E002D100016069010EC2
:1061F800616F70C062F071C063F0605162176151E5
:10620800631772C064F073C065F06251642763510C
:1062180065232F0E6425D96E000E6521DA6EDF50D6
:10622800676F666B66516A1367516B1347B006D088
:106238006A51686F0F0E6B15696F0FD06AC060F0F6
:106248006BC061F0040E626FD89061336033622FC7
:10625800FBD760C068F061C069F068C06CF069C0C5
:106268006DF04ED072C03AF073C03BF020EE1FF0D4
:106278007251D9267351DA22DECF60F0DECF61F099
:10628800DECF62F0DECF63F04850646F4950656F2F
:106298004A50666F676B605164253C6E6151652199
:1062A8003D6E625166213E6E635167213F6E18EC68
:1062B8005BF0000901E09BD000016069010E616F8D
:1062C80047C062F048C063F0D890623763376051C6
:1062D80062176151631772C064F073C065F0625150
:1062E8006427635165232F0E64250E6E000E652109
:1062F8000F6EE5EC65F00EC06CF00FC06DF000019C
:106308006E6B6F6B74D072C03AF073C03BF020EEC6
:106318001FF07251D9267351DA22DECF60F0DECF3A
:1063280061F0DECF62F0DECF63F047C064F048C0B2
:1063380065F049C066F04AC067F0080E05D0D890ED
:106348006733663365336433E82EF9D760516425C3
:106358003C6E615165213D6E625166213E6E63510E
:1063680067213F6E18EC5BF0000941E100016069AC
:10637800010E616F47C062F048C063F0D890623781
:106388006337D8906237633760516217615163177A
:1063980072C064F073C065F062516427635165236D
:1063A8002F0E64250E6E000E65210F6ED5EC59F088
:1063B8000E5000016C6F0F506D6F10506E6F0F0E06
:1063C80011146F6F14D072C0D9FF73C0DAFFDF5099
:1063D800606F616B615101E073D66051010A01E1A0
:1063E8007CD6030A01E13ED7010A8DE069D66CC06C
:1063F80045F06DC046F06EC047F06FC048F012001F
:10640800536A01015D6B536A030E536401D0A8D12E
:10641800535003E1266A276A03D0276A010E266EC5
:1064280053501E0D1B0EF324D96E020EF420DA6EA3
:10643800DF6A53501E0D000EF324D96E020EF420AD
:10644800DA6EDF6A53501E0D070EF324D96E020E62
:10645800F420DA6E070EDE6AE806FDE20D0E26026B
:10646800F3CFC2F0F4CFC3F02702F3500001C327E3
:10647800A20EC225D96E020EC321DA6EDF50C46F98
:10648800C4C0C5F0C66BC76BC86BC7C0C8F0C6C070
:10649800C7F0C5C0C6F0C56B0D0E2602F3CFC9F014
:1064A800F4CFCAF02702F350CA27A10EC925D96E26
:1064B800020ECA21DA6EDF50CB6FCBC0CCF0CD6BA9
:1064C800CE6BCF6BCDC0CFF0CCC0CEF0CD6BCC6B4C
:1064D8000D0E2602F3CFD0F0F4CFD1F02702F350FF
:1064E800D127A00ED025D96E020ED121DA6EDF5049
:1064F800D26FD2C0D3F0D46BD56BD66BD3C0D6F0E5
:10650800D56BD46BD36BCC51D325D76FCD51D42158
:10651800D86FCE51D521D96FCF51D621DA6FC55159
:10652800D725DB6FC651D821DC6FC751D921DD6F64
:10653800C851DA21DE6F0D0E2602F3CFDFF0F4CF5B
:10654800E0F02702F350E027A30EDF25D96E020EF4
:10655800E021DA6EDF50DB25E16F000EDC21E26F0F
:10656800000EDD21E36F000EDE21E46FE1C0E5F0EF
:10657800E2C0E6F0E3C0E7F0E4C0E8F0E96BE8BFAA
:10658800E969E9C0EAF0E9C0EBF0E9C0ECF0535082
:106598001E0D0F0EF324D96E020EF420DA6EE5C03C
:1065A800DEFFE6C0DEFFE7C0DEFFE8C0DEFFE9C0D1
:1065B800DEFFEAC0DEFFEBC0DEFFECC0DEFF5350BB
:1065C8001E0D1C0EF324D96E020EF420DA6EDECFF7
:1065D800C2F0DDCFC3F0C2C00EF0C3C00FF0106A26
:1065E800116A126A136A146A156A53501E0D0F0E47
:1065F800F324D96E020EF420DA6EDECFC4F0DECFBB
:10660800C5F0DECFC6F0DECFC7F0DECFC8F0DECFF4
:10661800C9F0DECFCAF0DECFCBF0C4C016F0C5C0DB
:1066280017F0C6C018F0C7C019F0C8C01AF0C9C022
:106638001BF0CAC01CF0CBC01DF066EC5DF00EC0AC
:10664800CCF00FC0CDF010C0CEF011C0CFF012C00A
:10665800D0F013C0D1F014C0D2F015C0D3F053500D
:106668001E0D0F0EF324D96E020EF420DA6ECCC084
:10667800DEFFCDC0DEFFCEC0DEFFCFC0DEFFD0C064
:10668800DEFFD1C0DEFFD2C0DEFFD3C0DEFF535035
:106698001E0D170EF324D96E020EF420DA6EDE6A90
:1066A800DE6ADE6A010EDD6E2C0E00019C6FFA0EAA
:1066B8009D6F53C09EF09F6B53501E0D0F0EF32419
:1066C800D96E020EF420DA6EDECFC2F0DECFC3F050
:1066D800DECFC4F0DECFC5F0DECFC6F0DECFC7F028
:1066E800DECFC8F0DECFC9F0C2C0A0F0C3C0A1F0B1
:1066F800C4C0A2F0C5C0A3F0C6C0A4F0C7C0A5F02E
:10670800C8C0A6F0C9C0A7F053501E0D0F0EF32441
:10671800D96E020EF420DA6EDECFCAF0DECFCBF0EF
:10672800DECFCCF0DECFCDF0DECFCEF0DECFCFF0B7
:10673800DECFD0F0DECFD1F0CAC0A8F0CBC0A9F030
:10674800CCC0AAF0CDC0ABF0CEC0ACF0CFC0ADF09D
:10675800D0C0AEF0D1C0AFF0ADEC67F0532A54D63C
:106768000101606B526A5F6B4E6A4F6A020E516E8E
:106778005E6F8390020C9EC0D9FF9FC0DAFFDECF08
:10678800B2F0DDCFB3F020EE0EF09E51D9269F5126
:10679800DA22DECFA2F0DECFA3F0DECFA4F0DECF88
:1067A800A5F0200EA225AE6F000EA321AF6F000E3C
:1067B800A421B06F000EA521B16FB15103E1200EE5
:1067C800B05D0AE320EE16F09E51D9269F51DA22D9
:1067D800DE6ADE6ADE6ADD6A20EE16F09E51D92690
:1067E8009F51DA22DE50DE10DE10DE1001E1040CCB
:1067F800AE51A26F010EAF15A36FA46BA56BA211CA
:10680800A411A51101E029D120EE16F09E51D92638
:106818009F51DA22DE2A000EDE22DE22DE2220EE60
:1068280012F09E51D9269F51DA22DE50DE10DE107A
:10683800DE102CE120EE07F0B251D926B351DA224E
:10684800DECFA2F0DDCFA3F0A251A46FA351A56FB4
:10685800A66BA76BAEC0A8F0AFC0A9F0B0C0AAF0F5
:10686800B1C0ABF0060E05D0D890AB33AA33A9332C
:10687800A833E82EF9D7A451A85DA551A959A65166
:10688800AA59A751AB5901E2E8D06ED0A269A36911
:1068980020EE09F0B251D926B351DA22DECFA4F0A6
:1068A800DDCFA5F0A251A427A351A523AEC0A6F021
:1068B800AFC0A7F0B0C0A8F0B1C0A9F00A0E05D0CB
:1068C800D890A933A833A733A633E82EF9D7A45113
:1068D800A615AA6FA551A715AB6FAC6BAD6BAA1126
:1068E800AC11AD1101E0B9D09EC045F09FC046F093
:1068F80020EE12F09E51D9269F51DA22DECF47F0C2
:10690800DECF48F0DECF49F0DECF4AF045EC30F07C
:1069180045C0B4F046C0B5F047C0B6F048C0B7F0BF
:106928000001B751B611B51104E1020EB45D01E2E0
:10693800020CB42907E1B52905E1B62903E1B72915
:1069480001E1010C20EE13F0B251D926B351DA223D
:10695800DE50B45DDE50B559DE50B659DE50B75939
:1069680050E3A051A1110BE120EE16F09E51D9265B
:106978009F51DA22DE6ADE6ADE6ADD6A040C9EC096
:1069880081F09FC082F020EE12F09E51D9269F51CF
:10699800DA22DECF83F0DECF84F0DECF85F0DECFE3
:1069A80086F03BEC28F081C0B4F082C0B5F083C01B
:1069B800B6F084C0B7F0B451B511B611B71101E102
:1069C800070CB405B511B611B71101E1020CB429D1
:1069D80007E1B52905E1B62903E1B72901E1010C71
:1069E800B2C03AF0B3C03BF0B4C03CF0B5C03DF023
:1069F800B6C03EF0B7C03FF086EC51F0000901E0A8
:106A0800010C000120EE12F09E51D9269F51DA2286
:106A1800B4C0DEFFB5C0DEFFB6C0DEFFB7C0DEFF24
:106A2800B2C00EF0B3C00FF0B4C010F0B5C011F092
:106A3800B6C012F0B7C013F0F2EC4FF0000120EE30
:106A480016F09E51D9269F51DA220EC0DEFF0FC0E4
:106A5800DEFF10C0DEFF11C0DEFF20EE0EF09E51FB
:106A6800D9269F51DA22AEC0DEFFAFC0DEFFB0C02C
:106A7800DEFFB1C0DEFFA269010EA36FAEC0A4F0B5
:106A8800AFC0A5F0A251A417A351A517B2C0A6F094
:106A9800B3C0A7F0A451A627A551A7232F0EA62758
:106AA800000EA72320EE1AF09E51D9269F51DA2214
:106AB800A6C0DEFFA7C0DDFF000C53500C0D030E6F
:106AC800F324D96E010EF420DA6EDF506D6F6DC1BC
:106AD8006EF16F6B706B716B70C171F16FC170F19A
:106AE8006EC16FF16E6B53500C0D0B0EF324D96E03
:106AF800010EF420DA6EDF50726F72C173F1746B9D
:106B0800756B766B53500C0D020EF324D96E010E83
:106B1800F420DA6EDF50776F77C178F1796B7A6B92
:106B28007B6B7AC17BF179C17AF178C179F1786BA5
:106B380078517303F3CF7CF1F4CF7DF17E6B7F6BDB
:106B48007403F3507D27F4507E23000E7F23795180
:106B58007303F3507D27F4507E23000E7F23785172
:106B68007503F3507E27F4507F2379517403F35053
:106B78007E27F4507F237A517303F3507E27F45015
:106B88007F2376517803F3507F2779517503F350AB
:106B98007F277A517403F3507F277B517303F35097
:106BA8007F2753500C0D0A0EF324D96E010EF420E2
:106BB800DA6EDF50806F80C181F1826B836B846BEA
:106BC80053500C0D0B0EF324D96E010EF420DA6E1F
:106BD800DF50856F85C186F1876B886B896B535051
:106BE8000C0D000EF324D96E010EF420DA6EDECF00
:106BF8008AF1DDCF8BF18AC18CF18BC18DF1000E4A
:106C08008DBFFF0E8E6F8F6F8C518603F3CF90F17F
:106C1800F4CF91F1926B936B8703F3509127F45063
:106C28009223000E93238D518603F3509127F4503D
:106C38009223000E93238C518803F3509227F4502B
:106C480093238D518703F3509227F45093238E5149
:106C58008603F3509227F450932389518C03F35001
:106C680093278D518803F35093278E518703F35050
:106C780093278F518603F350932792C193F191C1C3
:106C880092F190C191F1906B90518103F3CF94F1FF
:106C9800F4CF95F1966B976B8203F3509527F450D8
:106CA8009623000E972391518103F3509527F450B2
:106CB8009623000E972390518303F3509627F450A0
:106CC800972391518203F3509627F45097239251BA
:106CD8008103F3509627F450972384519003F3507F
:106CE800972791518303F350972792518203F350CA
:106CF800972793518103F35097277C519425986FD8
:106D08007D519521996F7E5196219A6F7F519721D8
:106D18009B6F6E5198250001DC6F01016F5199211D
:106D28000001DD6F010170519A210001DE6F010140
:106D380071519B210001DF6F5350220D000EF32487
:106D48009E6F030EF4209F6FDCC0A0F0DDC0A1F0A1
:106D5800DEC0A2F0DFC0A3F07CEC12F0DB6FDB51E9
:106D680011E0220E9C6FFB0E9D6FDCC09EF0DDC013
:106D78009FF0DEC0A0F0DFC0A1F0DBC0A2F0A36BE3
:106D8800ADEC67F07F0E9C6FFE0E9D6FADEC67F06B
:106D9800839053500C0D040EF324D96E010EF42089
:106DA800DA6EDCC0DEFFDDC0DEFFDEC0DEFFDFC086
:106DB800DEFF01015B6B5A6B70EF3FF0000E0001C4
:106DC800F36F250EF26F000EF16F050EF06F0101E3
:106DD800FB5105E1000E0001F36F280EF26F01016F
:106DE80064510DE1FA6B350E00017C6F0D0E7D6F5D
:106DF800720E7E6FFE0E7F6FD2EC64F00DD04C0EDB
:106E080000019C6FFA0E9D6F64C19EF09F6BFAC1E2
:106E1800A0F0A16BADEC67F0EB0E9C6FFD0E9D6FC3
:106E28000101FA510F0D350EF32400019E6F0D0E6E
:106E3800F4209F6FADEC67F0050E0001EF6F0F0EA9
:106E4800EE6FF10EE82EFED7EE2FFCD7EF2FFAD714
:106E5800E3D0AF0E0F6EFC0E106E34EC62F0030E32
:106E68000101CF6105D09650CF19F00BCF1905D08D
:106E7800CFC193FF9650F00B0A09966E000E0001E1
:106E8800CE6F030ECF6F650ED06FFE0ED16F010E61
:106E9800D26F4AEC15F00101686F6851B0EC62F0EE
:106EA800010168510AE1AAEC1AF0000E6D6F030E99
:106EB8006E6FB5EC64F00101686F6851B0EC62F078
:106EC800F36B280EF26FA4D00101FA510F0D350EA5
:106ED800F324D96E0D0EF420DA6E200EDE1806E1CA
:106EE800FA2B0F0EFA6594D0FA6B92D0B00E00010F
:106EF8009C6FFB0E9D6F0101FA510F0D350EF324A7
:106F080000019E6F0D0EF4209F6FADEC67F0000E30
:106F1800CE6F030ECF6F0101FA510F0D350EF3241A
:106F28000001D06F0D0EF420D16F030ED26F4AEC22
:106F380015F00101686F6851B0EC62F00101685109
:106F480004E10001F36B3C0EF26F040E01016819B5
:106F580004E10001F36B320EF26F050E0001EF6FD2
:106F68000F0EEE6FF10EE82EFED7EE2FFCD7EF2FA7
:106F7800FAD74ED06A0E9C6FFC0E9D6F0101FA5134
:106F88000F0D350EF32400019E6F0D0EF4209F6F38
:106F9800ADEC67F0000ECE6F030ECF6F0101FA5112
:106FA8000F0D350EF3240001D06F0D0EF420D16FB4
:106FB800070ED26F4AEC15F00101686F6851CDE1F8
:106FC8000001F36B3C0EC8D7450E9C6FFC0E9D6FFD
:106FD8000101FA510F0D350EF32400019E6F0D0EBD
:106FE800F4209F6FADEC67F013D0F2C0EEF0F3C061
:106FF800EFF0EF510DE1EE51250A01E12AD70D0A14
:1070080001E162D7050A04E01F0AB4E00E0ADCE0D9
:107018000001F007D8A0F1070001F1BF08D0F15135
:1070280002E1F00504E33C0EF219F311DEE1030E70
:10703800010164193BE1839E000E0E6EC00E01EC47
:1070480063F0CCEC66F0000E0E6EC00E01EC63F03F
:107058003C0E0001F219F31116E10101F0510CE0A8
:10706800F00E126E010E136EB3EC5EF0950E126EFA
:10707800FE0E136EB3EC5EF0920E126EFF0E136EE0
:10708800B3EC5EF0000C350E7C6F0D0E7D6F3B0E81
:107098007E6FFF0E7F6F68C180F0816BD2EC64F069
:1070A800350E126E0D0E136EB3EC5EF0000C74C04C
:1070B800D9FF75C0DAFFDECF8CF0DDCF8DF07951C6
:1070C80009E1200E785DD8B0020C76C07AF01F0E68
:1070D8007A1701E0020C20EE0EF07451D926755192
:1070E800DA2276C0DEFF77C0DEFF78C0DEFF79C027
:1070F800DEFF20EE06F07451D9267551DA22DECF74
:1071080088F0DECF89F0DECF8AF0DECF8BF08851B1
:1071180089118A118B1115E18CC0D9FF8DC0DAFF56
:10712800020EDF640ED020EE23F08C51D9268D514B
:10713800DA22DECF88F0DECF89F0DECF8AF0DECF2C
:107148008BF0885189118A118B1140E120EE07F0EC
:107158008C51D9268D51DA22DECF7AF0DDCF7BF043
:107168007A517C6F7B517D6F7E6B7F6B76C080F030
:1071780077C081F078C082F079C083F0060E05D020
:10718800D8908333823381338033E82EF9D77C510A
:10719800805D7D5181597E5182597F51835901E328
:1071A800020C20EE23F08C51D9268D51DA2210EEF4
:1071B80016F07451E1267551E222DECFE6FFDECFEC
:1071C800E6FFDECFE6FFDECFE6FF87D020EE09F050
:1071D8008C51D9268D51DA22DECF7AF0DDCF7BF0C3
:1071E8007A517C6F7B517D6F7E6B7F6B090ED890D7
:1071F8007C377D377E377F37E82EF9D77CC084F01F
:107208007DC085F07EC086F07FC087F040D074C016
:1072180045F075C046F088C047F089C048F08AC07C
:1072280049F08BC04AF045EC30F045C088F046C0C4
:1072380089F047C08AF048C08BF00001882907E12F
:10724800892905E18A2903E18B2901E1010C8B5188
:107258008A11891104E1020E885DD8A0020C20EE83
:1072680013F08C51D9268D51DA22DE50885DDE501C
:107278008959DE508A59DE508B5901E3020C84513A
:10728800765F8551775B8651785B8751795B84514E
:10729800765D855177598651785987517959B7E282
:1072A8008CC00EF08DC00FF088C010F089C011F0AE
:1072B8008AC012F08BC013F0F2EC4FF0000120EE00
:1072C80016F07451D9267551DA220EC0DEFF0FC0B0
:1072D800DEFF10C0DEFF11C0DEFF20EE12F0745199
:1072E800D9267551DA2288C0DEFF89C0DEFF8AC040
:1072F800DEFF8BC0DEFF20EE16F07451D9267551E3
:10730800DA22DE50DE10DE10DE1001E1020C76C05B
:107318007AF077C07BF078C07CF079C07DF00A0EF7
:1073280005D0D8907D337C337B337A33E82EF9D778
:1073380020EE16F07451D9267551DA227A51DE26DC
:107348007B51DE227C51DE227D51DE227A69010EDC
:107358007B6F76C07CF077C07DF07A517C177B51CB
:107368007D178CC07EF08DC07FF07C517E277D51CB
:107378007F232F0E7E27000E7F2320EE1AF07451F4
:10738800D9267551DA227EC0DEFF7FC0DDFF000CF2
:10739800350E0101796F0B0E7A6FE9C00EF0EAC065
:1073A8000FF0B7EC63F00E5001016D6FC70E0001CE
:1073B8009E6F9F6BA06BA16BA26BA36B7CEC12F012
:1073C8000101766F76510DE0F00E00019C6FFA0E08
:1073D8009D6FADEC67F00001C76BC86BC96BCA6BDA
:1073E8001200C70E0001746F756B79C176F07AC10F
:1073F80077F0010E796F786B740E7A6F010E7B6FE0
:1074080032EC1DF00101766F765108E0990E00010B
:107418009C6FFB0E9D6FADEC67F0DDD779C1D9FF8E
:107428007AC1DAFF800EDE1808E09E0E00019C6F1C
:10743800FC0E9D6FADEC67F0CED720EE0AF07951C7
:10744800D9267A51DA22DF500001EC6FEB6B01018B
:1074580020EE0BF07951D9267A51DA22DF5000015B
:10746800EB250101726F000E0001EC210101736F21
:10747800820E00019C6FFB0E9D6F72C19EF073C15E
:107488009FF0ADEC67F0C70E9E6F9F6B01017251C4
:107498000001EC6FEB6BEBC0A0F0ECC0A1F0A26BAD
:1074A800A36B7CEC12F00101766F765194E1C70E64
:1074B8000001746F756B79C176F07AC177F0010EAF
:1074C800796F786B740E7A6F010E7B6F32EC1DF05A
:1074D8000101766F765101E07ED7776B786BE9C052
:1074E8000EF0EAC00FF077C1EBF078C1ECF0050EB2
:1074F800D8900001EB37EC37E82EFAD7EB510101B1
:107508007925106E0001EC5101017A21116E6DC1CF
:1075180012F0136AD8EC5CF00E500F105DE177C1E1
:10752800EBF078C1ECF0050ED8900001EB37EC37A2
:10753800E82EFAD779C1EDF07AC1EEF0EB51ED27DC
:10754800EC51EE230E0EED25D96E000EEE21DA6E0B
:10755800DF50F06FEF6B77C1F1F078C1F2F0050EF4
:10756800D890F137F237E82EFBD779C1F3F07AC11A
:10757800F4F0F151F327F251F4230F0EF325D96EED
:10758800000EF421DA6EDF50F56FF66BEF51F52738
:10759800F051F623F5C06EF1F6C06FF10101000E4F
:1075A8006FBFFF0E706F716F730E00019C6FFD0E41
:1075B8009D6F6EC19EF06FC19FF070C1A0F071C148
:1075C800A1F0ADEC67F06EC1C7F06FC1C8F070C133
:1075D800C9F071C1CAF01200774B782B78BF7FD7FA
:1075E800785105E10F0E775D01E3F5D678D7F3D62C
:1075F8001850D96EDA6ADECF22F0DDCF23F01C0EE8
:107608001624266E000E1720276E26C00EF027C0FF
:107618000FF0116A200E106E136A0B0E126E2FEC0B
:1076280067F0286A296A246A256A216A080E206E8A
:1076380024502224196E255023201A6E19C0F6FFF3
:107648001AC0F7FF000EF86E0E0EF76403D008009C
:10765800F55005D0F6CFE9FFF7CFEAFFEF502A6ED5
:10766800244A252A210E2A6001D0BED02F0E2A18BE
:1076780006E05C0E2A1803E036D0244A252A245056
:107688002224196E255023201A6E19C0F6FF1AC03D
:10769800F7FF000EF86E0E0EF76403D00800F550E1
:1076A80005D0F6CFE9FFF7CFEAFFEF502F0AE5E064
:1076B80024502224196E255023201A6E19C0F6FF73
:1076C8001AC0F7FF000EF86E0E0EF76403D008001C
:1076D800F55005D0F6CFE9FFF7CFEAFFEF505C0A87
:1076E80001E082D0CAD72E0E2A1805E02050285C67
:1076F800215029580FE30B0E20182110D8B4060C7E
:107708002E0E2A1801E0060C296A080E286E216A36
:107718000B0E8DD72A50D9EC62F00E500F1044E0B2
:1077280024502224196E255023201A6E19C0F6FF02
:107738001AC0F7FF000EF86E0E0EF76403D00800AB
:10774800F55005D0F6CFE9FFF7CFEAFFEF501F6EEF
:10775800244A252A1F5048EC60F00E500F10D8B468
:10776800060C19681A6820C01BF021C01CF01950BB
:107778001B261A501C221B50285C1C50295801E358
:10778800060C28502624D96E29502720DA6E2AC0E4
:10779800DFFF284A292A28502624D96E2950272075
:1077A800DA6E1FC0DFFF1DD0910E0E6EFD0E0F6E3C
:1077B8002AC010F0116A28EC65F00E500F1001E095
:1077C800060C600E2A6405D07B0E2A6002D0200EBB
:1077D8002A5E28502624D96E29502720DA6E2AC01E
:1077E800DFFF284A292A24D724502224196E25503D
:1077F80023201A6E1850D96EDA6A19C0DEFF1AC033
:10780800DDFF2850291001E1060C26C0D9FF27C04A
:10781800DAFFE50EDE1806E126C0D9FF27C0DAFF39
:10782800050EDF6E200E2A6403D01D6A1E6A03D07F
:107838001E6A040E1D6E20EE0BF02650D926275026
:10784800DA221DC0DFFF000C0001F26FEE5102E0EA
:1078580004EC32F00001F16BED5101E1F8D0040EB7
:10786800F21902E1525003E1140EF21909E1010183
:107878005F6B4E6A4F6A0001EE6B070EED6F070CE7
:107888003F0EF21907E1526A01015F6B0001ED6BCF
:10789800EE6B12005F0EF21907E10101606B5F6B7E
:1078A8000001ED6BEE6B12003F0EF26506D05F0E25
:1078B800F26103D0400EF219F0E1400EF21909E12D
:1078C800010E0101606F01015F6B0001ED6BEE6B52
:1078D8001200200EF21903E1010E526EF4D7650E64
:1078E800F21909E1525007E04E6A4F6A010E010190
:1078F8005F6F8380EAD76E0EF21904E18380020E6F
:1079080001015F6F700E0001F21907E1010160517A
:1079180004E04E6A4F6A030E5F6F700E0001F219A1
:1079280008E1525006E083804E6A4F6A040E010156
:107938000FD0720EF21901E08AD0525001E187D0BF
:10794800838001015D6B1C0E4F6E2A0E4E6E050E74
:107958005F6FBBD7F251CCEC08F00001F16F8CD00F
:107968008390BC0E4E1809E1020E4F1806E15FEC39
:107978003EF001015F6B516AA8D7F25109EC53F050
:107988000001F16F01015F6B77D08380350E0E6EB9
:107998000B0E0F6E116A106A010E136E126A96ECC6
:1079A8004CF002500209026E2BEE35F051C0DFFF99
:1079B80001014A4B4B2B52514A1904E153514B19BF
:1079C80001E1889C010E66EC5BF0170E00019C6FCC
:1079D800FF0E9D6F51C09EF09F6BADEC67F0029259
:1079E800080EF16F01015F6B516A46D08390F16B0D
:1079F80043D0080EF21915E18390536AF16B516A6E
:107A0800030E01015D6513D00F0E5D1910E0010E24
:107A1800516E02011B5110091B6F09D04E6A4F6A43
:107A28002BD0090EF21906E18390F16B516A01011E
:107A38005F6BF4D71F0EF2651FD0300EF2611CD0B9
:107A4800F2510F0B01015D6F0001F16BCDD7010100
:107A58005F510001EF6FF06BF0510EE1EF510CE058
:107A6800010A01E177D7030A01E17AD7010A8DE01B
:107A7800070ABCE0010ABDE0F1C0EDF00001EE6BC1
:107A8800120001016B6B546B556BFF0E2124256EA0
:107A9800FF0E2220266E89868980898289848988BA
:107AA8008B68849084928494849883500F011391F6
:107AB800350EE82EFED700F007D0FC0E00019C6FB3
:107AC800FF0E9D6FADEC67F08EA8F7D7E1D08EA8BA
:107AD8008EAA14D0FB5112E1545155110FE0E20E59
:107AE80000019C6FFC0E9D6F54C19EF055C19FF024
:107AF800ADEC67F0630E01016B6FD0D0100E3C6FD8
:107B0800270E3D6F3E6B3F6BABD08EB28EA410D06C
:107B18003C07000E3D5B3E5B3F5B3C2906E13D298F
:107B280004E13E2902E13F29D8A4B2D0620E84D0F4
:107B3800010E82D08EA8ACD0020E7ED0350E542510
:107B4800D96E0B0E5521DA6EDF1C866E545125183E
:107B580005E15551261802E102B2899A544B552B7A
:107B68008B6A030E6B6F100E3C6F270E3D6F3E6BDA
:107B78003F6B06D08EA204D08990050E6B6F0ED095
:107B88003C07000E3D5B3E5B3F5B3C29F3E13D2932
:107B9800F1E13E29EFE13F297BE0ECD7100E3C6F85
:107BA800270E3D6F3E6B3F6B0DD08EA40BD0898A9C
:107BB80089808B682150545D22505559BDE3630E6E
:107BC80001013AD03C07000E3D5B3E5B3F5B3C2920
:107BD800ECE13D29EAE13E29E8E13F2959E0E5D712
:107BE8008EB20DD03C07000E3D5B3E5B3F5B3C29EF
:107BF8004FE13D294DE13E294BE13F2949E1040E82
:107C08001BD08990050E6B6F100E3C6F270E3D6FD1
:107C18003E6B3F6B3DD089848EB40DD03C07000E7F
:107C28003D5B3E5B3F5B3C2933E13D2931E13E2929
:107C38002FE13F292DE1060E6B6F2AD0898A8980B2
:107C48008B682150545D2250555901E271D7B7D73E
:107C58009E0E00019C6FFF0E9D6FADEC67F0AFD7D5
:107C68006B51236E246A245013E1235001E14DD750
:107C7800010A01E15FD7030A01E160D7010AB0E018
:107C8800070ABFE0010AC7E0030AD8E0640AE0E097
:107C9800630E01016B1902E08EBC19D789808982B5
:107CA80089848988898A8B680F01138154C121F0DE
:107CB80055C122F0120002500209026E350E0E6EF6
:107CC8000B0E0F6E116A106A010E136E126A96EC93
:107CD8004CF0040E531804E10F0EE8CF35FB04D026
:107CE8002BEE35F053C0DFFFFF0EE8CF36FB020165
:107CF8001B5102E0000E0BD0395102E0010E07D0F3
:107D0800575102E0020E03D0755103E0030EE8CF8D
:107D180036FB050E53604ED053501E0D1B0EF32438
:107D2800D96E020EF420DA6EDFA403D0810EE8CFFC
:107D380037FB53501E0D1B0EF324D96E020EF42090
:107D4800DA6EDFA803D0020EE8CF37FB53501E0DC2
:107D58001B0EF324D96E020EF420DA6EDFA003D0D6
:107D6800020EE8CF39FB53501E0D1B0EF324D96EBB
:107D7800020EF420DA6EDFA203D0020EE8CF39FB40
:107D880053501E0D1B0EF324D96E020EF420DA6E2A
:107D9800DFA603D0800EE8CF38FB53501E0D1B0E14
:107DA800F324D96E020EF420DA6EDFAA03D0040E93
:107DB800E8CF37FB8FA403D0080EE8CF3BFB2C6A33
:107DC8002D6A300E2C24D96E010E2D20DA6EDF1CA0
:107DD8002B6E370E2C24D96E0B0E2D20DA6E370E33
:107DE8002C24E16E0B0E2D20E26EE7502B14DF6E73
:107DF8002C4A2D2A2DBEE5D72D5003E1070E2C5C09
:107E0800E0E3516A020E01015D6548D053501E0D32
:107E1800010EF324D96E020EF420DA6EDF502A6EBA
:107E28002AC03FFB53501E0D020EF324D96E020EDA
:107E3800F420DA6EDF502A6E2AC040FB53501E0D24
:107E4800030EF324D96E020EF420DA6EDF502A6E88
:107E58002AC041FB53501E0D040EF324D96E020EA6
:107E6800F420DA6EDF502A6E2AC042FB53501E0DF2
:107E7800050EF324D96E020EF420DA6EDF502A6E56
:107E88002AC043FB53501E0D060EF324D96E020E72
:107E9800F420DA6EDF502A6E2AC044FB53501E0DC0
:107EA8001B0EF324D96E020EF420DA6E000EDF6E7C
:107EB800140E66EC5BF0350E216E0B0E226E000E72
:107EC800246E140E236ECC0E256EFF0E266E80ECEB
:107ED80061F00292839012000001D16B010ED06F05
:107EE800838E8380D26BD36BD46BD56BE1D0535028
:107EF800220D000EF324746F030EF420756F350EF7
:107F0800766F0B0E776F010E796F786BD80E7A6FDC
:107F18007B6B32EC1DF0DA6FDA5118E0180E0101B4
:107F2800596F010E5B6F0001D96BD86F0A0E9C6FF9
:107F3800FA0E9D6F53C09EF09F6BDAC0A0F0A16B44
:107F4800D8C0A2F0D9C0A3F0ADEC67F0010162512E
:107F580035E0385139113A113B1130E053500C0DCE
:107F6800040EF324D96E010EF420DA6E38C1C7F07E
:107F780039C1C8F03AC1C9F00001C66B000EC62568
:107F8800CA6F010EC721CB6F000EC821CC6F000E3F
:107F9800C921CD6FDE50CA1911E1DE50CB190EE1AF
:107FA800DE50CC190BE1DE50CD1908E1350E2B6EF1
:107FB8000B0E2C6E01016251FFEC54F0029201018C
:107FC800595103E002500209026ED8C021F0D9C00D
:107FD80022F045EC3DF021C0D6F022C0D7F0CF0EFC
:107FE80000019C6FFE0E9D6FADEC67F0D651D22755
:107FF800D751D323000ED423D5238EBC8EA85DD0B1
:10800800D851D61903E1D951D7190CE0310E9C6F1C
:10801800FE0E9D6FD6C09EF0D7C09FF0ADEC67F006
:1080280083944BD064EC67F0CBEC65F021502210C0
:1080380004E0010E01015B6F40D00001CF6B050E1B
:10804800CE6F1CD0D00E0001C26FC90EE82EFED72D
:10805800C22FFCD700D0CBEC65F0215022100EE0E7
:108068000001D06BD16BF30E9C6FFC0E9D6FCEC0E0
:108078009EF0CFC09FF0ADEC67F008D00001CE07AE
:10808800D8A0CF07CE29DEE1CF29DCE18EB808D011
:108098000E0E9C6FFF0E9D6FADEC67F0D06BD16B31
:1080A800CBEC65F02150221003E00001D06BD16BBE
:1080B8000001D051D11101E01AD701015B6B839EF9
:1080C80083901200838E8380516A56EC41F001013F
:1080D8009B6F9B5102E09B5112006C6B936B946BEE
:1080E800956B966B996B010E986F9E6BD0D09C6BBD
:1080F8009D6B1CD0CBEC65F02150221015E09E0E34
:108108000E6E010E0F6EF0EC5DF00101976F000E20
:108118006C25D96EDA6A040EDA2297C1DFFF6C2B60
:108128009C4B9D2B9EBB05D08EAC03D001019D05B9
:10813800E1E301019C5193279D519423000E95235F
:10814800962353501E0D170EF324D96E020EF420F9
:10815800DA6EDE50935DDE509459DE509559DE504C
:10816800965902E3986B996B9EAB02D0986B996B0A
:108178008EBC02D0986B996B9D0519E2000E6C2598
:108188000E6E0F6A040E0F22FF0E6C25D96EDA6A86
:10819800030EDA22DF50106E116A6C510008126E5D
:1081A800000ED8A0E82A0108136E96EC4CF00101E5
:1081B800625145E0385139113A113B1140E05350B2
:1081C8003EE153501E0D070EF324D96E020EF42023
:1081D800DA6E38C188F139C189F13AC18AF1876B01
:1081E800000E87258B6F010E88218C6F000E892168
:1081F8008D6F000E8A218E6F8F6B906B916B926BD7
:10820800DE508B191CE1DE508C1919E1DE508D19F6
:1082180016E1DE508E1913E1DE508F1910E1DE50A1
:1082280090190DE1DE5091190AE1DE50921907E12B
:10823800000E256E040E266E62511FEC5DF001ECF7
:1082480051F001019A6F6C6B9A5121E03A0E0001CE
:108258009C6FFB0E9D6F9AC19EF09F6BADEC67F013
:10826800010E516E53501E0D1B0EF324D96E020ED3
:10827800F420DA6E53501E0D1B0EF324E16E020E2D
:10828800F420E26EE7500409DF6E51501200985155
:10829800991101E02CD78FA402D0010E516E839062
:1082A800839E000C53501E0D070EF324D96E020E48
:1082B800F420DA6EDECFEBF0DECFECF0DECFEDF0BF
:1082C800DECFEEF053501E0D070EF324D96E020ECA
:1082D800F420DA6E53501E0D0F0EF324E16E020ED9
:1082E800F420E26EDE50E65CDE50E658DE50E658DA
:1082F800DE50E658DE50E658DE50E658DE50E658C6
:10830800DE50E65815E2010E516E53501E0D1B0E3D
:10831800F324D96E020EF420DA6E53501E0D1B0E94
:10832800F324E16E020EF420E26EE7500409DF6EDA
:1083380053501E0D070EF324D96E020EF420DA6E88
:10834800DECFC7F0DECFC8F0DECFC9F0DECFCAF08F
:10835800DECFCBF0DECFCCF0DECFCDF0DECFCEF06F
:1083680053501E0D170EF324D96E020EF420DA6E48
:10837800DECFCFF0DECFD0F0DECFD1F0DECFD2F03F
:108388000001CF51D36FD051D46FD151D56FD25195
:10839800D66FD76BD86BD96BDA6BC751D325DB6F28
:1083A800C851D421DC6FC951D521DD6FCA51D621FE
:1083B800DE6FCB51D721DF6FCC51D821E06FCD5183
:1083C800D921E16FCE51DA21E26F53501E0D0F0E05
:1083D800F324D96E020EF420DA6EDB51DE5CDC5138
:1083E800DE58DD51DE58DE51DE58DF51DE58E051EF
:1083F800DE58E151DE58E251DE5815E2010E516EA9
:1084080053501E0D1B0EF324D96E020EF420DA6EA3
:1084180053501E0D1B0EF324E16E020EF420E26E83
:10842800E7500409DF6E516A5350220D000EF32401
:108438009E6F030EF4209F6FEBC0A0F0ECC0A1F07C
:10844800EDC0A2F0EEC0A3F07CEC12F0EF6FEF519C
:1084580015E0010E516E53501E0D1B0EF324D96EFC
:10846800020EF420DA6E53501E0D1B0EF324E16E3B
:10847800020EF420E26EE7500409DF6E515012003C
:108488008EA604D0940E216EFE0E03D0B30E216E7C
:10849800FF0E226E8EAA04D0940E236EFE0E03D019
:1084A800AE0E236EFF0E246E8EA804D0940E256E99
:1084B800FE0E03D0C10E256EFE0E266E8EAE04D0C3
:1084C800940E276EFE0E03D0B80E276EFF0E286E90
:1084D8008EAC04D0940E296EFE0E03D0A90E296E20
:1084E800FF0E2A6E8EA404D0940E2B6EFE0E03D0BF
:1084F800C20E2B6EFF0E2C6E8EA204D0940E2D6E23
:10850800FE0E03D0C70E2D6EFF0E2E6E8EA004D069
:10851800940E2F6EFE0E03D0BD0E2F6EFF0E306E22
:1085280090AE04D0940E316EFE0E03D0F90E316E6B
:10853800FF0E326E90AC04D0940E336EFE0E03D054
:10854800F60E336EFF0E346E90AA04D0940E356E7C
:10855800FE0E03D0F30E356EFF0E366E90A804D0D3
:10856800940E376EFE0E03D0F00E376EFF0E386E87
:1085780090A604D0940E396EFE0E03D0ED0E396E1F
:10858800FF0E3A6E90A404D0940E3B6EFE0E03D0FC
:10859800EA0E3B6EFF0E3C6E90A204D0940E3D6E28
:1085A800FE0E03D0E70E3D6EFF0E3E6E90A004D087
:1085B800940E3F6EFE0E03D0E40E3F6EFF0E406E2B
:1085C800FA0E00019C6FF80E9D6F901C9E6F9F6BBA
:1085D8008ECFA0F0A16B3FC0A2F040C0A3F03DC079
:1085E800A4F03EC0A5F03BC0A6F03CC0A7F039C03F
:1085F800A8F03AC0A9F037C0AAF038C0ABF035C02F
:10860800ACF036C0ADF033C0AEF034C0AFF031C01E
:10861800B0F032C0B1F02FC0B2F030C0B3F02DC00E
:10862800B4F02EC0B5F02BC0B6F02CC0B7F029C0FE
:10863800B8F02AC0B9F027C0BAF028C0BBF025C0EE
:10864800BCF026C0BDF023C0BEF024C0BFF021C0DE
:10865800C0F022C0C1F0ADEF67F0070E0E241D6E0A
:10866800000E0F201E6E0EC0D9FF0FC0DAFFDF50BC
:10867800126E12380F0B0A0DF3CF13F0F4CF14F06B
:108688000EC0D9FF0FC0DAFFDF500F0B1326000E04
:10869800142213281B6E000E14201C6E206A010E73
:1086A8001F6E216A226A236A246AB2D01F502010E2
:1086B80054E021C012F022C013F023C014F024C0EB
:1086C80015F00A0E1202F3CF16F0F4CF17F0186A5D
:1086D800196A1302F3501726F4501822000E1922B3
:1086E8001202F3501726F4501822000E19220A0E0F
:1086F8001402F3501826F4501922000E1302F350F6
:108708001826F4501922000E1202F3501826F450BD
:1087180019220A0E1502F3501926000E1402F350FE
:108728001926000E1302F3501926000E1202F350F8
:1087380019261DC0D9FF1EC0DAFFDF501A6E1A387D
:108748000F0B1624216E000E1720226E000E182023
:10875800236E000E1920246E54D021C012F022C0BE
:1087680013F023C014F024C015F00A0E1202F3CF40
:1087780016F0F4CF17F0186A196A1302F350172687
:10878800F4501822000E19221202F3501726F45042
:108798001822000E19220A0E1402F3501826F4505B
:1087A8001922000E1302F3501826F4501922000E55
:1087B8001202F3501826F45019220A0E1502F3502B
:1087C8001926000E1402F3501926000E1302F35056
:1087D8001926000E1202F35019261DC0D9FF1EC01B
:1087E800DAFFDF500F0B1624216E000E1720226EC1
:1087F800000E1820236E000E1920246E1D06D8A026
:108808001E061F502010010ED8A4000E1F6E206AED
:108818001B06D8A01C061B2802E11C28D8A446D792
:1088280021C00EF022C00FF023C010F024C011F0B8
:10883800120046C027F047C028F02BEC48F0486EDD
:10884800485001E0D4D046C0D9FF47C0DAFF030E34
:10885800DE1801E0BCD020EE04F04650D92647507F
:10886800DA22DE0401E0B3D02F0E46240E6E000E8D
:1088780047200F6E116A106A020E136E126A2FECEF
:1088880067F02D0E46240E6E020E47200F6EAA0EBC
:10889800116E550E106EF5EC66F02F0E46240E6E16
:1088A800000E47200F6E520E106E116E610E126E82
:1088B800410E136EB6EC60F0130E46240E6E020ED7
:1088C80047200F6E720E106E116E410E126E610E01
:1088D800136EB6EC60F0170E46240E6E020E47209B
:1088E8000F6E20EE0FF04650D9264750DA22DECF21
:1088F80010F0DECF11F0DECF12F0DECF13F0B6ECC1
:1089080060F01B0E46240E6E020E47200F6E20EEFE
:108918000BF04650D9264750DA22DECF10F0DECFD2
:1089280011F0DECF12F0DECF13F0B6EC60F020EEDF
:108938001BF04650D9264750DA22DECF60F0DECF52
:1089480061F0DECF62F0DECF63F0010E000160253A
:10895800646F000E6121656F000E6221666F000E64
:108968006321676F20EE2BF04650D9264750DA2254
:1089780064C0DEFF65C0DEFF66C0DEFF67C0DEFFE5
:108988002F0E46241D6E000E47201E6E20EE2BF083
:108998004650D9264750DA22DECF1FF0DECF20F02E
:1089A800DECF21F0DECF22F0246A010E236E20EE06
:1089B80001F04650D9264750DA22DF5060EC56F0D5
:1089C80020EE04F04650D9264750DA22DF6A1D6AA5
:1089D8001E6A1F6A20EE01F04650D9264750DA2257
:1089E800DF5018EC24F0000902E0010E486E4850F0
:1089F80012006251D8B41200230E00019C6FFD0EC4
:108A08009D6FADEC67F07BEC5AF021C07DF122C080
:108A18007EF123C07FF124C080F101017D517E11D8
:108A28007F11801117E1DE0E00019C6FFB0E9D6F18
:108A38007DC19EF07EC19FF07FC1A0F080C1A1F0F2
:108A4800ADEC67F00A0E116E000E126A136A146A12
:108A58005EEC62F00101816B826BE00E00019C6F9D
:108A6800FF0E9D6F7D0E01018125D96E010E8221B9
:108A7800DA6EDF5000019E6F9F6BADEC67F001016D
:108A8800814B822B82BFE9D7825103E1040E815DBD
:108A9800E4E3740E00019C6FF90E9D6FADEC67F076
:108AA800BC0E9C6FFA0E9D6FADEC67F023EE00F0E4
:108AB80000EEC7F0210EDBCFEBFFE806FCE2D40E98
:108AC800E96FFF0EEA6FCCEC39F0C7C038F1C8C0C7
:108AD80039F1C9C03AF1CAC03BF101013851391125
:108AE8003A113B11D8B41200A20E00019C6FFA0E85
:108AF8009D6F38C19EF039C19FF03AC1A0F03BC1CB
:108B0800A1F0ADEC67F0000E9E6F030E9F6F38C1A9
:108B1800F8F039C1F9F03AC1FAF0F76B000EF72511
:108B2800A06F010EF821A16F000EF921A26F000EAF
:108B3800FA21A36F7CEC12F00101686F000E0001AE
:108B4800746F030E756F350E766F0B0E776F796B3A
:108B5800080E786F7B0E7A6F010E7B6F32EC1DF07A
:108B68000101686F836B846B9A0E00019C6FFC0E89
:108B78009D6F350E01018325D96E0B0E8421DA6EA7
:108B8800DF5000019E6F9F6BADEC67F00101834BD6
:108B9800842B84BFE9D7845105E1080E835DD8B0E2
:108BA8001200E2D71200C0C0D9FFC1C0DAFFDECF81
:108BB800CAF0DDCFCBF003D00001C24BC32BC2C03B
:108BC800F6FFC3C0F7FF000EF86E0E0EF76403D071
:108BD8000800F55005D0F6CFE9FFF7CFEAFFEF50D0
:108BE8002F0AEAE0C2C0F6FFC3C0F7FF000EF86E16
:108BF8000E0EF76403D00800F55005D0F6CFE9FF54
:108C0800F7CFEAFFEF505C0AD7E0000120EE06F04C
:108C1800C051D926C151DA22DE6ADE6ADE6ADD6A0F
:108C2800C2C0F6FFC3C0F7FF000EF86E0E0EF76461
:108C380003D00800F55005D0F6CFE9FFF7CFEAFFDB
:108C4800EF500001C46F200EC46114D020EE27F04D
:108C5800C051D926C151DA22800EDF6EC0C074F02F
:108C6800C1C075F0000E766F776F786F796F5BEC27
:108C780038F023D0C0C016F0C1C017F0C20E186E6D
:108C8800FCEC3AF00001CD6FCD5158E1C0C0B8F00E
:108C9800C1C0B9F02CEC4DF0CD6F20EE27F0C051DB
:108CA800D926C151DA22DF50CC6FCD5108E0040E2D
:108CB800CD1944E1CCB542D0050ECD6F3FD0CCB52F
:108CC8003DD020EE04F0C051D926C151DA22DFA8E8
:108CD800F3D7CAC015F0CBC016F0C469010EC56F32
:108CE80020EE0EF0C051D926C151DA22DECFC6F0EF
:108CF800DDCFC7F0C451C617C551C717CAC0C8F0E1
:108D0800CBC0C9F0C651C827C751C9232F0EC825E3
:108D1800176E000EC921186E65EC5FF0000120EE99
:108D280006F0C051D926C151DA2215C0DEFF16C09F
:108D3800DEFF17C0DEFF18C0DEFF9CD7CD51120042
:108D480081C0D9FF82C0DAFFDECF98F0DDCF99F07D
:108D580086518511841104E1020E835DD8A0020CAE
:108D680020EE13F09851D9269951DA22DE50835D0E
:108D7800DE508459DE508559DE50865901E3020CD5
:108D88008751881189118A1117E098C060F099C03D
:108D980061F087C062F088C063F089C064F08AC05F
:108DA80065F06669676968696969FBEC21F0976F26
:108DB800975102E09751120081C045F082C046F0F9
:108DC80083C047F084C048F085C049F086C04AF0A7
:108DD80045EC30F045C093F046C094F047C095F09C
:108DE80048C096F00001935194119511961170E0C6
:108DF800930594119511961101E1020C932907E14D
:108E0800942905E1952903E1962901E1010C98C00F
:108E180060F099C061F083C062F084C063F085C0DF
:108E280064F086C065F0666B676B686B696BFBEC1A
:108E380021F0976F9751BEE120EE13F09851D92693
:108E48009951DA22FE0EDE248B6FFF0EDE208C6F26
:108E5800FF0EDE208D6FFF0EDE208E6F20EE0FF0EE
:108E68009851D9269951DA228B51DE5C8C51DE5803
:108E78008D51DE588E51DE5813E220EE0FF09851D6
:108E8800D9269951DA22DE2A000EDE22DE22DE22DF
:108E980020EE04F09851D9269951DA22000EDB8091
:108EA80093C083F094C084F095C085F096C086F096
:108EB80020EE13F09851D9269951DA22DE50835DBD
:108EC800DE508459DE508559DE50865901E274D748
:108ED800000C1E6E1E5001E0010C55A202D0555028
:108EE8001200000EE1EC66F00A0E296E03D0C9EC00
:108EF80067F029062950FBE1266A000E176A186AEE
:108F0800196A1A6A44EC65F0E80601E097D0AA0EDF
:108F1800176E010E186E196A1A6A080E44EC65F08D
:108F2800E80651E1296A29501F0FD96EDA6AC9EC9F
:108F380067F0DF6E292A030E2964F5D721047EE144
:108F4800AA0E22187BE1030E286EE80E276E15D0B4
:108F5800176A186A196A400E1A6EA90E44EC65F071
:108F680000090EE0150E1D6EC60EE82EFED71D2E4A
:108F7800FCD700D02706D8A0280627502810E8E1FB
:108F8800275028105BE0176A186A196A1A6A3A0E9D
:108F980044EC65F0000952E1296A29501F0FD96E87
:108FA800DA6AC9EC67F0DF6E292A030E2964F5D75F
:108FB8001FBC03D0246A040E02D0246A0C0E236E50
:108FC80023C026F03BD0176A186A196A1A6AA90ED4
:108FD80044EC65F01D6E020E1D6003D0266EA90ECE
:108FE80002D0010E266E256E030E286EE80E276E3F
:108FF80014D0176A186A196A1A6A255044EC65F081
:1090080000090EE0150E1D6EC60EE82EFED71D2EA9
:10901800FCD700D02706D8A0280627502810E9E159
:10902800275028100AE0176A020E186E196A1A6A81
:10903800100E44EC65F0000901E0266A26C054F0E1
:10904800D6EC67F0265001E14AD7559048D7396ADF
:1090580020EE03F02750D9262850DA22DF5001E10C
:10906800A7D02F0E27241D6E000E28201E6E20EE7E
:109078002BF02750D9262850DA22DECF1FF0DECF7A
:1090880020F0DECF21F0DECF22F0246A010E236E1D
:1090980020EE01F02750D9262850DA22DF5060EC64
:1090A80056F0000901E082D020EE03F02750D926BF
:1090B8002850DA22DF6A20EE17F02750D9262850E8
:1090C800DA2210EE1FF02750E1262850E222E6CFE0
:1090D8002DF0E6CF2EF0E6CF2FF0E6CF30F010EEF1
:1090E8002BF02750E1262850E222E6CF31F0E6CFD8
:1090F80032F0E6CF33F0E6CF34F02D50315C356EE8
:109108002E503258366E2F503358376E30503458F0
:10911800386EDE50355CDE503658DE503758DE503B
:10912800385846E220EE02F02750D9262850DA2295
:10913800020EDE183DE12F0E27241D6E000E28209A
:109148001E6E20EE17F02750D9262850DA22DECFDF
:1091580029F0DECF2AF0DECF2BF0DECF2CF020EE88
:109168002BF02750D9262850DA22DECF2DF0DECF7B
:109178002EF0DECF2FF0DECF30F029502D241F6ED9
:109188002A502E20206E2B502F20216E2C5030205C
:10919800226E246A010E236E20EE01F02750D92694
:1091A8002850DA22DF5060EC56F002D0010E396EFA
:1091B8003950120049C00FF04AC010F0690E116E04
:1091C8007FEC59F00001686F685101E099D020EEFA
:1091D8000EF04950D9264A50DA22DFAC91D069C046
:1091E8003AF06AC03BF020EE1CF04950D9264A50AC
:1091F800DA22DECF3CF0DECF3DF0DECF3EF0DECF30
:109208003FF018EC5BF00001686F685179E120EEDF
:1092180020F04950D9264A50DA22DECF6BF0DDCF54
:109228006CF020EE0BF06B51D9266C51DA22000E4F
:10923800DB8A49C0D9FF4AC0DAFFDECF12F0DDCFA2
:1092480013F06BC014F06CC015F020EE06F0495016
:10925800D9264A50DA22DECF16F0DECF17F0DECF5D
:1092680018F0DECF19F039EC64F01C0E00016B2504
:109278000E6E000E6C210F6E20EE0AF04950D926B2
:109288004A50DA22DECF10F0DECF11F0DECF12F036
:10929800DECF13F0B6EC60F0160E00016B250E6EF3
:1092A800000E6C210F6E106A116A210E126E500E9C
:1092B800136EB6EC60F0120E00016B250E6E000EF8
:1092C8006C210F6E000E116A106AF5EC66F0000151
:1092D80020EE03F06951D9266A51DA22010EDF6EB9
:1092E80069C046F06AC047F01DEC44F00001686FA1
:1092F80020EE0EF04950D9264A50DA22BF0EDF166A
:109308006851120089688B68F29E8E280BE1090E5D
:1093180000019C6FFB0E9D6F8ECF9EF09F6BADEC96
:1093280067F00AD0C20E00019C6FF90E9D6F8ECFB8
:109338009EF09F6BADEC67F090280AE1C70E9C6F1A
:10934800FB0E9D6F8ECF9EF09F6BADEC67F009D042
:10935800E70E9C6FF90E9D6F8ECF9EF09F6BADEC64
:1093680067F0290E426E960E416E7F0EE82EFED7EC
:10937800412EFCD7422EFAD700F04B0E00019C6F0D
:10938800FE0E9D6FADEC67F089988498090E426EC9
:109398001E0E416EE40EE82EFED7412EFCD7422E5B
:1093A800FAD700D03E0E00019C6FFE0E9D6FADEC0B
:1093B80067F0899A849A090E426E1E0E416EE40E79
:1093C800E82EFED7412EFCD7422EFAD700D0AF0E9A
:1093D80000019C6FFE0E9D6FADEC67F088908D903C
:1093E80090280AE0C70E9C6FFB0E9D6F90CF9EF0F1
:1093F8009F6BADEC67F009D0770E9C6FF90E9D6FEF
:1094080090CF9EF09F6BADEC67F08D80A30E426EFF
:10941800570E416E020EE82EFED7412EFCD7422E83
:10942800FAD700D089688B688A6883928382290E6C
:10943800426E960E416E7F0EE82EFED7412EFCD767
:10944800422EFAD700F044EC42F0EFD71F6A1DAE67
:1094580012D01D1E1C1E1B1E1A1E191E181E171E9A
:10946800166C000E1722182219221A221B221C22FF
:109478001D22010E1F6E15AE12D0151E141E131ECE
:10948800121E111E101E0F1E0E6C000E0F2210222F
:1094980011221222132214221522010E1F1A206AE9
:1094A800216A226A236A246A256A266A276A16506C
:1094B8001710181019101A101B101C101D1045E059
:1094C800010E1E6E0AD0D890163617361836193681
:1094D8001A361B361C361D361E2A1DAEF4D7D890F8
:1094E80020362136223623362436253626362736A8
:1094F80016500E5C17500F58185010581950115824
:109508001A5012581B5013581C5014581D501558F7
:1095180011E316500E5E17500F5A1850105A195072
:10952800115A1A50125A1B50135A1C50145A1D50D3
:10953800155A2080D8901D321C321B321A3219322B
:109548001832173216321E2ECAD71F5010E0271EA7
:10955800261E251E241E231E221E211E206C000EE0
:10956800212222222322242225222622272220C029
:109578000EF021C00FF022C010F023C011F024C05B
:1095880012F025C013F026C014F027C015F0120001
:10959800176818680E50D96EDA6ADECF19F0DDCF79
:1095A8001AF019C014F01AC015F019501A1003E176
:1095B8000E680F68120014C0F6FF15C0F7FF000E02
:1095C800F86E0E0EF76403D00800F55005D0F6CFFC
:1095D800E9FFF7CFEAFFEF50166E144A152A200E5E
:1095E800166403D03A0E1618E6E13A0E161868E12A
:1095F800000E136E010E126E19C0F6FF1AC0F7FFA7
:10960800000EF86E0E0EF76403D00800F55005D072
:10961800F6CFE9FFF7CFEAFFEF50106E2F0E106478
:1096280039D019C0F6FF1AC0F7FF000EF86E0E0EFB
:10963800F76403D00800F55005D0F6CFE9FFF7CF5F
:10964800EAFFEF50106E3A0E106024D0020E192473
:10965800106E000E1A20116E145010181BE11550D0
:10966800111818E119C0F6FF1AC0F7FF000EF86EBE
:109678000E0EF76403D00800F55005D0F6CFE9FFC9
:10968800F7CFEAFFEF50106ED00E1024126E136A57
:10969800FF0E132213BE04D013500DE112040BE287
:1096A80012C017F013C018F00E50D96EDA6A14C041
:1096B800DEFF15C0DDFF17C00EF018C00FF0120056
:1096C8000E6A0F6A120060C045F061C046F0476A32
:1096D800486A496A4A6A07EC54F045C078F046C0BF
:1096E80079F0020E0001781979110DE0795106E13F
:1096F800030E785D03E26251631105E178C060F002
:1097080079C061F012007A6B7B6B7AC064F07BC021
:1097180065F0643B653BF00E651764510F0B6513EC
:10972800F00E641760C066F061C067F06451662788
:1097380065516723F50E66250E6E010E67210F6EC3
:10974800D5EC59F000017A51040DF350680FD96E29
:10975800DA6A0EC0DEFF0FC0DEFF10C0DEFF11C0E8
:10976800DEFF7A4B7B2B7B5103E1040E7A5DCDE360
:109778006251631103E17A6B7B6B06D0FF0E6225A1
:109788007A6FFF0E63217B6F7A51040DF350680FD7
:10979800D96EDA6ADE50DE10DE10DE1004E1796B75
:1097A800030E786F18D060C045F061C046F07A515A
:1097B800040DF350680FD96EDA6ADECF47F0DECFBA
:1097C80048F0DECF49F0DECF4AF007EC54F045C050
:1097D80078F046C079F00001625163118FE1795148
:1097E80003E1020E785D8AE37A4B7B2B7B5186E19D
:1097F800040E7A5D83E2C8D72F6C69666461746170
:10980800302E62696E20002F6C6966646174613164
:109818002E62696E20002F6C696664617461322E55
:1098280062696E20002F6C696664617461332E6210
:10983800696E20002F6C696664617461342E6269F8
:109848006E20002F6C696664617461352E62696EE2
:1098580020002F6C696664617461362E62696E201F
:10986800002F6C696664617461372E62696E20002E
:109878002F6C696664617461382E62696E20002FEE
:109888006C696664617461392E62696E20002F6CA0
:10989800696664617461612E62696E20002F6C696B
:1098A8006664617461622E62696E20002F6C69665D
:1098B80064617461632E62696E20002F6C6966644E
:1098C800617461642E62696E20002F6C6966646140
:1098D8007461652E62696E20002F6C69666461741C
:1098E80061662E62696E2000000000000000000022
:1098F8000000000000000000000000000000000060
:10990800000000000000000000000000000000004F
:10991800000000000000000000000000000000003F
:10992800000000000EC018F00FC019F012501310FC
:1099380001E1120018C0D9FF19C0DAFF10C0DFFF1B
:1099480012501824146E13501920156EFF0E14248B
:10995800D96EFF0E1520DA6E10C0DFFF135004E138
:10996800030E125C01E2120020EE01F01850D92615
:109978001950DA2210C0DFFF20EE02F01850D92665
:109988001950DA2210C0DFFF12501824146E135039
:109998001920156EFE0E1424D96EFF0E1520DA6EEE
:1099A80010C0DFFF12501824146E13501920156EC2
:1099B800FD0E1424D96EFF0E1520DA6E10C0DFFFDD
:1099C800135004E1070E125C01E2120020EE03F0CE
:1099D8001850D9261950DA2210C0DFFF1250182467
:1099E800146E13501920156EFC0E1424D96EFF0E38
:1099F8001520DA6E10C0DFFF135004E1090E125C67
:109A080001E2120018C014F019C015F0141E151E3A
:109A1800144A152A030E1414166E176A16501826BF
:109A2800175019221650125E1750135AFC0E1216B0
:109A38000BD018C0D9FF19C0DAFF10C0DFFF12061B
:109A4800D8A01306184A192A12501310F2E112006E
:109A5800B8C0D9FFB9C0DAFFDECFBCF0DDCFBDF0AA
:109A6800B8C074F0B9C075F0000E766F776F786F74
:109A7800796F5BEC38F0BF6FBF5103E00001BF5155
:109A88001200BCC03AF0BDC03BF020EE16F0B85151
:109A9800D926B951DA22DECF3CF0DECF3DF0DECF59
:109AA8003EF0DECF3FF018EC5BF00001BF6FBF5116
:109AB800E5E120EE1AF0B851D926B951DA22DECF05
:109AC800BAF0DDCFBBF0BAC0D9FFBBC0DAFFDF50B8
:109AD800BE6FBE5103E1040EBF6FD0D720EE04F075
:109AE800B851D926B951DA2210EE1AF0B851E12648
:109AF800B951E22200EE0BF0E650E926E550EA22E1
:109B0800EF503F0BDF6E20EE1AF0B851D926B9514D
:109B1800DA2210EE0BF0DE50E126DD50E222E7B645
:109B280018D020EE1AF0B851D926B951DA22DECF72
:109B38000EF0DDCF0FF01C0EB825106E000EB92107
:109B4800116E136A0B0E126E80EC60F00E500F103F
:109B580095E0B8C09EF0B9C09FF00001A16BA06B62
:109B6800BFEC33F00001BF6FBF5188E18AD71BC03B
:109B78000EF01CC00FF0116A106A136A080E126EFC
:109B880096EC4CF0266A020E256E25501B24D96EE1
:109B980026501C20DA6E25501B24216E26501C20CE
:109BA800226E2128E16E000E2220E26EE750236E1D
:109BB800233AF00E2316231625501B24E16E265057
:109BC8001C20E26EE750246E24380F0B2310DF6E42
:109BD800254A262A26BED9D7265003E1070E255C3A
:109BE800D4E325501B24D96E26501C20DA6E1DC0E4
:109BF8000EF01EC00FF01FC010F020C011F00A0EAA
:109C0800126E136A146A156A1FEC61F00E3AF00EB0
:109C18000E1625501B24E16E26501C20E26EE750DC
:109C2800216E21380F0B0E10DF6E1BC0D9FF1CC030
:109C3800DAFFDF2A1DC00EF01EC00FF01FC010F0A3
:109C480020C011F00A0E126E136A146A156AF0EC3D
:109C58005EF00EC01DF00FC01EF010C01FF011C046
:109C680020F01D501E101F1020108CE11BC0D9FFC2
:109C78001CC0DAFFDF06090EDF64090C1BC0D9FF20
:109C88001CC0DAFF100EDF6E100C000E0101AF6F62
:109C98000A0EAE6F000EAD6F050EAC6F7DD00101E0
:109CA800AF6B140EAE6F70D01E0E0F6EFC0E106EE2
:109CB80034EC62F08FB204D00101AF6B1E0EAE6FB0
:109CC800090E0001FE6F1E0EFD6FE40EE82EFED792
:109CD800FD2FFCD7FE2FFAD700F056D0970E0F6E47
:109CE800FE0E106E34EC62F0060E0001B16F090E24
:109CF800B26F760EB36FF90EB46FB56B90EC5CF083
:109D08000101686F6851B0EC62F001016851D8E157
:109D1800AF6B230ED4D7DC0E0F6EFD0E106E34EC35
:109D280062F0000E0001CE6F030ECF6FE50ED06F0C
:109D3800010ED16F010ED26F4AEC15F00101686F68
:109D48006851B0EC62F0010168510AE149EC2AF06F
:109D5800000E6D6F030E6E6FB5EC64F00101686F55
:109D68006851B0EC62F0010CAEC1FDF0AFC1FEF07D
:109D78000001FE5109E1FD510A0A91E01E0A94E032
:109D88000A0AACE03D0AC7E0140E0101AE19AF1192
:109D980003E0AC07D8A0AD07ADBF000CAD51E4E1BE
:109DA800AC05E2E2000C1F6A15AE12D0151E141E97
:109DB800131E121E111E101E0F1E0E6C000E0F22F7
:109DC800102211221222132214221522010E1F6EB4
:109DD8001DAE10D01D1E1C1E1B1E1A1E191E181E7D
:109DE800171E166C000E1722182219221A221B227F
:109DF8001C221D2216501710181019101A101B10AB
:109E08001C101D103BE0010E1E6E0AD0D8901636AD
:109E18001736183619361A361B361C361D361E2AC2
:109E28001DAEF4D716500E5C17500F581850105826
:109E3800195011581A5012581B5013581C501458C6
:109E48001D50155810E316500E5E17500F5A185033
:109E5800105A1950115A1A50125A1B50135A1C50A2
:109E6800145A1D50155AD8901D321C321B321A3202
:109E780019321832173216321E2ED4D71F5010E05E
:109E8800151E141E131E121E111E101E0F1E0E6C00
:109E9800000E0F2210221122122213221422152240
:109EA8000EC00EF00FC00FF010C010F011C011F06E
:109EB80012C012F013C013F014C014F015C015F03E
:109EC8001200FAC123F079D042EC67F0236EFA1938
:109ED80001E182D0290E226E960E216E7F0EE82EA9
:109EE800FED7212EFCD7222EFAD700F075D04FECE2
:109EF80063F0246E245070E024A002D00101612B8D
:109F080024A202D0010161070F0E01016117000EA2
:109F18000E6EC00E01EC63F0CCEC66F0000E0E6E17
:109F2800C00E01EC63F0010161510F0D350EF324F1
:109F3800126E0D0EF420136EB3EC5EF0110E226E4D
:109F48003C0E216ECB0EE82EFED7212EFCD7222EFA
:109F5800FAD700F024A440D00F6A0E6A61C110F04D
:109F6800EFEC64F00A0E00019C6FFC0E9D6F61C15E
:109F78009EF09F6BADEC67F061C123F0000E0E6E92
:109F8800800E01EC63F0CCEC66F0000E0E6E800ED5
:109F980001EC63F0010161510F0D350EF324126ECF
:109FA8000D0EF420136EB3EC5EF0000E0E6EC00EB4
:109FB80001EC63F0CCEC66F00FD001016451216E26
:109FC800226A225009E12150010A01E17DD7030AE2
:109FD80001E17AD7010A8BE023501200020E105ECD
:109FE800000E115A125A135A20EE13F00E50D926A9
:109FF8000F50DA22FE0EDE24146EFF0EDE20156EE0
:10A00800FF0EDE20166EFF0EDE20176E1450105C59
:10A0180015501158165012581750135805E30E6A68
:10A028000F6A106A116A120020EE27F00E50D92626
:10A038000F50DA22DECF14F0DECF15F0DECF16F0A7
:10A04800DECF17F020EE09F00E50D9260F50DA2295
:10A05800DECF18F0DDCF19F018501A6E19501B6EAC
:10A068001C6A1D6A1A501002F3CF1EF0F4CF1FF0BD
:10A07800206A216A1102F3501F26F4502022000E94
:10A0880021221B501002F3501F26F4502022000EEC
:10A0980021221A501202F3502026F45021221B507C
:10A0A8001102F3502026F45021221C501002F350C4
:10A0B8002026F450212213501A02F35021261B5057
:10A0C8001202F35021261C501102F35021261D5074
:10A0D8001002F350212614501E240E6E15501F2016
:10A0E8000F6E16502020106E17502120116E12008E
:10A0F800838E83800001FB6BFC6B76EC5EF025C0E1
:10A10800FDF026C0FEF0040E0001FE5D07E3000E20
:10A11800FD25FB6FFC0EFE21FC6F04D0FDC0FBF09B
:10A12800FEC0FCF00101625133E0385139113A1197
:10A138003B112EE053500C0D040EF324D96E010E82
:10A14800F420DA6E38C172F139C173F13AC174F191
:10A15800716B000E7125756F010E7221766F000EFE
:10A168007321776F000E7421786FDE50751910E136
:10A17800DE5076190DE1DE5077190AE1DE507819C4
:10A1880007E1000E256E040E266E62511FEC5DF08D
:10A198008FB415D05350220D000EF32400019E6F8A
:10A1A800030EF4209F6F000EA06F040EA16F010E26
:10A1B800A36FA26BFB0EA46F1AEC0CF0FA6F0001F0
:10A1C800FA5109E0130E9C6FFD0E9D6FFAC09EF0C8
:10A1D8009F6BADEC67F04AEC2EF05B6B8390839E2F
:10A1E8007C0E00019C6FFC0E9D6FCECF9EF09F6B86
:10A1F800CDCFA0F0A16BADEF67F053501E0D070E49
:10A20800F324D96E020EF420DA6EDECF6DF1DECFC4
:10A218006EF1DECF6FF1DECF70F1DECF71F1DECF00
:10A2280072F1DECF73F1DECF74F16DC10EF06EC145
:10A238000FF06FC110F070C111F071C112F072C14E
:10A2480013F073C114F074C115F053501E0D1C0E99
:10A25800F324D96E020EF420DA6EDECF75F1DDCF6D
:10A2680076F175C116F076C117F0186A196A1A6A7C
:10A278001B6A1C6A1D6AAAEC57F00EC077F10FC062
:10A2880078F110C079F111C07AF112C07BF113C0D6
:10A298007CF114C07DF115C07EF177C1F0F078C172
:10A2A800F1F079C1F2F07AC1F3F056EC41F0F66FB3
:10A2B800F65102E0F65112008FB414D05350220D1B
:10A2C800000EF3249E6F030EF4209F6F000EA06F04
:10A2D800040EA16F010EA36FA26BF40EA46F1AEC0B
:10A2E8000CF0F76FF7510BE0130E9C6FFD0E9D6F8E
:10A2F800F7C09EF09F6BADEC67F0F751120089EC48
:10A3080053F0000C3AC027F03BC028F02BEC48F083
:10A31800000901E0010C3AC00EF03BC00FF03CC050
:10A3280010F03DC011F03EC012F03FC013F0F2EC47
:10A338004FF00EC044F00FC045F010C046F011C0F9
:10A3480047F020EE2BF03A50D9263B50DA2244C091
:10A35800DEFF45C0DEFF46C0DEFF47C0DEFF2F0E32
:10A368003A240E6E000E3B200F6E116A106A020E20
:10A37800136E126A2FEC67F02F0E3A24426E000E0D
:10A388003B20436E496A010E486E4A6A4B6A04D004
:10A3980048504A2649504B2220EE09F03A50D92617
:10A3A8003B50DA22DE504A5CDE504B581FE242C076
:10A3B8001DF043C01EF04A5044241F6E4B504520E8
:10A3C800206E000E4620216E000E4720226E48C0E7
:10A3D80023F049C024F020EE01F03A50D9263B5032
:10A3E800DA22DF5060EC56F00009D2E020EE09F0E6
:10A3F8003A50D9263B50DA224A50DE1803E14B5036
:10A40800DE18D8A4010C000C226A236A1B6A1C6A95
:10A4180001D0152A010E216E1550D96EDA6A200E68
:10A42800DE1813E0F70E176E18681550D96EDA6A41
:10A43800DF50196E1A6A1750192618501A221A5026
:10A4480003E1050E195C01E3216A21C01DF01E6AB3
:10A458001D501E1006E0DDD71C6A010E1B6E152A62
:10A4680025D01550D96EDA6ADF50176E186A185061
:10A478001DE117502B0AF3E0060AEEE017D00A0E8A
:10A488002202F3CF17F0F4CF18F02302F350182666
:10A498001550D96EDA6ADF50175E000E185A300E62
:10A4A8001724226E000E1820236ED9D7D00E176EEF
:10A4B80018681550D96EDA6ADF50196E1A6A175083
:10A4C800192618501A221A5005E10A0E195C02E2E0
:10A4D800010E01D0000E1F6E206A1F502010CFE120
:10A4E8001B501C100DE122C017F023C018F0171ED6
:10A4F800181E174A182A17C015F018C016F01200AF
:10A5080022C015F023C016F01200818E819C000E27
:10A51800F66E980EF76E000EF86E0DEE35F011EE31
:10A528002CF00900F5CFEEFFE550E150FAE1E250DA
:10A53800F8E1520EF66EC60EF76E000EF86E03EED8
:10A54800AAF010EE4CF00900F5CFEEFFE550E1500F
:10A55800FAE1620EF66ECB0EF76E000EF86E02EEA2
:10A5680098F010EE34F00900F5CFEEFFE550E15019
:10A57800FAE1F00EF66EC80EF76E000EF86E01EEF8
:10A58800BDF010EE3DF00900F5CFEEFFE550E150CB
:10A59800FAE1D00EF66ECF0EF76E000EF86E0900D7
:10A5A800F5CF55F005EE00F018EE35F0EE6AE550FF
:10A5B800E150FCE1E250FAE104EE00F011EE00F0A7
:10A5C800EE6AE550E150FCE1E250FAE103EE00F0FA
:10A5D800AA0EEE6AE806FDE102EE00F0980EEE6AB9
:10A5E800E806FDE101EE00F06D0EEE6AE806FDE119
:10A5F80000EE4CF0090EEE6AE806FDE15690569220
:10A60800000EF86E000159EF0FF0820E9C6FFD0EE0
:10A618009D6F4EC09EF04FC09FF04AC1A0F04BC145
:10A62800A1F0ADEC67F0CE6ACD6A53501E0D070E4F
:10A63800F324D96E020EF420DA6EDECF21F0DECFDD
:10A6480022F0DECF23F0DECF24F0DECF25F0DECF00
:10A6580026F0DECF27F0DECF28F021C00FF022C091
:10A6680010F023C011F024C012F025C013F026C04A
:10A6780014F027C015F028C016F0CAEC5AF00D0ED9
:10A68800A2EC67F00A0EA2EC67F0010152514A19D8
:10A6980015E153514B1912E1889C10D0030E0AD0D2
:10A6A800050E296E4E6A4F6A2ED00A0E03D0010E8F
:10A6B80001D0020E296E27D0296A25D04EC021F07C
:10A6C8004FC022F0225009E0020A0EE00E0A10E004
:10A6D800010A12E02A0A14E0EFD72150DFE00A0A43
:10A6E800DDE01E0ADDE0E8D72150BC0AE2E0E4D74D
:10A6F80021501C0ADAE0E0D72150AC0AD8E0DCD7B8
:10A7080021500F0AD9E12950120053501E0D070E8F
:10A71800F324D96E020EF420DA6EDECFC7F0DECF56
:10A72800C8F0DECFC9F0DECFCAF0DECFCBF0DECF87
:10A73800CCF0DECFCDF0DECFCEF053501E0D1C0E88
:10A74800F324D96E020EF420DA6EDECFCFF0DDCF1F
:10A75800D0F0CF51C725D16FD051C821D26F000E8C
:10A76800C921D36F000ECA21D46F000ECB21D56F3B
:10A77800000ECC21D66F000ECD21D76F000ECE2152
:10A78800D86F53501E0D070EF324D96E020EF42015
:10A79800DA6ED1C0DEFFD2C0DEFFD3C0DEFFD4C088
:10A7A800DEFFD5C0DEFFD6C0DEFFD7C0DEFFD8C0D3
:10A7B800DEFF53501E0D070EF324D96E020EF4204F
:10A7C800DA6EDECFD9F0DECFDAF0DECFDBF0DECF27
:10A7D800DCF05350220D000EF3249E6F030EF4207C
:10A7E8009F6FD9C0A0F0DAC0A1F0DBC0A2F0DCC036
:10A7F800A3F07CEC12F0DD6FDD5103E0010E516E29
:10A80800010C516A120020EE03F04550D92646503B
:10A81800DA22DF6A20EE2BF04550D9264650DA229C
:10A82800DE68DE68DE68DD6845C03AF046C03BF0A9
:10A8380047C03CF048C03DF049C03EF04AC03FF038
:10A8480018EC5BF0000904E0466A040E456E040C3F
:10A858002D0E45240E6E020E46200F6EE5EC65F0B7
:10A86800550E0E1803E1AA0E0F1804E0466A030EEF
:10A87800456E030C20EE2FF04550D9264650DA22BB
:10A88800E90EDE1812E020EE2FF04550D92646508A
:10A89800DA22EB0EDE1809E020EE2FF04550D9261B
:10A8A8004650DA22E80EDE1827E1650E45240E6EC2
:10A8B800000E46200F6ED00E106EFF0E116E136A3A
:10A8C800030E126E80EC60F00E500F1003E1456A23
:10A8D800466A1200810E45240E6E000E46200F6E49
:10A8E800800E106EFF0E116E136A050E126E80EC4C
:10A8F80060F00E500F10EBE0466A020E456E020C37
:10A90800256A286A8380880E00019C6FFA0E9D6F65
:10A91800CECF9EF09F6BCDCFA0F0A16BADEC67F0D2
:10A9280019D0270E0E6E0F6AF0EC5DF0266E040E3D
:10A9380000019C6FFF0E9D6F252A25C09EF09F6B1E
:10A9480026C0A0F0A16BADEC67F027AA03D026C003
:10A9580028F005D0CBEC65F021502210E2E1030E7F
:10A9680000019C6FFD0E9D6F28C09EF09F6BADECA3
:10A9780067F0020E28183CE15350130DAE0EF32475
:10A98800D96E030EF420DA6E020EDF6E5350130DEB
:10A99800BA0EF324D96E030EF420DA6E080EDF6EB9
:10A9A80053500D0D9A0EF324D96E020EF420DA6E70
:10A9B8004C0EDF6E53500D0D9D0EF324D96E020E12
:10A9C800F420DA6E080EDF6E53500D0DA20EF3243C
:10A9D800D96E020EF420DA6E050EDF6E53500D0D9F
:10A9E800A30EF324D96E020EF420DA6E690EDF6E20
:10A9F800516A839012002F6E580E00019C6FFC0E56
:10AA08009D6F2FC09EF09F6B2BC0A0F02CC0A1F0B3
:10AA1800ADEC67F05DD07BEC5AF021C030F022C07D
:10AA280031F023C032F024C033F02BC0D9FF2CC042
:10AA3800DAFFDF6A20EE01F02B50D9262C50DA22FB
:10AA480033C0DFFF20EE02F02B50D9262C50DA223B
:10AA5800DF6A20EE03F02B50D9262C50DA2232C0C0
:10AA6800DFFF20EE04F02B50D9262C50DA22DF6AC3
:10AA780020EE05F02B50D9262C50DA2231C0DFFF0A
:10AA880020EE06F02B50D9262C50DA22DF6A20EE71
:10AA980007F02B50D9262C50DA2230C0DFFF1200E5
:10AAA8007BEC5AF021C030F022C031F023C032F0E4
:10AAB80024C033F02BC01BF02CC01CF030C01DF09C
:10AAC80031C01EF032C01FF033C020F0BBEF4DF094
:10AAD8002F502D6E2E6A2E50D8A412002D50010A28
:10AAE8009AE0030ADDE012000001FC6B8380838E8C
:10AAF8006AD076EC5EF025C0FAF026C0FBF0040EB2
:10AB08000001FB5D03E3010EFC6F03D0FFC0FDF005
:10AB1800FE6B8FB414D05350220D000EF3249E6F99
:10AB2800030EF4209F6F000EA06F040EA16F010E9C
:10AB3800A36FA26BFD0EA46F1AEC0CF0FF6FFF5110
:10AB480009E0130E9C6FFD0E9D6FFFC09EF09F6B7A
:10AB5800ADEC67F00101625133E0385139113A1117
:10AB68003B112EE053500C0D040EF324D96E010E48
:10AB7800F420DA6E38C172F139C173F13AC174F157
:10AB8800716B000E7125756F010E7221766F000EC4
:10AB98007321776F000E7421786FDE50751910E1FC
:10ABA800DE5076190DE1DE5077190AE1DE5078198A
:10ABB80007E1000E256E040E266E62511FEC5DF053
:10ABC8004AEC2EF05B6B0001FC5193E0839E83906E
:10ABD80012000F015969116B196B216B8C948C92BF
:10ABE8008C90889A110E136E3C0E126ECB0EE82EC6
:10ABF800FED7122EFCD7132EFAD700F0110E136EC3
:10AC08003C0E126ECB0EE82EFED7122EFCD7132E5A
:10AC1800FAD700F0020E136EA00E126E920EE82EF6
:10AC2800FED7122EFCD7132EFAD700D0000E0E6EC8
:10AC3800300E01EC63F02A0E126E8E0EE82EFED74F
:10AC4800122EFCD7000E0E6E300E01EC63F0000ED3
:10AC58000E6E300E01EC63F0000E0E6E390E01EC34
:10AC680063F0000E0E6E140E01EC63F0000E0E6E13
:10AC7800560E01EC63F0000E0E6E6D0E01EC63F0E3
:10AC8800000E0E6E700E01EC63F0000E0E6E0C0ED0
:10AC980001EC63F0000E0E6E060E01EC63F0000E80
:10ACA8000E6E010E01EC63F0D00E126ECA0EE82E85
:10ACB800FED7122EFCD71200266E2650D8A4040CFC
:10ACC8002350241001E1040C55B0030C55B4020CB8
:10ACD80054B608D0090ED8901F36203621362236B1
:10ACE800E82EF9D7230424101AE11FC017F020C05A
:10ACF80018F021C019F022C01AF0180E44EC65F0C3
:10AD0800000945E11DC010F01EC011F0FE0E126EC4
:10AD18000AEC62F000093BE0236A246A38D054C088
:10AD280025F0060E251609E023C017F024C018F0F8
:10AD3800196A1A6A970E44EC65F01FC017F020C014
:10AD480018F021C019F022C01AF0190E44EC65F071
:10AD580000091DE11DC010F01EC011F0FC0E126E9E
:10AD68000AEC62F0000908E0020E1E262306D8A0AD
:10AD7800240623502410EEE1106A116AFD0E126EAB
:10AD88000AEC62F0000903E1246A010E236ED6EC96
:10AD980067F023502410D8A4010C000CB8C0D9FFC8
:10ADA800B9C0DAFFDECFBFF0DDCFC0F0B8C074F0B5
:10ADB800B9C075F0000E766F776F786F796F5BECBE
:10ADC80038F0C36FC35153E1C16BC26BBFC03AF0D7
:10ADD800C0C03BF020EE16F0B851D926B951DA229E
:10ADE800DECF3CF0DECF3DF0DECF3EF0DECF3FF0F1
:10ADF80018EC5BF00001C36FC35139E120EE1AF083
:10AE0800B851D926B951DA22DECFBCF0DDCFBDF07A
:10AE1800BCC0D9FFBDC0DAFFE50EDE1810E020EE99
:10AE28001AF0B851D926B951DA22DECFBCF0DDCFFD
:10AE3800BDF0BCC0D9FFBDC0DAFFDF5009E1C14B8E
:10AE4800C22BBA51C11906E1BB51C21910E002D098
:10AE5800C16BC26BB8C09EF0B9C09FF0A16B010E68
:10AE6800A06FBFEC33F00001C36FC351AFE0040E15
:10AE7800C31902E1070EC36FC3511200838E83808A
:10AE88000001D16BD26BD36BD46B5350220D000EE3
:10AE9800F324746F030EF420756F350E766F0B0E66
:10AEA800776F010E796F786BD50E7A6F7B6B32EC0A
:10AEB8001DF0D06F0101625135E0385139113A1156
:10AEC8003B1130E053500C0D040EF324D96E010EE3
:10AED800F420DA6E38C1C7F039C1C8F03AC1C9F0F8
:10AEE8000001C66B000EC625CA6F010EC721CB6FC5
:10AEF800000EC821CC6F000EC921CD6FDE50CA19D3
:10AF080011E1DE50CB190EE1DE50CC190BE1DE5019
:10AF1800CD1908E1350E2B6E0B0E2C6E0101625116
:10AF2800FFEC54F002920001D55166EC5BF0000191
:10AF3800CE6FCF6BCE51D127CF51D223000ED32362
:10AF4800D42301015B6B839E839012001E6A1F6AE3
:10AF5800206A216A226A236A246A256A1650171011
:10AF6800181019101A101B101C101D1045E0010EA6
:10AF7800266E0AD0D89016361736183619361A366D
:10AF88001B361C361D36262A1DAEF4D7D8901E3621
:10AF98001F362036213622362336243625361650DB
:10AFA8000E5C17500F5818501058195011581A5055
:10AFB80012581B5013581C5014581D50155811E3A3
:10AFC80016500E5E17500F5A1850105A1950115A31
:10AFD8001A50125A1B50135A1C50145A1D50155A05
:10AFE8001E80D8901D321C321B321A321932183288
:10AFF80017321632262ECAD71EC00EF01FC00FF009
:10B0080020C010F021C011F022C012F023C013F0AC
:10B0180024C014F025C015F01200C4C0D9FFC5C063
:10B02800DAFFDECFC6F0DDCFC7F0C4C0B8F0C5C0C8
:10B03800B9F0000EBB6F010EBA6FD2EC56F0C86FB4
:10B04800C85147E1C6C03AF0C7C03BF020EE16F041
:10B05800C451D926C551DA22DECF3CF0DECF3DF00F
:10B06800DECF3EF0DECF3FF018EC5BF00001C86F9A
:10B07800C8512FE120EE1AF0C451D926C551DA2261
:10B08800DECF0EF0DDCF0FF0116A106A136A200EC2
:10B09800126E2FEC67F0000120EE1AF0C451D92689
:10B0A800C551DA22DECF0EF0DDCF0FF01C0EC4251D
:10B0B800106E000EC521116E136A0B0E126ED8ECBD
:10B0C80063F020EE03F0C651D926C751DA22010EEB
:10B0D800DF6EC851120001015C6B506A486B496B06
:10B0E800020E5B6F83905A6B596B536A030E53645D
:10B0F80001D049D053500C0D030EF324D96E010E24
:10B10800F420DA6EDF6A53500C0D020EF324D96E68
:10B11800010EF420DA6EDF6A53500C0D000EF32492
:10B12800D96E010EF420DA6EDE6ADD6A53500C0D1A
:10B13800040EF324D96E010EF420DA6EDE6ADE6A9C
:10B14800DE6ADD6A53500C0D0B0EF324D96E010E26
:10B15800F420DA6E100EDF6E53500C0D0A0EF32435
:10B16800D96E010EF420DA6E020EDF6E53500C0D0C
:10B17800080EF324D96E010EF420DA6E240EDE6E6A
:10B18800DD6A532AB3D7536A0101586B12008380D2
:10B19800838E000E0E6E040E0F6E116A1068010E7B
:10B1A800136E126A96EC4CF0FA0E00019C6FFD0EBD
:10B1B8009D6FADEC67F0CB6BCC6BCBC04BF0010E49
:10B1C8004B164B324B3283504B187F0B4B18836E08
:10B1D8002E0EA2EC67F08FB415D05350220D000E3E
:10B1E800F32400019E6F030EF4209F6F000EA06FE2
:10B1F800040EA16F010EA36FA26BC80EA46F1AEC08
:10B208000CF0CA6F0001CA5109E0640E9C6FFF0E72
:10B218009D6FCAC09EF09F6BADEF67F0CB4BCC2BF8
:10B22800CCBFCBD7CC5103E10A0ECB5DC6E3E60E0B
:10B238009C6FFE0E9D6FADEC67F0839E83908390AC
:10B24800516A120002500209026E040E536033D094
:10B25800350E0E6E0B0E0F6E5350050DD10EF324E6
:10B26800106E010EF420116E136A050E126E96EC24
:10B2780063F03A0E0E6E0B0E0F6E5350130DAA0E9E
:10B28800F324106E030EF420116E136A130E126E5F
:10B2980096EC63F04D0E0E6E0B0E0F6E53500D0DA7
:10B2A800980EF324106E020EF420116E136A0D0E20
:10B2B800126E96EC63F0030E536409D0010E516EC2
:10B2C80002011B5110091B6F000EE8CF36FB250E3B
:10B2D80066EC5BF0350E216E0B0E226E000E246EAE
:10B2E800250E236E200E256EFF0E266E80EC61F073
:10B2F800029283901200090E186E0F5010103BE056
:10B308000FC0D9FF10C0DAFFDE50DE1034E00FC0E6
:10B31800D9FF10C0DAFFDECF12F0DDCF13F012C074
:10B32800D9FF13C0DAFFDF5026E00FC0D9FF10C0E5
:10B33800DAFF10EE05F0DE50E126DD50E22220EEC5
:10B3480002F00F50D9261050DA22E650DE1813E129
:10B35800E650DE1810E10FC0D9FF10C0DAFF10EE7A
:10B3680001F0DE50E126DD50E222E750D0EC67F034
:10B37800126E12A0186A185003E0166A176A08D0ED
:10B388000FC0D9FF10C0DAFFDECF16F0DDCF17F0FF
:10B398001150D96EDA6A16C0DEFF17C0DDFF1850EB
:10B3A800120020EE03F00E50D9260F50DA22DF509B
:10B3B800166E176A186A196A20EE02F00E50D9261E
:10B3C8000F50DA22DF5016C013F017C014F018C05F
:10B3D80015F0126A1210166E1350176E1450186E6C
:10B3E8001550196E20EE01F00E50D9260F50DA22B2
:10B3F800DF5016C013F017C014F018C015F0126A09
:10B408001210166E1350176E1450186E1550196ED0
:10B418000EC0D9FF0FC0DAFFDF5016C013F017C0F7
:10B4280014F018C015F0126A1210166E1350176E29
:10B438001450186E1550196E16C00EF017C00FF084
:10B4480018C010F019C011F01200256E2550D8A4AC
:10B45800040C2350241001E1040C55B0030C54B61D
:10B4680008D0090ED8901F36203621362236E82E0D
:10B47800F9D7245006E1020E235C03E2276A110E75
:10B4880002D0276A120E266E26C028F01FC017F0B9
:10B4980020C018F021C019F022C01AF0285044EC3E
:10B4A80065F000091DE11DC00EF01EC00FF0020E70
:10B4B800116E106AB0EC61F0000908E0020E1E2659
:10B4C8002306D8A0240623502410EDE1120E2818D4
:10B4D80007E1176A186A196A1A6A0C0E44EC65F0D3
:10B4E800D6EC67F023502410D8A4010C000C60ECB3
:10B4F80065F0CC0E72EC67F0660E72EC67F055ECF6
:10B5080067F0276E275005E1216A226A236A246AB8
:10B518001200256A266A2550270FD96EDA6A55EC7B
:10B5280067F0DF6E254A262A26BEF5D7265003E1A6
:10B53800040E255CF0E3F50E00019C6FFB0E9D6F79
:10B5480027C09EF09F6B28C0A0F0A16B29C0A2F075
:10B55800A36B2AC0A4F0A56B27C0A6F028C0A7F04B
:10B5680029C0A8F02AC0A9F0ADEC67F02A5029102C
:10B57800281003E1060E275CC7E327C021F028C086
:10B5880022F029C023F02AC024F01200196A0F0EF5
:10B59800186E070E1826176A1850D96EDA6ADF5027
:10B5A8001A6E1A3A0F0E1A161A161A500CE0BD0E19
:10B5B8001A24D96EDA6A010EDA22DF50A2EC67F09B
:10B5C800010E196E0BD0190409E1BD0E1A24D96EAB
:10B5D800DA6A010EDA22DF50A2EC67F01850D96E51
:10B5E800DA6ADF501A6E0F0E1A161A500CE0BD0EEA
:10B5F8001A24D96EDA6A010EDA22DF50A2EC67F05B
:10B60800010E196E0BD0190409E1BD0E1A24D96E6A
:10B61800DA6A010EDA22DF50A2EC67F01806172A60
:10B62800070E1764B9D7070C446A20EE2BF03A507E
:10B63800D9263B50DA223C50DE1809E13D50DE188D
:10B6480006E13E50DE1803E13F50DE1839E03AC00B
:10B6580027F03BC028F02BEC48F0446E445030E112
:10B668002F0E3A241D6E000E3B201E6E3CC01FF0AC
:10B678003DC020F03EC021F03FC022F0246A010EF8
:10B68800236E20EE01F03A50D9263B50DA22DF50E3
:10B6980029EC5AF0000906E03C683D683E683F68BE
:10B6A800010E446E20EE2BF03A50D9263B50DA2298
:10B6B8003CC0DEFF3DC0DEFF3EC0DEFF3FC0DEFF18
:10B6C80044501200016E838C839C0BEE35F08490FD
:10B6D800849A1390F29E83A4FED78968838C839CF6
:10B6E8008EA821D0010428E0EE50866E861E8B6A53
:10B6F8008EA819D08EA2FCD78EA2FAD7838C839CF1
:10B70800838C839C89908EA80ED08EB2FCD78EA491
:10B71800FED78980898A8EA806D08EB4FCD78EA8D9
:10B7280002D0012EDDD78B68F90E896E129012981F
:10B738001380F28E015012008EA2FED702B2899AAF
:10B74800EE50866E861E8B6AD9D7838C0000839C48
:10B75800EAD70000032EFDD7000C03D00E4A0F2AAB
:10B76800102A1050D96EDA6ADF50116E0EC0F6FF3B
:10B778000FC0F7FF000EF86E0E0EF76403D0080036
:10B78800F55005D0F6CFE9FFF7CFEAFFEF501118D3
:10B7980013E10EC0F6FF0FC0F7FF000EF86E0E0E95
:10B7A800F76403D00800F55005D0F6CFE9FFF7CFCE
:10B7B800EAFFEF500009D2E10EC0F6FF0FC0F7FF15
:10B7C800000EF86E0E0EF76403D00800F55005D091
:10B7D800F6CFE9FFF7CFEAFFEF50116E1050D96EA0
:10B7E800DA6ADF50115C0E6E0F6AD8A00F061200DD
:10B7F800175018100AE140C117F041C118F017504E
:10B80800181003E1176A186A120017C012F018C05E
:10B8180013F019C014F0F9EC63F012501726135006
:10B82800182217C0D9FF18C0DAFFDF5006E101015E
:10B83800406B416B176A186A120017C012F018C0E3
:10B8480013F019C014F019EC64F012501724010118
:10B85800406F13501820416F40C1D9FF41C1DAFF32
:10B86800DF5009E040C1D9FF41C1DAFF000EDF6AAD
:10B87800404B412B02D0406B416B17C017F018C0EA
:10B8880018F01200A96BAA6B9FC0ABF0A0C0ACF077
:10B89800A107D8A0A20727D0A3C074F0A4C075F050
:10B8A800A50E766F776B796B010E786FB10E7A6F94
:10B8B8007B6B32EC1DF0B105B2111EE1A551AD6FE5
:10B8C800AE6BAF6BB06BABC0D9FFACC0DAFFADC02D
:10B8D800DFFFAB4BAC2BA94BAA2B0A0EAD19AE114F
:10B8E800AF11B01109E0A151A95DAA51800A4B6EB0
:10B8F800A251800A4B58D0E3ABC0D9FFACC0DAFFE5
:10B90800DF6AA951AA1103E19F6BA06B12009FC0C7
:10B918009FF0A0C0A0F01200B3C0B7F0B4C0B8F058
:10B92800B70E0E6ECCEC4AF00EC0BBF00FC0BCF0E8
:10B938000001BCBF0B0CD890BB35D96EBC35DA6E94
:10B948004E0ED926010EDA22DECFB9F0DDCFBAF0DD
:10B95800B951BA1105E0B9C0D9FFBAC0DAFFDF6A38
:10B96800B151B21105E0B1C0D9FFB2C0DAFFDF6A48
:10B97800D890BB35D96EBC35DA6E4E0ED926010E7D
:10B98800DA22B1C0DEFFB2C0DDFFB55101E1000C23
:10B99800B30E7C6FB10E7D6F7E6B7F6BADEC00F0EC
:10B9A8000001B66FB65112000EC015F00FC016F0A8
:10B9B80010C017F011C018F01206D8A013061228EC
:10B9C8000CE113280AE10E6A0F6A1200154A162ABA
:10B9D800174A182A1206D8A0130615C0F6FF16C073
:10B9E800F7FF0800F55015E017C0D9FF18C0DAFFB7
:10B9F800DF500FE0125013100CE017C0D9FF18C029
:10BA0800DAFF15C0F6FF16C0F7FFDE500900F5187B
:10BA1800DDE015C0F6FF16C0F7FF0800F5CF14F0FB
:10BA280017C0D9FF18C0DAFFDF50145C0E6E0F6A1A
:10BA3800D8A00F061200296E39D020EE01F025504B
:10BA4800D9262650DA22DF502D6E20EE03F025503D
:10BA5800D9262650DA22DF502C6E20EE05F025502C
:10BA6800D9262650DA22DF502B6E20EE07F025501B
:10BA7800D9262650DA22DF502A6E2AC011F02BC0B0
:10BA880012F02CC013F02DC014F05EEF62F025C048
:10BA98000EF026C00FF031EC43F00EC02AF00FC0B4
:10BAA8002BF010C02CF011C02DF0E7D72950276ECD
:10BAB800286A2850D8A412002750010ABEE0030AB9
:10BAC800E6E012001E6A1F6A206A216A226A236A57
:10BAD800246A256A0EA010D016501E2617501F2261
:10BAE80018502022195021221A5022221B5023229A
:10BAF8001C5024221D502522D89016361736183689
:10BB080019361A361B361C361D36D89015321432A3
:10BB180013321232113210320F320E320E500F1011
:10BB2800101011101210131014101510D3E11EC0AC
:10BB38000EF01FC00FF020C010F021C011F022C07D
:10BB480012F023C013F024C014F025C015F0120021
:10BB5800115002E0115003E10F5097EF67F01150B8
:10BB6800D96EDA6A040ED926DE50DE1014E01150C0
:10BB7800D96EDA6A040ED9261150E16EE26A020E15
:10BB8800E126DE50E65CE650800A166EDE50800A3A
:10BB98001658D8B012001150D96EDA6A020ED9269A
:10BBA800DECF12F0DDCF13F01150D96EDA6ADECF96
:10BBB80014F0DDCF15F012501424D96E135015204F
:10BBC800DA6E0FC0DFFF1150D96EDA6A020ED9267D
:10BBD800DE2A000EDD22000C25EE04F0DE50DE1019
:10BBE800FBE000C516F001C517F0060E1624D96E45
:10BBF800050E1720DA6EDF50146E060E1624D96E65
:10BC0800070E1720DA6EDF50156E164A172A1068CD
:10BC1800010E116E16C012F017C013F01050121654
:10BC28001150131612C000F513C001F5F29E25EE4F
:10BC380004F0DE06000EDD5AF28E0EC0D9FF0FC0EA
:10BC4800DAFF15C0DFFF25EE04F0010EDBBE04D0DD
:10BC5800DB5003E1DE0401E28982145012000E5029
:10BC68001202F3CF16F0F4CF17F0186A196A0E50C3
:10BC78001302F3501726F4501822000E19220F5001
:10BC88001202F3501726F4501822000E19220E50F3
:10BC98001402F3501826F45019220F501302F350CF
:10BCA8001826F450192210501202F3501826F45096
:10BCB800192215500E02F35019260F501402F35092
:10BCC800192610501302F350192611501202F3507E
:10BCD800192616C00EF017C00FF018C010F019C0C2
:10BCE80011F01200286A296A01016C6B2A6A30D0A7
:10BCF800CBEC65F02150221020E02A0E0E6E0F6A60
:10BD0800F0EC5DF0276E2AA80CD0BB0E00019C6FEA
:10BD1800FE0E9D6F27C09EF09F6BADEC67F0839081
:10BD28000CD0000E01016C25D96EDA6A040EDA22F5
:10BD380027C0DFFF6C2B284A292A2AAA07D0000E21
:10BD48002824256E040E2920266E12008EAC02D0FF
:10BD58002904CEE328C025F029C026F01200150ECC
:10BD6800146EC60EE82EFED7142EFCD700D020D0B5
:10BD7800150E146EC60EE82EFED7142EFCD700D072
:10BD8800010E0E6E12C0F6FF13C0F7FF000EF86E1C
:10BD98000E0EF76403D00800F55005D0F6CFE9FF82
:10BDA800F7CFEAFFEF5001EC63F0124A132AD7D716
:10BDB80012C0F6FF13C0F7FF000EF86E0E0EF76400
:10BDC80003D00800F55005D0F6CFE9FFF7CFEAFF1A
:10BDD800EF500009CDE11200166A176A186A196A4D
:10BDE800125013101410151029E0010E1A6E06D007
:10BDF800D89012361336143615361A2A15AEF8D7D7
:10BE0800D890163617361836193612500E5C13505D
:10BE18000F58145010581550115809E312500E5E5F
:10BE280013500F5A1450105A1550115A1680D890A2
:10BE380015321432133212321A2EE2D716C00EF00F
:10BE480017C00FF018C010F019C011F01200866A60
:10BE5800846A8B68896801016C6B83928394566B42
:10BE6800576B0AD0000E5625D96E040E5721DA6E8C
:10BE7800000EDF6E564B572B57BFF4D7575102E1D0
:10BE88005605F0E3566B576B09D0350E5625D96E1B
:10BE98000B0E5721DA6EDF6A564B572B57BFF5D773
:10BEA8005705F3E30F011769D6501F0B4009D66EEB
:10BEB800D6980F0ED612D588D5120E01C29BD58EF4
:10BEC8000F0C1A0E17240E6E000E18200F6EE5ECDC
:10BED80065F00EC01DF00FC01EF01F6A206A15C065
:10BEE800D9FF16C0DAFF030EDE181CE1140E172462
:10BEF8000E6E000E18200F6EE5EC65F00E50196EF0
:10BF08000F501A6E1B6A1C6A1AC01CF019C01BF06D
:10BF18001A6A196A19501D121A501E121B501F1244
:10BF28001C5020121DC015F01EC016F01FC017F0BF
:10BF380020C018F01200166E0C0E161807E0D6EC8A
:10BF480067F07FEC67F0000901E1FF0C165040092B
:10BF5800C0EC67F01350C0EC67F01250C0EC67F00B
:10BF68001150C0EC67F01050C0EC67F0010E156E70
:10BF7800165002E1950E156E080E161802E1870E8E
:10BF8800156E1550C0EC67F00C0E161802E1C9ECDE
:10BF980067F00A0E156EC9EC67F0146E14AE02D085
:10BFA800152EF9D714501200838002500209026E30
:10BFB80058050DE1000EE8CF35FB500EE8CF36FBF3
:10BFC800000EE8CF37FBE8CF38FB586B1DD02BEEBF
:10BFD80035F059C1DFFF000EE8CF36FB0D0EE8CF74
:10BFE80037FB000EE8CF38FB8FA403D0600EE8CFF4
:10BFF80038FB8FA406D037CB0EF0200E0E120EC0E1
:10C0080037FB010EE8CF39FB050E66EC5BF00292B8
:10C018000101596B8390120012501310D8B4000C10
:10C0280012C0D9FF13C0DAFFDF5001E1000C12C0C3
:10C038000EF013C00FF0B7EC63F00EC014F00FC091
:10C0480015F0020E1418151001E0000C160E0E6EF5
:10C0580012C0D9FF13C0DAFFDF5087EC62F0000985
:10C06800D8B4000C170E0E6E20EE01F01250D9262F
:10C078001350DA22DF5087EC62F0000901E1000C6E
:10C088001638F00B17101200106EAD0EF66EF80E83
:10C09800F76E0900F550105C2CE3AE0EF66EF80E44
:10C0A800F76E10500900F55C04E30F6A010E0E6E7E
:10C0B800010CAF0EF66EF80EF76E0900F550105C25
:10C0C80008E3B00EF66EF80EF76E10500900F55C36
:10C0D800ECE2B10EF66EF80EF76E0900F550105C42
:10C0E80008E3B20EF66EF80EF76E10500900F55C14
:10C0F800DCE20E6A0F6A12000EC015F00FC016F0CF
:10C1080010C017F011C018F015C0D9FF16C0DAFF1B
:10C11800DF50146E17C0F6FF18C0F7FF000EF86E58
:10C128000E0EF76403D00800F55005D0F6CFE9FFEE
:10C13800F7CFEAFFEF50145C196E1A6AD8A01A06F6
:10C14800174A182A154A162A1206D8A0130612509A
:10C15800131003E019501A10D7E019C00EF01AC0D6
:10C168000FF012000EC0D9FF0FC0DAFF10C0DFFFBA
:10C178000E4A0F2A1150106E1250116E1350126E83
:10C18800136A0EC0D9FF0FC0DAFF10C0DFFF0E4AD6
:10C198000F2A1150106E1250116E1350126E136A3E
:10C1A8000EC0D9FF0FC0DAFF10C0DFFF0E4A0F2AFA
:10C1B8001150106E1250116E1350126E136A0EC089
:10C1C800D9FF0FC0DAFF10C0DFFF0E4A0F2A120096
:10C1D800536A030E536401D02AD053500C0D030E3A
:10C1E800F324D96E010EF420DA6EDF6A53500C0D79
:10C1F800020EF324D96E010EF420DA6EDF6A535072
:10C208000C0D000EF324D96E010EF420DA6EDE6AEE
:10C21800DD6A53500C0D040EF324D96E010EF42080
:10C22800DA6EDE6ADE6ADE6ADD6A532AD2D7536ABC
:10C2380083905B6B1200125013101410151023E03A
:10C24800010E166E06D0D8901236133614361536EF
:10C25800162A15AEF8D712500E5C13500F5814500A
:10C2680010581550115808E312500E5E13500F5A0B
:10C278001450105A1550115AD890153214321332DE
:10C288001232162EE8D70EC00EF00FC00FF010C0F5
:10C2980010F011C011F01200536A0E6A0F6A535061
:10C2A8001E0D070EF324D96E020EF420DA6E070E67
:10C2B800DE6AE806FDE253501E0D1B0EF324D96E0C
:10C2C800020EF420DA6EDF6A53501E0D170EF324A7
:10C2D800D96E020EF420DA6EDE6ADE6ADE6ADD6A84
:10C2E8000E4A0F2A0FBEDBD70F5003E1040E0E5C77
:10C2F800D6E38390516A1200245003E1810E235C37
:10C3080004E3000E246E800E236E980E00019C6FCD
:10C31800FF0E9D6F25C09EF026C09FF0ADEC67F024
:10C32800286A296A13D028502124D96E295022203E
:10C33800DA6EDF50276E090E9C6FFF0E9D6F27C0C7
:10C348009EF09F6BADEC67F0284A292A2350285CA1
:10C3580024502958E8E31200070E136ED00E126E0F
:10C368000FD0C9EC67F0146E14280DE1E40E00D06C
:10C3780000D0E82EFCD700D000D01206D8A01306B3
:10C3880012501310EEE1FE0E141801E0000CC9EC77
:10C3980067F00EC0D9FF0FC0DAFFDF6E0E4A0F2A12
:10C3A8001006D8A0110610501110F1E1C9EC67F081
:10C3B800C9EC67F0010C0EC014F00FC015F013D0D3
:10C3C8001206D8A0130610C0D9FF11C0DAFF104A10
:10C3D800112A14C0E1FF15C0E2FF144A152ADFCF65
:10C3E800E7FFE7500BE01250131008E0E9D714C03C
:10C3F800D9FF15C0DAFFDF6A144A152A1206D8A039
:10C4080013061228F4E11328F2E112007BEC65F020
:10C41800000901E1000C1250C0EC67F0FD0E121883
:10C428001EE0020E146E136A10C0D9FF11C0DAFFA5
:10C43800DF50C0EC67F0104A112A1306D8A0140682
:10C4480013501410F1E1C9EC67F0C9EC67F0C9ECBE
:10C4580067F0156E15501F0B050A01E0000C010C62
:10C4680015D00FC0F6FF10C0F7FF000EF86E0E0EC5
:10C47800F76403D00800F55005D0F6CFE9FFF7CFF1
:10C48800EAFFEF50A2EC67F00F4A102A0FC0F6FF40
:10C4980010C0F7FF000EF86E0E0EF76403D0080008
:10C4A800F55005D0F6CFE9FFF7CFEAFFEF500009C6
:10C4B800D8E1120011C015F012C016F013C017F021
:10C4C80014C018F060EC65F0CC0E72EC67F0990EB1
:10C4D80072EC67F00C0E72EC67F0196A1A6A195060
:10C4E800150FD96EDA6ADF5072EC67F0194A1A2A0A
:10C4F8001ABEF5D71A5002E060EF65F0040E195C19
:10C50800EEE360EF65F00F6E0E5001E1000C2F0EA8
:10C518000F6409D03A0E0F6006D00E50D96EDA6A51
:10C528000F50D00F17D0400E0F6409D0470E0F6080
:10C5380006D00E50D96EDA6A0F50C90F0BD0600EB4
:10C548000F64000C670E0F60000C0E50D96EDA6A8B
:10C558000F50A90FDF6E010C226EB50E236EF80E78
:10C56800246E216A0AD023C0F6FF24C0F7FF234AAD
:10C57800242A0800F550F7E1212A2250211807E063
:10C5880023C0F6FF24C0F7FF0800F550ECE1080EC1
:10C5980000019C6FFE0E9D6F22C09EF09F6B23C012
:10C5A800A0F024C0A1F0ADEF67F0106EA90EF66EF2
:10C5B800F80EF76E0900F550105C1CE3AA0EF66E33
:10C5C800F80EF76E10500900F55C04E30F6A010ECF
:10C5D8000E6E010CAB0EF66EF80EF76E0900F550F4
:10C5E800105C08E3AC0EF66EF80EF76E10500900FA
:10C5F800F55CECE20E6A0F6A12000F6E87920A0E63
:10C60800E82EFED700D00EB002D0879401D08784E0
:10C61800000E116E010E106E0FAE02D0838A01D08B
:10C62800839AD8900F36879000F000F0878000F04A
:10C6380000F08790104A112A11BEEED7115003E17D
:10C64800090E105CE9E3878212000109122001003B
:10C6580001001700002D119420D00F0001010912CC
:10C6680020010001001700002D119420D00F0001B7
:10C6780001091220010001001700002D119420D09B
:10C688000F000101091220010001001700002D11FF
:10C698009420D00F0001010E0E6E0F6A88868782E3
:10C6A800878400F000F0879400F000F0106A116AA7
:10C6B8008DA602D00E500F12D8900E36879000F03B
:10C6C80000F0878000F000F08790104A112A11BE10
:10C6D800EFD7115003E1030E105CEAE30F5012008C
:10C6E8009F0E166E176814C018F015C019F0165072
:10C6F800182617501922195005E11A0E185C02E283
:10C70800010E01D0000E1A6E1B6A1A501B1005E0AC
:10C718005F0E1414146E156A120014C014F015C0BC
:10C7280015F0120010C016F011C017F00EC014F06A
:10C738000FC015F010D016C0D9FF17C0DAFFDF50B0
:10C74800186E164A172A14C0D9FF15C0DAFF18C088
:10C75800DFFF144A152A1206D8A013061228EBE1A7
:10C768001328E9E112000EC010F00FC011F002D03A
:10C778000E4A0F2A0EC0F6FF0FC0F7FF000EF86E24
:10C788000E0EF76403D00800F55005D0F6CFE9FF88
:10C79800F7CFEAFFEF500009EBE110500E5C0E6E88
:10C7A80011500F580F6E12000EC014F00FC015F084
:10C7B80010C016F011C017F012501310D8B41200A0
:10C7C80016C0D9FF17C0DAFF14C0E1FF15C0E2FF99
:10C7D800DFCFE7FF164A172A144A152A1206D8A0EF
:10C7E800130612501310ECE11200156A166A04D0F1
:10C7F800124A132A154A162A12C0D9FF13C0DAFFA3
:10C80800DF500EE014C00EF012C0D9FF13C0DAFFDB
:10C81800DF500F6E106A1CEC67F00E500F10E8E145
:10C8280015C012F016C013F01200156A166A04D06B
:10C83800124A132A154A162A12C0D9FF13C0DAFF62
:10C84800DF500EE014C00EF012C0D9FF13C0DAFF9B
:10C85800DF500F6E106A1CEC67F00E500F10E8E006
:10C8680015C012F016C013F012001A0E14240E6E22
:10C87800000E15200F6E16C010F017C011F0F5EC61
:10C8880066F012C0D9FF13C0DAFF030EDE18D8A471
:10C898001200140E14240E6E000E15200F6E18C010
:10C8A80010F019C011F0F5EF66F05B6B8380838E92
:10C8B800000E0E6E040E0F6E116AF60E106E010E4B
:10C8C800136E126A96EC4CF0FA0E00019C6FFD0E86
:10C8D8009D6FADEC67F0E60E9C6FFE0E9D6FADECA4
:10C8E80067F0839E83901200303132333435363707
:10C8F8003839414243444546350B1FE7800102E879
:10C9080005800102E805800102E805800102E805CA
:10C9180068706469736B2E636667004850393132FA
:05C92800314400000095
:10C92E000E6E0E500EE0DDEC67F0200EE82EFED7F8
:10C93E00E0EC67F0CC0E00D0E82EFDD700D000D092
:10C94E001200DDEC67F0C00E00D0E82EFDD7E0EC53
:10C95E0067F0350EE82EFED700F012006DC049F0DC
:10C96E006EC04AF0DEEC48F0716F715112E16DC08D
:10C97E000FF06EC010F06F0E116E7FEC59F00001CB
:10C98E00716F715106E16DC0D9FF6EC0DAFFDE6ABC
:10C99E00DD6A71511200800E826F7CC083F07DC003
:10C9AE0084F0856B866B876B886B830E766F7EC08B
:10C9BE0077F07FC078F0820E796F21EC05F00001E0
:10C9CE0085517C25D96E86517D21DA6EDF6A000C89
:10C9DE00000EF2BE010E116E0F50030B7F6E0EC0D5
:10C9EE007EFF10C080FF3F0E81168184F29E550E91
:10C9FE00826EAA0E826E818281B2FED7819411B0B0
:10CA0E0002D0F29E01D0F28E1200350E0E6E0B0E7B
:10CA1E000F6E116A106A010E136E126A96EC4CF0CC
:10CA2E0002500209026E2BEE35F05BC1DFFF226A67
:10CA3E00010E216E45EC3DF00292838001015B6B8D
:10CA4E00120002D00E4A0F2A0EC0F6FF0FC0F7FFDB
:10CA5E000800F55009E00EC0F6FF0FC0F7FF080002
:10CA6E00F55010181110EEE10EC0F6FF0FC0F7FFD3
:10CA7E000800F5500E6E0F6A12001B6E1BAE0ED024
:10CA8E001B9E106A116A126A136A370E9FEC5FF0D2
:10CA9E001C6E010E1C6402D01C50120017C010F048
:10CAAE0018C011F019C012F01AC013F01B509FEFEE
:10CABE005FF0DDEC67F00A0E0F6EF80EE82EFED773
:10CACE000F2EFCD700D0E0EC67F0E00E00D0E82E81
:10CADE00FDD7B7EC67F0090E0F6E840EE82EFED769
:10CAEE000F2EFCD7E0EF67F0130E0F6E880E0E6E52
:10CAFE000ED0C9EC67F0FF0A0DE0E40E00D000D0B6
:10CB0E00E82EFCD700D000D00E06D8A00F060E508F
:10CB1E000F10EFE10E500F10D8A4010C000C010EF7
:10CB2E00146E200E0E180F1011E0F70E106E116815
:10CB3E000EC012F00FC013F0105012261150132217
:10CB4E00135003E1050E125C01E3146A14C00EF0DB
:10CB5E000F6A120000004F01000F0000000009FFD5
:10CB6E000000004F01000F0000000009FF00000050
:10CB7E004F01000F0000000009FF0000004F0100F0
:10CB8E000F0000000009FF00898225EE04F0010E5F
:10CB9E00DBBE0FD0DE28010EDE580BE35C0E00016B
:10CBAE009C6FFF0E9D6F04C59EF005C59FF0ADEC0A
:10CBBE0067F004C521F005C522F0120020EE01F049
:10CBCE000E50D9260F50DA22DF50136E146A0EC0A3
:10CBDE00D9FF0FC0DAFFDF50106E1350116E1050D8
:10CBEE00136E11C014F013C00EF014C00FF012002B
:10CBFE0060900F0E0F01596F070E396F356F4F0E84
:10CC0E00936E8A6A8A888A828A82010E8F6E130ECA
:10CC1E000E01B76F0F0EFA6F100EFC6F140EB86F79
:10CC2E00140C9F0E106E1168200E0E10126E000E58
:10CC3E000F10136E1050122611501322135005E1CF
:10CC4E001A0E125C02E2010E01D0000E0E6E0F6A79
:10CC5E00120021BE04D021500FE120040DE220C0AD
:10CC6E0022F021C023F0221E231E224A232A22C094
:10CC7E0020F023C021F0120020C020F021C021F0AE
:10CC8E0012001B6A1C6A09D01AC00FF0106A19C074
:10CC9E0011F0ACEC5DF01B4A1C2A1B501724D96E08
:10CCAE001C501820DA6EDF501A6E1A50EDE1120089
:10CCBE00350E0E6E0B0E0F6E116A106A010E136E8C
:10CCCE00126A96EC4CF0010EE8CF35FB02500209C9
:10CCDE00026E010E66EC5BF0029212009F0E106E59
:10CCEE0011680EC012F00FC013F010501226115022
:10CCFE001322135005E11A0E125C02E2010E01D04E
:10CD0E00000E0E6E0F6A1200BF0E106E11680EC06E
:10CD1E0012F00FC013F010501226115013221350A0
:10CD2E0005E11A0E125C02E2010E01D0000E0E6E2B
:10CD3E000F6A1200D00E106E11680EC012F00FC0E6
:10CD4E0013F01050122611501322135005E10A0E43
:10CD5E00125C02E2010E01D0000E0E6E0F6A12007E
:10CD6E009F869E84090E0E01FD6F9F98890E9B6E05
:10CD7E009C6A9E989D8E9D889D9AC599F28AF28E88
:10CD8E009E909D9C9E9A9E8A1200136A110E126EA0
:10CD9E0009D00A0EE82EFED700D0010E0E6E200E20
:10CDAE0001EC63F01206D8A013061228F2E1132844
:10CDBE00F0E112000E6E0E5009E0966A4F0E936E61
:10CDCE00220E966E400E956E968A400C966A100E46
:10CDDE00966E2A0E966E900E936EF4D70EC0D9FFF5
:10CDEE000FC0DAFF10C0DFFF0E4A0F2A11C010F07D
:10CDFE00116A0EC0D9FF0FC0DAFF10C0DFFF0E4A56
:10CE0E000F2A1200DDEC67F0200EE82EFED7E0ECC4
:10CE1E0067F0300EE82EFED7B7EC67F00F6EB00E4F
:10CE2E0000D0E82EFDD70F5012000E50D96EDA6AE0
:10CE3E000F50DE1804E10EC00EF00F6A12000E2A1B
:10CE4E000E04D96EDA6ADF50F0E10E6A0F6A120034
:10CE5E000EC014F00FC015F014C0D9FF15C0DAFFC4
:10CE6E0010C0DFFF144A152A1206D8A0130612505E
:10CE7E001310F2E11200070E8C6E9150070B0E6E1E
:10CE8E00888A8DAA02D0080E0E26020E01016419A0
:10CE9E0003E10E1C0F0B0E6E0E501200106A116A7B
:10CEAE00D890103209EC67F0000901E0108E112ABB
:10CEBE00070E1164F5D710501200000EE8CF00F5E2
:10CECE00E8CF01F5E8CF02F5E8CF03F5E8CF04F59A
:10CEDE00E8CF05F5000C0F6E106A0F50010B97ECA2
:10CEEE0064F0D8900F32102A070E1064F6D7070C94
:10CEFE00E5EC67F0C9EC67F07BEC65F0000901E04A
:10CF0E00010CD6EC67F0000C0F50030B7F6E0EC0B9
:10CF1E007EFF3F0E8116818000F000F080501200DF
:10CF2E000E6E03D0E7EC67F004000E01CDA9FAD720
:10CF3E000EC09AFF12000E6E03D0E7EC67F00400ED
:10CF4E000E01CDA9FAD70EC09AFF12009E0E206ECA
:10CF5E009CC01BF09DC01CF0200E1D6E2BEF26F00A
:10CF6E0088888DA803D0010E0E6E01D00E6A0E5069
:10CF7E0012000E6E0EC092FF0E01CDA1FDD7CD9107
:10CF8E009250120092680E01CDA1FDD7CD91925014
:10CF9E0012000E6E0E5001E0010C55501200E3EC23
:10CFAE0067F0C9EF67F083905B6B120083988898E7
:10CFBE0012008398888812008580120085901200D6
:03CFCE001200014D
:10F8A80000819FE0FC407E80FC000020004F4B0060
:10F8B8004449534B5F455252004E4F545F524541A5
:10F8C8004459004E4F5F46494C45004E4F545F4FD8
:10F8D80050454E4544004E4F545F454E41424C45BD
:10F8E80044004E4F5F46494C455F53595354454D6C
:10F8F80000000D0A20253258202532582025327361
:10F908002025327320253273202532732025327347
:10F918002025327320253273202532732025347335
:10F92800202534732025347320253473202534731F
:10F9380020253473202534732025347320000D0AC4
:10F9480048504469736B204D6B2049492028313851
:10F958004634364B343029202573202573202573EF
:10F96800205374617274696E672E2E2E0D0A000D75
:10F978000A4461746120706F72742069732025587D
:10F98800202D2053686F756C64206265203C3E20F2
:10F9980030784646000D0A5365656B206572722003
:10F9A8002564203E2025642C202564203E202564E3
:10F9B8002C202564203E202564000D0A53746174B0
:10F9C800757320706F7274206973202558202D205C
:10F9D80053686F756C642062652030784646000D68
:10F9E8000A4461746120706F72742069732025580D
:10F9F800202D2053686F756C64206265203078462E
:10FA080046000D0A526420752025642072746E2009
:10FA180025642C20256420627974657320726561E1
:10FA2800640D0A000D0A4D617820566563746F7283
:10FA3800206469736B20256420256C642028256C5C
:10FA4800582920000D0A44736B73656C2069732074
:10FA580025642C206E756D6265722069732025649B
:10FA680020000D0A426C6F636B73697A6520666FBC
:10FA780072206469736B20256420697320256400F3
:10FA88000D0A2530325825303258205353383078F3
:10FA98003A466D74206F70747300466F756E6420FB
:10FAA800616E205254432066696C6520617420257C
:10FAB800580D0A004C6F6F6B696E6720666F722075
:10FAC800616E205254432066696C650D0A000D0A68
:10FAD8005573696E67206469736B2067656F6D6520
:10FAE800747279202573200046696E6446696C65D6
:10FAF800206661696C6564207365617263680D0ACC
:10FB0800000D0A53746174757320706F72742069E4
:10FB180073202558202D204F4B000D0A5365656B27
:10FB280020746F20256C64206661696C65642025EB
:10FB380064000D0A57726974655F736563746F7248
:10FB480073206661696C202564000D0A4545505292
:10FB58004F4D206469736B206E756D626572202548
:10FB680064000D0A4469736B2073656C65637420C7
:10FB78006E756D626572202564005365656B696EEC
:10FB88006720746F20736563746F722025580D0A9F
:10FB98000046696E6446696C65206661696C6564D7
:10FBA80020726561640D0A000D0A4F70656E696EFA
:10FBB80067206578697374696E6720257320000D66
:10FBC8000A4461746120706F72742069732025582B
:10FBD800202D204F4B000D0A476F7420256C75208F
:10FBE800202D20726573657474696E67002025582E
:10FBF80020255820255820255820256C75202020A0
:10FC08000A000D0A57726F7465206469736B6E6F12
:10FC18003A20256420000D0A57616974696E6720CF
:10FC2800666F72206361726420000D0A54726967FE
:10FC3800706F696E7420697320256420000D0A4670
:10FC4800696C65202573206973206F70656E2000CC
:10FC58000D0A7274635F726561642825642C2558E7
:10FC680029000D0A4F70656E696E67206E657720F2
:10FC7800257320000D0A253032582530325820458A
:10FC8800786974200020436F6C642025582C202547
:10FC9800582C202558004E6F742061204C4946206E
:10FCA8006469736B0D0A000D0A526561642064650E
:10FCB80073637269626520000D0A46696C652025C8
:10FCC8005820697320257320000D0A4469736B203E
:10FCD800255820697320257320002041544E206147
:10FCE80073736572746564202564000D0A48737423
:10FCF80020627974657332202564000D0A204F70E4
:10FD080074696F6E732025640D0A000D0A577269B5
:10FD18007465206661696C202564000D0A5265616E
:10FD280064696E67205254430D0A000D0A416D69DB
:10FD3800676F2039313231440D0A000D0A53532FB1
:10FD480038302039313232440D0A000D0A44736BC1
:10FD580073656C20697320256420000D0A52656163
:10FD68006420256420627974657300566563746F36
:10FD7800722069732025580D0A000D0A5353383034
:10FD8800782025642025642000222A2B2C3A3B3C2D
:10FD98003D3E3F5B5D7C7F000D0A4F70656E696E6E
:10FDA800672025732020000D0A4465627567206965
:10FDB8007320256420000D0A436C6F636B20697300
:10FDC80020256420000D0A50726F746F206973201B
:10FDD800256420000D0A5265616420636F6E6669B0
:10FDE8006720000D0A46696C656E616D6520257394
:10FDF80020000D0A466F726D617474696E67200089
:10FE080072633D25752046525F25730D0A002A2A24
:10FE1800204E4F204449534B202A2A002A2A205694
:10FE28006572696679202A2A000D0A7362797465F9
:10FE38007331202564000D0A41737365727420457F
:10FE48004F49000D0A4173736572742041544E0086
:10FE58000D0A4E6F20636172642025640064657327
:10FE680063726962652E636667002F6C69666461F8
:10FE780074612E62696E000D0A456E61626C6520C0
:10FE8800505000EB76904558464154202020000DF4
:10FE98000A4D6F756E74696E6720004E6F7620206C
:10FEA800362032303232000D0A4173736572742085
:10FEB80050500020255820772041544E20004C6F88
:10FEC8006164696E672E2E2E00204944202558252E
:10FED800303258002A2A20525141202A2A00466DE1
:10FEE80074206578697420000D0A476F74204946AC
:10FEF80043000D0A476F742041544E002025643A90
:10FF080020253032580020476F742041544E000D90
:10FF18000A51532025642000446573637269626541
:10FF28000031323A30313A3235005B2532582025DB
:10FF3800645D004572726F72202564004850446900
:10FF4800736B20003C6964656E743E004E6F2063DD
:10FF5800617264004669466F2025580072633D252A
:10FF680064200044534B53454C004E414D452558A1
:10FF7800004449534B255800464154333200444508
:10FF88004255470050524F544F0052656164790002
:10FF98000D0A257320007B4552527D00302E3234E5
:10FFA800004946432000454F49200052454E200055
:10FFB800535251200044415620004E444143004EC4
:10FFC8005246440053743200464154005254430090
:10FFD80054524700434C4B002532580044300044EB
:10FFE8003100443200443300443400443500443680
:07FFF800004437002B00005C
:020000040020DA
:10000000FF0FFF0FFF0FFF0FFF0FFF0FFF0FFF0F80
:020000040030CA
:0C0000008CFFFFFC8EFFFFFFFFFFFFFFE7
:00000001FF
